:020000040800F2
:10000000F0FF0010A5EA050891750508C9EA010886
:1000100045EB050845EB050845EB05080000000029
:1000200000000000000000000000000095750508B9
:1000300099750508000000009D75050879A2000863
:1000400045EB050845EB050845EB050845EB0508BC
:1000500045EB050845EB0508B1BA0008D5BA00081C
:10006000F9BA00081DBB000841BB00087DB50008B7
:1000700091B50008A5B50008B9B50008CDB50008D0
:10008000E1B50008F5B5000845EB050845EB0508A6
:1000900045EB050845EB050845EB050865BB000881
:1000A00099CC0008F9CB0008A9CC0008E9CB0008DE
:1000B00021CC000831CC000841CC000891AF0008E9
:1000C00069C4000899AF00086DC4000845EB050835
:1000D00045EB050831260508312705085528050890
:1000E000A1BB000845EB0508D5A80508B9CC000858
:1000F00071CC0008C9CC000861CC000809B6000822
:1001000045EB050845EB050851CC000845EB050813
:10011000792905089D2A050819DE000851DE000826
:100120001DB6000831B6000845B6000859B60008EB
:100130006DB6000845EB050845EB050845EB0508DD
:1001400045EB050845EB050845EB0508A1750508D5
:1001500081B6000895B60008A9B60008C12B0508AD
:10016000A1AF000871C4000845EB050845EB050880
:1001700045EB050845EB050845EB050845EB05088B
:0801800045EB050845EB0508FD
:1080000010B40C4B4FF0E02C1A68DCF8180019681B
:108010008A42F9D159688842F6D89C684FF47A713F
:1080200001FB04F31B1AB3FBF4F35DF8044B01FBF3
:108030000230704798190020074BD0F8E4105B68B5
:10804000D0F8F0205B1A9A42B8BFC0F8F030012394
:1080500080F81C3100207047001000E0B04A00EBAF
:10806000800102EBC1012DE9F041CB685B68B3F8F8
:1080700014C01CF0010F4FEA800E40F082805FFABE
:108080008CF4A6074DD5BFF35F8F91F82840012CE3
:10809000E5B200F0F7804FEA400C198BBFF35F8F19
:1080A0000EEB000102EBC10191F82840022C00F018
:1080B00017810EEB000102EBC10191F82840032C5F
:1080C0000AD191F82A1039B10CEB0001114491F852
:1080D0008440002C40F06381998889B241F480612A
:1080E00099800CEB0001114491F986100EEB00040D
:1080F00002EBC40494F8284001348C420FD184442C
:10810000944400218CF884109CF88510002940F0DC
:10811000E080704402EBC000002380F82530BDE809
:10812000F08165076BD400EB4007174414F040045E
:108130001FFA8CF697F986504FEA400C00F0E68063
:108140001E8A0C6BF6B26655EEB2741C64B291F8DE
:10815000288087F88640E51CA845214600F0458127
:108160000EEB000502EBC50595F82850AC42BDD1D9
:108170000CEB00011144023676B281F8866031467C
:10818000B4E71C8824F400642404240C1C801C889C
:10819000A4B244F480641C8000EB4004144491F8C1
:1081A0002A50002684F886604FEA400C002D56D0F5
:1081B00094F88440002C4ED00EEB000102EBC1017C
:1081C000844491F828109444012402298CF88440B6
:1081D00004D1198889B241F4006119800EEB0001C5
:1081E00002EBC10191F8261041F0010119820EEB5A
:1081F000000302EBC30292F82830BDE8F08100EBE7
:108200004005154491F82A40012685F8856000FA5A
:1082100006FC002C7ED095F88440002C40F0828033
:108220000EEB000102EBC10191F82910002900F0CA
:10823000B98019880CEB0004144489B241F4007130
:10824000198094F88610013149B284F886101C8890
:10825000E705FCD44AE791F82710FF29ACD00EEBD4
:10826000000102EBC10191F8264004F0FE041C82DB
:1082700091F82730FF2BBAD084449444FF238CF824
:108280008630B4E791F82A1000293FF404AF00EBE0
:10829000400111444FEA400C91F88440002C3FF417
:1082A000FCAE1C8824F480642404240C1C80BFF3DE
:1082B0005F8F1C8B1C8881F88550A4B244F4007435
:1082C0001C809C8891F98610A4B244F480649C8040
:1082D0000CE7998821F440710904090C998018E78A
:1082E00091F82A1000293FF4E4AE0CEB0001114490
:1082F00091F88440002C3FF4DCAE1C8891F9861084
:1083000024F480642404240C1C8041E036062FD41D
:108310002946EBE695F88410002981D089E700BF53
:108320009819002091F828400E6B022C1C8847D920
:1083300024F480642404240C1C801F8A95F9864050
:10834000FFB237550F6B198889B241F4007119805B
:10835000E4B21E8A611C49B2F6B27E54A11C9C880C
:10836000A4B249B244F4806485F886109C806EE71C
:108370006E1C41D0CC6A665D6C1CF5B21D8291F812
:10838000285064B2A54287F8864021467FF4AEAEFD
:108390009C8824F480642404240C9C80A6E691F933
:1083A0008610F5E7198889B241F4807119800CEBC9
:1083B00000011144012481F8844091F9861046E7B8
:1083C000A4B244F400741C801F8A95F98640FFB261
:1083D0003755E4B20F6B1E8A611C49B2F6B27E5467
:1083E000E11C49B285F8861031E79D8825F4806547
:1083F0002D042D0C9D80B3E687F8864091F8274028
:10840000E4B21C8291F82A4024B991F8281000297E
:108410007FF4EDAE998821F480610904090C9980FC
:10842000E5E600BF10B404698269E468416814603D
:1084300000234024C2E90234446993630C31C2E949
:108440000433C2E90633C2E90833C2E90A33C2E998
:108450000C33516094B1C269E46893634FF4803087
:10846000C2E90041C2E90233C2E90433C2E906337A
:10847000C2E90833C2E90A03C2E90C335DF8044BD0
:10848000704700BFD0E9001300221A60037D1F2B44
:1084900007D9203B202202FA03F343F01803CB60F4
:1084A0007047202202FA03F343F018038B607047F1
:1084B0001B4B016803F57D7C02E02C3363452CD017
:1084C0001A688A42F9D170B593F804E0427996456A
:1084D0000BD02C33634505D01A688A42F4D02C3374
:1084E0006345F9D14FF0FF3070BD9E468468DEF8D9
:1084F0000C50A5424FF0000208D00132032A0EF1C1
:108500000C0EE6D0DEF80C50A542F6D1DEF8105085
:10851000C668B542F1D150B270BD4FF0FF30704720
:1085200050080608002A4FEA014C30B503460ABF3E
:10853000E6468E468C4600F1C005002419689A680C
:1085400041EA0C0142EA0E029A60C3E900140C33BE
:10855000AB42F3D1D0F8C030C0F8C44043EA0E03B8
:10856000C0F8C030C0F8C84030BD00BF8369196989
:10857000B3F80CC00A6830B49C6822F00102246889
:108580000A60A28992B222EA0C02A281027D0068EE
:108590001F2A06D94568203A082494402C4245D029
:1085A000FEE70568082494402C42F9D1202404FAFF
:1085B00002F28260264A1278002A35D01A7E012AF9
:1085C00039D0D3F8F4200132C3F8F420EFF311814D
:1085D000502282F3128858685C6C026822EA040216
:1085E0009C6C2243C9B2026081F31188D3E90C402C
:1085F0001A6999681D6C096814605061D3E90E40CE
:10860000546090600024B3F8A800D5604C62C86242
:1086100010680124204310601C7683F8F1408A8999
:108620009B8913439BB28B8130BC7047202404FA92
:1086300002F2C260BEE7002283F8F120D3F8F8000E
:108640000A68013022F00102C3F8F8000A60EBE783
:108650000400001010B40C4C6368002B11DD0020E6
:1086600004F1080C0146DCF8A03003F1C0025960A7
:108670000C339342FBD16368013083420CF5807C5C
:10868000F1DC5DF8044B704704000010F0B5414C7C
:1086900004EB401393F8243403B9F0BD3E4B93F838
:1086A0008D5093F88E2095424FEA401C0CD002EB7F
:1086B000420E03EBCE0E9EF89060771E012F4FEA1C
:1086C000420E58D9032E51D004EB0C00A0F8081428
:1086D000EFF31182902383F3128890F80A34B0F8F4
:1086E000081443EA41030021D2B29BB280F80A1475
:1086F00082F311882178D0F820441A0982EA1322E3
:108700005A40C9B1D0F80C14D4F8A040D2431B0190
:108710009BB202F00F0201208840134304F1C00114
:108720005A0013F4004F93B202D1626802436260B0
:108730000C34A142F4D1F0BDD0F80C14D4F8A04010
:108740001B0110319BB202F00F020120884013433D
:1087500004F1C0015A0013F4004F93B202D16268D1
:10876000024362600C34A142F4D1F0BD561C06F005
:108770000306AE42A8D0964403EBCE03184490F80B
:108780009D100029A0D004EB0C03012283F80A24D9
:108790009AE700BF0400001098190020704700BF3E
:1087A000024B03EB401393F82504704704000010BC
:1087B0004368B0F8502010B41A83EFF311825023AD
:1087C00083F312884168446C0B6823EA0403C46C89
:1087D0002343D2B20B6082F31188D0E9074182684B
:1087E000036912681C605961D0E909415C60C46A80
:1087F0009960B0F86010DC600023D1625DF8044B32
:108800000376704710B4037D02681F2B09D95468A2
:10881000203B202101FA03F31C4215D15DF8044BE3
:1088200070471468202101FA03F31C42F6D00D4969
:108830004068002481F8F04001685DF8044B21F0A5
:10884000010101609360704706494068002481F887
:10885000F04001685DF8044B21F001010160D36034
:10886000704700BF98190020122301480B80704701
:1088700088010020042301480B8070479C010020E0
:108880001C48D0F8103AD0F8182A10B59B184FF0B1
:108890001A040C8001D1184810BD174AD0F8140AE8
:1088A00002F1100411464FF0000E4FEA137CB3F1B1
:1088B000204F34BF0CF1300C0CF1370C81F802C0A2
:1088C00081F803E002318C424FEA0313EDD102F14B
:1088D00008040021030FB0F1204F34BF3033373389
:1088E0009374D174023294424FEA0010F2D10248DC
:1088F00010BD00BF0070FF1FA0010020D0E90920BB
:10890000131A58425841704790F84F3830B53BB968
:1089100090F84D1890F84E380124DAB2914200D800
:1089200030BDB0F8565804FA03F22A43A0F856288E
:108930000133F2E70379024613F0010006D0D2E9D1
:108940000731D2685B1A013A03EA0200704710B59A
:10895000037913F0010304460ED0FFF7EBFF034643
:1089600050B1226A6369E1689B5C0132B2FBF1F0AD
:1089700001FB1022DBB22262184610BD03799B076F
:108980000AD5436A8269D154436A02690133B3FB51
:10899000F2F102FB11334362704770470171704777
:1089A0000379014613F0020007D00B69D1E90921D0
:1089B000013B521A1A40D2B2981A704782B01D4B2E
:1089C0001D49002201920193019B04330193019BF5
:1089D0001A688B6803F00C03042B02D0082B05D017
:1089E000164A174BC3F8F42002B0704748684B682A
:1089F000400203F03F0314D44A681049B1FBF3F37B
:108A0000C2F3881203FB02F20B4B5B68C3F3014312
:108A100001335B00B2FBF3F2094BC3F8F42002B060
:108A200070474968B2FBF3F2C1F3881303FB02F20B
:108A3000EAE700BF50280040003802400024F4005C
:108A4000981900204A484B494B4BDFF830C12DE9BB
:108A5000F04F4FF0010A4FF002094FF004080827C9
:108A60001026202540244FF0800E30F8022B12F003
:108A7000010F03D01960A3F804A0083312F0020F0D
:108A800003D01960A3F80490083312F0040F03D048
:108A90001960A3F80480083312F0080F02D019609F
:108AA0009F80083312F0100F02D019609E800833A7
:108AB00012F0200F02D019609D80083312F0400F91
:108AC00002D019609C80083312F0800F03D0196027
:108AD000A3F804E0083312F4807F05D04FF4807BC4
:108AE0001960A3F804B0083312F4007F05D04FF4E6
:108AF000007B1960A3F804B0083312F4806F05D02E
:108B00004FF4806B1960A3F804B0083312F4006FBF
:108B100005D04FF4006B1960A3F804B0083312F4C9
:108B2000805F05D04FF4805B1960A3F804B0083370
:108B300012F4005F05D04FF4005B1960A3F804B095
:108B4000083312F4804F05D04FF4804B1960A3F81E
:108B500004B00833D20B04D04FF4004219609A805D
:108B6000083301F5806161457FF47FAFBDE8F08F88
:108B7000440C060800000240901A00200018024031
:108B800010B584464FEA810E102312F4004F14BF33
:108B90000E2407245200013BCCF8004092B2F4446A
:108BA000F3D100EB81128C01035142F821301220E5
:108BB00010BD00BF10B584464FEA810E0424130B8C
:108BC00003EB430318331201013CCCF8003092B29E
:108BD000F444F4D100EB01130A01845043F821401E
:108BE000062010BD704700BF704700BF034B00EB6D
:108BF000400003EBC00393F8190570470400001010
:108C0000064B93F8C825824283BF00EB400003EB7C
:108C1000C003D3F81C050020704700BF04000010FB
:108C20001D4B93F8CC25AAB3D3F8081509B1002041
:108C30000860012A2ED0D3F8201509B10020086061
:108C4000022A27D0D3F8381509B100200860032A7A
:108C500020D0D3F8501509B100200860042A19D09B
:108C6000D3F8681509B100200860052A12D0D3F89E
:108C7000801509B100200860062A0BD0D3F898159A
:108C800009B100200860072A04D0D3F8B0350BB131
:108C900000221A60704700BF040000101D4B93F8BB
:108CA000CC25AAB3D3F8081509B100200860012A21
:108CB0002ED0D3F8201509B100200860022A27D051
:108CC000D3F8381509B100200860032A20D0D3F862
:108CD000501509B100200860042A19D0D3F868158E
:108CE00009B100200860052A12D0D3F8801509B117
:108CF00000200860062A0BD0D3F8981509B100208F
:108D00000860072A04D0D3F8B0350BB100221A60EE
:108D1000704700BF04000010C24B93F83230002BA4
:108D200040F05781C04B93F8CC25002A00F05181C8
:108D300093F8181530B500294ED1D3F80815002046
:108D4000012A086047D993F83015002967D1D3F874
:108D500020150020022A08603DD993F84815002903
:108D600040F0D080D3F838150020032A086032D9AB
:108D700093F86015002940F0E880D3F850150020E2
:108D8000042A086027D993F87815002940F0FF805D
:108D9000D3F868150020052A08601CD993F89015AF
:108DA000002940F01781D3F880150020062A0860BA
:108DB00011D993F8A81500295BD1D3F89815002094
:108DC000072A086007D993F8C025002A76D1D3F87E
:108DD000B03500221A6030BDD3F80C158A0AA2F50E
:108DE0008012522A40F218814FF0FE0CEFF31180EE
:108DF000502282F312888D4C4D6A8A8A4FF02C0ED5
:108E00000EFB0C4C92B2013542F00102CCF820541A
:108E1000C0B28A8280F3118893F8CC258DE7D3F80D
:108E200024158A0AA2F58012522A40F203814FF0DB
:108E3000FE0CEFF31180502282F312887B4C4D6AB6
:108E40008A8A4FF02C0E0EFB0C4492B2013542F090
:108E50000102C4F82054C0B28A8280F3118893F8CA
:108E6000CC25D3F820150020022A08603FF675AF04
:108E7000B1E7D3F89C158A0AA2F58012522A00F2B3
:108E8000F2806B48024492F800C4EFF31180502244
:108E900082F31288654C4D6A8A8A4FF02C0E0EFBC5
:108EA0000C4492B2013542F00102C4F82054C0B221
:108EB0008A8280F3118893F8CC257EE7D3F8B41525
:108EC0008A0AA2F58012522A9BBF594812184FF005
:108ED000FE0C92F800C4EFF31180502282F3128846
:108EE000524C4D6A8A8A4FF02C0E0EFB0C4492B203
:108EF000013542F00102C4F82054C0B28A8280F3E6
:108F0000118864E7D3F83C158A0AA2F58012522A28
:108F100040F295804FF0FE0EEFF31180502282F365
:108F20001288424C4D6A8A8A4FF02C0C0CFB0E447E
:108F300092B2013542F00102C4F82054C0B28A82D4
:108F400080F3118893F8CC250CE7D3F854158A0ADE
:108F5000A2F58012522A77D94FF0FE0CEFF3118060
:108F6000502282F31288314C4D6A8A8A4FF02C0EBF
:108F70000EFB0C4492B2013542F00102C4F82054B9
:108F8000C0B28A8280F3118893F8CC25F5E6D3F835
:108F90006C158A0AA2F58012522A5AD94FF0FE0C9B
:108FA000EFF31180502282F31288204C4D6A8A8A96
:108FB0004FF02C0E0EFB0C4492B2013542F0010230
:108FC000C4F82054C0B28A8280F3118893F8CC256B
:108FD000DEE67047D3F884158A0AA2F58012522A79
:108FE0003CD94FF0FE0CEFF31180502282F312882F
:108FF0000E4C4D6A8A8A4FF02C0E0EFB0C4492B236
:10900000013542F00102C4F82054C0B28A8280F3D4
:10901000118893F8CC25C6E60548024492F800C4AE
:10902000E4E600BF88010020040000109819002029
:10903000500806080D48024492F800C4F9E60B48AF
:10904000024492F800E467E70848024492F800C43A
:1090500084E70648024492F800C4A1E703480244AA
:1090600092F800C4BFE74FF0FE0C0EE75008060868
:1090700000EE100AB8EE400A704700BFBCEEC00A0E
:1090800010EE103A98B27047072809D8054B8C2289
:1090900002FB0033B3F8D005B0FA80F04009704706
:1090A0000020704704000010072806D8034B8C22CC
:1090B00002FB0033012283F8D22570470400001020
:1090C00070B53F4C8C2303FB004393F8DF3503B9A5
:1090D00070BD3C4B93F88DE093F88E2096450CD0F4
:1090E00002EB420C03EBCC0C9CF890506E1E012E50
:1090F0004FEA420C44D9032D3DD08C2202FB0042A2
:10910000A2F8D015EFF31181902383F31288B2F8FF
:10911000D05592F8D23543EA45030025C9B29BB237
:1091200082F8D25581F311881A09217882EA132234
:109130005A4001B1D2431B019BB294F8341AD4F8BF
:10914000305A02F00F021A438C2303FB004431BB58
:109150000121D4F85806A847D4F85416B4F8DC55C1
:109160008A8AD4F850362A438A8258601A6842F0B4
:1091700001021A6070BD551C05F003057545BCD091
:10918000944403EBCC03034493F89D100029B4D01E
:109190008C2303FB0043012283F8D225ADE7D4F8EA
:1091A000D835D4F854165B79086903F0FC031844E9
:1091B0000421A847D4F854368000988170BD00BFC0
:1091C00004000010981900207AE700BF072808D88B
:1091D000044B03EB401393F8242412B1012283F8CB
:1091E0000A24704704000010072808D8054B03EB39
:1091F0004013B3F80804B0FA80F04009704700202B
:10920000704700BF04000010054B93F8C825824248
:1092100086BF03EB4013D3F814040020704700BF4F
:109220000400001038B5074BD3F860361B6A1446AB
:109230000D4698474FF4007302682A6000202360AF
:1092400038BD00BF9819002008B5064BD3F860362A
:1092500023B15B699847013840B208BD4FF0FF3039
:1092600008BD00BF98190020002070472DE9F0418B
:109270000BB3144C16460F4603EB0208D4F86016E5
:1092800000238D681A4639463046A8470028F5D095
:10929000D4F86036002BFBD05B6998470028F7D0E4
:1092A0000136B04507F50077E8D12368C4F8643685
:1092B0000020BDE8F081034C2368C4F86436002028
:1092C000BDE8F081981900202DE9F0413BB3174C1F
:1092D00016460F4603EB020804E0D4F8601619B1F5
:1092E0004B699847D4F860160D6900231A46394631
:1092F0003046A8470028F0D1D4F86036002BFBD0C8
:109300005B6998470028F7D00136B04507F500772C
:10931000E8D12368C4F864360020BDE8F081034C2E
:109320002368C4F864360020BDE8F0819819002055
:1093300000207047034B93F88C06003818BF0120BB
:10934000704700BF98190020826D136A5B681B7814
:10935000FF2B09D090F8F030013B5BB2002B80F876
:10936000F03006DD01207047082380F8F03000203F
:109370007047136A5B68002202201A70704700BFB2
:10938000836D1B6A5B681B78FF2B0AD190F9F03064
:10939000002B03F1FF3280F8F020D4BF022001201F
:1093A00070470020704700BF30B540F040030022F6
:1093B00063F307020B0E63F30F220B0C99B063F3F8
:1093C00017420446080A60F31F620023029201223A
:1093D000CDE90D33CDE91333049306928DF81C309B
:1093E0000A938DF8303010928DF858208DF8443063
:1093F000082215931793164B08930DEB0203154D96
:109400000993062395208DF80C100B930DF107019D
:109410006B4405918DF80D000F9304A90E4B85F850
:10942000582705F5D860129348F0EEFAD5F8C02613
:10943000136A002BFCD19DF80730FF2B00D01CB91C
:109440009DF8060019B030BD4FF0FF30FAE700BFBD
:10945000499300089819002081930008836D1B6AC6
:109460005B681B78FE2B0CD0FF2B08D190F9F030F5
:109470005A1E002B80F8F02001DD012070470220E9
:1094800070470020704700BF30B597B01E4C1F4D8D
:1094900008909FED1B7B002308460DF10702082171
:1094A000CDE90232CDE906530122CDE91033CDE9F1
:1094B000123384F858178DF8143009908DF828303D
:1094C0000B938DF83C3015936944022304F5D86062
:1094D0000E938DED0C7B04928DF8502048F094FA99
:1094E000D4F8C036186A0028FCD19DF80730FE2B4E
:1094F00003D0FF2B0CBF0120022017B030BD00BFEE
:109500000000000000000000981900205D94000891
:1095100030B52C4C9DB0002301220020002104F521
:10952000D865CDE90C01CDE91601CDE912324FF035
:10953000FD0CC4F888368DF83C3010938DF850300F
:10954000159318931A930CA90DF1060328460E9251
:109550008DF864208DF806C0119348F055FAD4F8C0
:10956000C026136A002BFCD1174906910DF10700A4
:109570000122039002A92846CDE9073302938DF812
:10958000143009930B9304928DF8282084F85827FF
:1095900048F03AFAD4F8C036186A0028FCD19DF891
:1095A0000730FF2B07D02368C4F87C36092384F8E2
:1095B0008C361DB030BD0423022084F88C361DB0DB
:1095C00030BD00BF9819002081930008034B93F829
:1095D0008C06032894BF00200120704798190020B2
:1095E000004870472820002030B4184B00209C7B96
:1095F00014B11D688D4206D001300B2803F1100311
:10960000F5D130BC7047B2B1114B03EB40218A4217
:1096100018D0104B93F8E42712B9012283F8E427FD
:109620000D4B01225A7000F5B17003EB00130122BB
:109630009A7130BC7047084B00F5B17003EB001312
:109640009A71DEE7022CE4D1183BECE76C6F002046
:109650006C590020546900205459002030B41D4C2E
:10966000002384F8D03604F5C36004E001330B2BEB
:1096700000F1100015D005688D42F7D190F80EC0AA
:10968000BCF1030FF2D1C2B1134901EB4320824276
:1096900009D1A1F1180203F5B17302EB0312012302
:1096A000937130BC704794F8E42712B9012284F812
:1096B000E4270A4A01215170EDE70849D4F8CC2685
:1096C00003F5B17301EB0313013204219971C4F85E
:1096D000CC26E6E7546900206C590020545900203C
:1096E000A8B183681BB10E4B07229A7070470C4AD1
:1096F0001178D36003294FF0040014BF4FF4807138
:109700008021C2E901111361137590707047044AFA
:1097100002F580510123537081F8E437704700BF90
:109720005459002030B585B068464DF0CBFB0F484A
:109730000F4AD0F8FC10009B0E4D41F08071C0F82C
:10974000FC10002400F1C840C2F8B05FA0F565002D
:1097500054601168084CA0F67D60A0FB030341F043
:1097600001019B0CA360116005B030BD00ED00E06D
:10977000001000E055CEACC5981900202DE9F04F3F
:10978000A84CA94D83B081464F1E102651F05AFDBA
:109790004FF4FA784FF0E0214FF47A7C4FF0010E4D
:1097A0006B68C3F30803002B40F05E81EFF3118375
:1097B000002B40F059812368886922689342FAD1CE
:1097C00062689042F7D8A2680CFB02FAAAEB000A82
:1097D000BAFBF2FA0CFB03AA6B68C3F30803002B75
:1097E00040F02481EFF31183002B40F01F812368A8
:1097F000886922689342FAD162689042F7D8D4F817
:1098000008B00CFB0BF2121AB2FBFBF20CFB0323A9
:10981000A3EB0A03B3F57A7FDED3B8F10108BFD119
:10982000D4F8681794F860C7D4F8642731B10B688E
:1098300088881CF0020F14BF1883588332B11CF0C3
:10984000010F9088136840F02D82188348464FF02E
:10985000010C4FF0E02359B1D1F800E08988DEF81F
:10986000148011EA080F14BFAEF81A10AEF81810E1
:1098700042B111689288D1F814E012EA0E0F14BFB9
:109880004A830A83B4F87027002A40F07F8194F855
:109890007817D4F87427002940F0718112B111684B
:1098A00092884A83FA21BA464FF47A7E01900F4695
:1098B0006A68C2F30802002A40F02C81EFF311829B
:1098C000002A40F027812268986921688A42FAD1EB
:1098D00061688842F7D8A1680EFB01FBABEB00087A
:1098E000BB46B8FBF1F80EFB02886A68C2F30802B7
:1098F000002A40F0DF80EFF31182002A40F0DA8086
:1099000021689F6922689142FAD162689742F7D82C
:10991000A0680EFB00F2D21BB2FBF0F20EFB01229C
:10992000A2EB0802B2F57A7FDFD35F46013FBFD1D9
:10993000D4F868170198574641B10A688988D2F867
:1099400014E011EA0E0F14BF51831183D4F8641789
:1099500041B10A688988D2F814E011EA0E0F14BFE9
:1099600051831183B4F87027002A40F0F08094F8F6
:109970007817D4F87427002940F0FA8012B11168E2
:1099800092880A83FA21BA464FF47A7E01900F46F4
:109990006A68C2F30802002A40F09F80EFF3118248
:1099A000002A40F09A802268986921688A42FAD198
:1099B00061688842F7D8A1680EFB01FBABEB000899
:1099C000BB46B8FBF1F80EFB02886A68C2F30802D6
:1099D000002A5CD1EFF31182002A58D121689F69D7
:1099E00022689142FAD162689742F7D8A0680EFBCC
:1099F00000F2D21BB2FBF0F20EFB0122A2EB080236
:109A0000B2F57A7FE1D35F46013FC1D101980138B9
:109A1000C0B2FF28574600F0CD80D4F86817D4F8BC
:109A2000642718E79819002000ED00E0EFF3118398
:109A300086F31288D1F818B00A69D00344BFC4F87D
:109A40005CE7D1F818B02068D4F85C27DBB283F368
:109A500011880244A0680CFB00F3A3EB0B03B3FBDB
:109A6000F0F30CFB0233D3E6EFF3118286F3128896
:109A700088690B69DB0344BFC4F85CE78869236825
:109A8000D4F85CA7D2B282F3118853449BE6EFF37B
:109A9000118286F312889F691969C90344BFC4F80B
:109AA0005CC79F692068D4F85C17D2B282F3118832
:109AB00001449BE7EFF3118286F312889F691969CD
:109AC000C90344BFC4F85CC79F692068D4F85C1719
:109AD000D2B282F3118801441AE7EFF3118186F3C1
:109AE000128898691A69D20344BFC4F85CC79869A0
:109AF0002268D4F85C87C9B281F31188A168424416
:109B00000EFB01F8A8EB0008BB46B8FBF1F80EFB12
:109B100002885AE7EFF3118186F3128898691A696F
:109B2000D20344BFC4F85CC798692268D4F85C8744
:109B3000C9B281F31188A16842440EFB01F8A8EB79
:109B40000008BB46B8FBF1F80EFB0288CDE6D4F85E
:109B50009027002A3FF416AFB4F89427002A3FF468
:109B600011AFD4F87C270021116084F88D1709E724
:109B7000002A3FF407AF116892884A8302E7002A5F
:109B80003FF490AE116892880A838BE6D4F8902750
:109B9000002A3FF487AEB4F89427002A3FF482AE3F
:109BA0004149B1FBF2F1D4F87C274910116084F8E7
:109BB0008DC777E64FF47A7E4FF0E021F4464FF000
:109BC00001086B68C3F30803002B58D1EFF311832E
:109BD000002B54D12368886922689342FAD16268C5
:109BE0009042F7D8A2680CFB02FAAAEB000ABAFB73
:109BF000F2FA0CFB03AA6B68C3F308030BBBEFF389
:109C00001183F3B92368886922689342FAD16268A4
:109C10009042F7D8D4F808B00CFB0BF2121AB2FB42
:109C2000FBF20CFB0323A3EB0A03B3F57A7FE2D329
:109C3000BEF1010EC5D1013FBFF4A8AD03B0BDE830
:109C4000F08FEFF3118386F31288D1F818B00A6908
:109C5000D20344BFC4F85C87D1F818B02068D4F8A8
:109C60005C27DBB283F311880244A0680CFB00F38D
:109C7000A3EB0B03B3FBF0F30CFB0233D3E7EFF3DF
:109C8000118286F3128888690B69DB0344BFC4F82C
:109C90005C8788692368D4F85CA7D2B282F3118804
:109CA00053449FE75883D1E540420F002DE9F0412E
:109CB0001D4CDFF87C801D4F82B004F540750126F5
:109CC00002E00834A54224D094F90630002BF8D1E4
:109CD000206800F13F4303F57E0308EB932393F8DC
:109CE00054345A09032A03F01F0306FA03F317D06A
:109CF000042A11D0022A02D17A6C13437B64002318
:109D0000A1881A46CDE90036083452F0D9FEA542A2
:109D1000DAD102B0BDE8F0813A6B13433B63EEE762
:109D20003A6C13433B64EAE7901A00200038024083
:109D30005008060809494B6C10B5094C43F48043A0
:109D40004B644022002104F5F36056F045FB4FF0D0
:109D5000FF33C4F8D837C4F8DB3710BD00380240F1
:109D6000981900202DE9F0411348144D4FF41A7250
:109D7000002156F031FB4FF00008A5F25C4705F6D4
:109D8000880440F2222655F82810002354F8332086
:109D900091420BD001330E2BF8D1002008F10708B7
:109DA00050F05CFEB045EED1BDE8F08107EBC30397
:109DB00093F8E80CF2E700BF901D0020AC0C0608F9
:109DC0002DE9F843038AB0F80C801FFA88F818EAE6
:109DD000030829D005460E464FF00047B8FA88F32D
:109DE00027FA03F2D24391B21B3B298208EA020808
:109DF000042B16D8DFE803F0352C231A0300B36ACE
:109E0000002B37D003F1FF3900231FFA89F9B36221
:109E1000746A34B123682046494698476468002C28
:109E2000F8D1B8F1000FD9D1BDE8F8837068696B3B
:109E3000036889B29847B8F1000FCFD1F4E7B06852
:109E4000A96B036889B29847B8F1000FC6D1EBE758
:109E5000F068E96B036889B29847B8F1000FBDD18B
:109E6000E2E73069296C036889B29847B8F1000FBE
:109E7000B4D1D9E7EB6A1FFA83F9C9E770B50B4C87
:109E800005460726013E00D170BD94F9000015F08B
:109E9000C7F9031E08DBEA1861789171A178E954CB
:109EA000052BDCBFE37813730434EBE7A415060835
:109EB00010B5274B93F88D2093F88E309A4242D1FB
:109EC000244A92F8F80AF8B192F8344A02F6382394
:109ED00000EB4000D2F8382A03EBC000B4B140F2E6
:109EE0000D3C00E01A6899689C894C600C6844F04D
:109EF00001040C60A2F848C09189183389B241F47A
:109F0000807183429181EDD110BD1A68118821F0D2
:109F1000800109041833090C118033F8141CD16234
:109F2000118889B241F0800111805462B2F80CC0EE
:109F300033F8041C41EA0C0189B28342918123F871
:109F4000044CE2D110BD53F0B7F80028B8D110BDD1
:109F500098190020040000102DE9F041224C94F8DB
:109F60008CC6BCF1040F0746884616461D4609D02C
:109F7000BCF1080F02D00020BDE8F081FFF7C8FA5D
:109F80000228F8D194F88236B3B139461120FFF790
:109F90000BFAC0B2B8B90522236884F88C26C4F83D
:109FA0006886C4F86C76C4F87466C4F87856C4F849
:109FB0007C360120BDE8F08179021120FFF7F4F929
:109FC000C0B20028E7D0D4F8C026136A002BFCD119
:109FD00051F0F8FDD4F8C836002BCCD01A689B8815
:109FE00013830020C8E700BF9819002010B504466D
:109FF00055F0C2FC81B22046BDE81040FEF746BBDA
:10A0000010B5044655F0B8FC81B22046BDE81040BA
:10A01000FFF756B838B50B4D00EB400005F5A163CE
:10A0200003EBC00393ED027AD3ED037AE7EE007AF7
:10A03000C4002544B0EE670A55F09EFCD5F80835FB
:10A04000186038BD040000100A4608B5054920B95B
:10A0500005484DF031FA034808BD04484DF02CFA8C
:10A06000004808BD78210020E88206081083060811
:10A0700010B5044C04480A4621464DF01DFA20460E
:10A0800010BD00BF782100203883060810B5044CAD
:10A0900004480A4621464DF00FFA204610BD00BF85
:10A0A000782100204C83060810B5044C04480A4669
:10A0B00021464DF001FA204610BD00BF7821002056
:10A0C00058830608F8B5A0F668042379DB0725D580
:10A0D000657994F84C3805F001073D46FBB1D4F89A
:10A0E00048341A68D36A5B08536294F8503823B135
:10A0F000B4F85A380133A4F85A38606C85F001017D
:10A1000050F06AF9012384F84F38002384F84D3861
:10A1100084F84E38A4F8563884F84C38F8BD94F8D2
:10A120004F68012E04BF94F84D3884F84E3820460D
:10A13000FEF7EAFB4EB9012384F84F3887EA0301A2
:10A14000606CBDE8F84050F047B9002384F84F3800
:10A150003946F5E78069002836D003681A6A127B11
:10A160002ABBD3E904125B68496872B110B4546821
:10A1700000220A6022609A885DF8044B22F00302F4
:10A180001204120C9A8047F0C9BD1A891206FCD439
:10A190001A89D20709D400220A609A8822F00202A2
:10A1A0001204120C9A8047F0B9BD9A89F0E78268D0
:10A1B000002AD6D0116892880A83D3E904125B681A
:10A1C0004968002AD2D1E0E7704700BF806900B932
:10A1D0007047016830B4D1E904424B6864687AB1D1
:10A1E0005568002222602A609A8822F00302120435
:10A1F000120C9A800B6A1B7BA3B930BC47F08EBD52
:10A200001A891506FCD41A89D20714D400222260B8
:10A210009A8822F002021204120C9A800B6A1B7BAD
:10A22000002BEAD08368002BE7D01A689B88138341
:10A2300030BC47F073BD9A89E5E700BF10B50D4CFF
:10A24000D4F864373BB194F8602799881B68D2072B
:10A2500054BF198359834FF055FCD4F86036002B56
:10A26000FBD05B6998470028F7D02368C4F86436B0
:10A27000002010BD9819002010B4EFF311821023B4
:10A2800083F31288084B19684FF0E0200131196000
:10A29000816959600024C3F85C470369D3B283F332
:10A2A00011885DF8044B70479819002010B4EFF343
:10A2B0001181102383F312884FF0E022C9B2946910
:10A2C000136913F4803F0C4B1EBF0120C3F85C07D9
:10A2D00094691868D3F85C2781F31188996802445F
:10A2E0004FF47A7000FB01F31B1B5DF8044BB3FBCA
:10A2F000F1F300FB0230704798190020234B5B6894
:10A30000C3F3080310B4DBB9EFF31183C3B9204BD7
:10A310004FF0E02C1A68DCF8180019688A42F9D16D
:10A3200059688842F6D89C684FF47A7101FB04F3AF
:10A33000181AB0FBF4F05DF8044B01FB0200704703
:10A34000EFF31181102383F312884FF0E022C9B29A
:10A350009469136913F4803F0D4B1EBF0120C3F8AD
:10A360005C0794691868D3F85C2781F311889968B1
:10A370004FF47A73024403FB01F0001B5DF8044BB9
:10A38000B0FBF1F003FB0200704700BF00ED00E0FE
:10A39000981900202DE9F04F037D02681F2B83B030
:10A3A000044609D95068A3F120052021A9400142A3
:10A3B00007D103B0BDE8F08F106820219940014219
:10A3C000F7D04749474D4968A769C5F8FC1A8C2161
:10A3D00001FB075195F834CAD1F8D8050668BCF1DD
:10A3E000000F18D1D1F85006B1F8DCC5016821F092
:10A3F00001010160B18989B221EA0C01B18129789A
:10A40000B9B91F2B60D9A3F1200120238B40D36061
:10A4100003B0BDE8F08F0069016821F0010101601F
:10A42000B18921F480710904090CB18129780029CE
:10A43000E7D04FF08C0808FB07F805EB0803019301
:10A44000D3F850A6DFF8A0B050464CF09DFD019B1C
:10A45000012283F82426D5F8043B08F11809D944D1
:10A46000002B38D033889BB243F08003338008F14F
:10A4700074084FF0FF330BEB0801F36230464CF0E9
:10A480006DFF8C2303FB0757494600235046C7F84E
:10A49000F4354CF00FFED7F8503616225A601A6881
:10A4A00042F001021A60D7F8D825B7F8DC351268F7
:10A4B00091890B439BB293810949237D49682268A6
:10A4C000C5F8001B1F2B9ED8202101FA03F39360CF
:10A4D00003B0BDE8F08FFFF711FFC5F8040BC1E72B
:10A4E000001000E004000010D40500102DE9F8432E
:10A4F000FFF704FF204F214E7C6805464FF000080F
:10A50000002C2DDD00231A4607EB0321013391F8BF
:10A51000F9109C4242EA0102F6D142EA08095FFAC8
:10A5200089F990467368C3F30803B3B9EFF3118355
:10A530009BB9FDF765FD401BB0F5FA6F02DCB8F181
:10A54000000FDDD1B9F1000F04D00D4B93F8DF28D7
:10A55000542A09D04846BDE8F883FFF7A7FEEAE78A
:10A56000C1464FF00008DDE7B3F8E4280132A3F854
:10A57000E4284846BDE8F8830400001000ED00E040
:10A5800098190020AB4B1B780BB9012070472DE9BF
:10A59000F04FDFF8B4B2A849DBF80020A74BA1FBCD
:10A5A00002125209A3FB0213DB08A24987B003EB96
:10A5B0008303A2EB430391F8C825049201F6083403
:10A5C000DAB2059204EB8307002201F6E853019307
:10A5D00001F5816A9046049B984500F00981DAF8FC
:10A5E0001820DAF80490D2F8E830D2F8EC60029340
:10A5F000FFF784FE029B03904FEA890C9BF8DF98DB
:10A600009BF8F0080CF1085C06F180610CEB431C30
:10A610003939B9F1540F0CEB81110CEB801301D1D6
:10A62000ABF8E608994240F279811A68002A00F0F6
:10A630006D811A6C002A00F07F81D3F88020002AF7
:10A6400000F07C81D3F8C02003F58073002AE9D1A3
:10A65000A3EB0C0C99424FEAAC1240F25F81B11AA5
:10A6600045294FF0000628BF45213046B64603EB8A
:10A6700081111D4616460DE01A6C002A40F0E68056
:10A68000D3F88020002A40F01181D3F8C02003F5D0
:10A6900080732AB9994206D91A68002AECD040334F
:10A6A000994200F2D78032467646112E40F23A8126
:10A6B000DEF1150100F13681614B1D465B6B9A425C
:10A6C00038BF2B46039D38BF5A63DBF8F438EA1ACB
:10A6D000002A16DB03F5F42303F590739D4284BF33
:10A6E0002B460533CBF8F438554B554A5B6B052B9D
:10A6F00086BF053BDBB200238BF8F0384FF0FF3309
:10A70000536331B100FA01F1C6F114060120B040E3
:10A7100008434C4EC0F3C43306EB8303D3F86C1DDF
:10A7200000F01F0306EB8303D3F86C2D42EA0132DD
:10A73000C0F3441106EB8101C0F3842306EB8303CD
:10A74000D1F86C1DD3F86C3D42EA011141EA0321B6
:10A7500081EA112383EA131303F00F02354BD3F878
:10A76000F03D0F2A03F1010340F0BD80B1F5803FB9
:10A7700080F0B980B9F1540F4FEA111140D02D4A41
:10A78000B1F5606FC2F8F03D45D0019B998194F816
:10A790005830059883420CD0BA6823689B1A23600E
:10A7A0003A6B63689B1A63600023BB603B6384F869
:10A7B0005800236801332360BB680133BB604FF648
:10A7C000FF73994205D16368013363603B6B0133CA
:10A7D0003B63019B08F101081433B8F1080F04F141
:10A7E0005C0407F15C0701930AF1200A7FF4F3AEE1
:10A7F000104A0123012082F8EC3E07B0BDE8F08F3B
:10A80000BBF8E0280132ABF8E0280A4AB1F5606FE6
:10A81000C2F8F03DB9D19BF88E3003EB43030BEB4C
:10A82000C303434493F89D300D2BAED1019A80238E
:10A830009377ACE7040000101F85EB51CDCCCCCC56
:10A84000880100205008060898190020803399429A
:10A850007FF629AFA3EB050C3C4A4FEAAC1C0CF188
:10A86000010C82FB0C52A2EBEC72012AB8BF012250
:10A8700090404FF0010C9644013A0CFA02F210435A
:10A880009C46DCF800209AB1DCF84020002A57D022
:10A89000DCF88020002A56D0DCF8C0200CF5807C43
:10A8A00042B16145EDD81D466346F3E6C033F7E695
:10A8B0000CF1400C6145F6D9ACEB03029211234B2D
:10A8C000013283FB0253A3EBE273012BB8BF0123D8
:10A8D00098409E440122013B02FA03F31843634669
:10A8E0001D466346D6E6B9F1540F04D1BBF8E02803
:10A8F0000132ABF8E028164AC2F8F03DD2F8EC3D40
:10A900000133C2F8EC3D4FF6FF7140E74033A3EB53
:10A910000C0C99424FEAAC123FF6A1AE10B10138CF
:10A920008BF8F008B9F1540F7FF453AFBBF8E2385D
:10A930000133ABF8E2384CE7803389E6C03387E671
:10A940000CF1800CB6E70CF1C00CB3E75655555529
:10A9500004000010F8B51D4B93F88D2093F88E304D
:10A960009A422ED11A4F7D68002D11DD3846002401
:10A9700010F8086B16B1037E012B1CD00269136816
:10A98000013443F00103A54200F580701360F1D15A
:10A99000FFF7B4FCD7F8F04E002C0BDD0D4A02EBAC
:10A9A000C404116893888889083203439BB2944297
:10A9B0008B81F6D1F8BD002380F8F030FDF7F8FE6A
:10A9C000DCE752F079FB0028CCD1F8BD98190020C3
:10A9D00004000010F80E00102DE9F8430546FFF7BB
:10A9E0008DFC244E244B044610274FF0E02C4FF4EE
:10A9F0007A7E4FF001087268C2F30802CAB9EFF319
:10AA00001182B2B91A68DCF8180019688A42F9D1C3
:10AA100059688842F6D8D3F808900EFB09F1091A54
:10AA2000B1FBF9F10EFB0212121BAA42E3D3BDE8FF
:10AA3000F883EFF3118287F31288DCF81800DCF852
:10AA40001010C90344BFC3F85C87DCF81800D3F8C2
:10AA50000090D3F85C17D2B282F311884944D3F83E
:10AA600008900EFB09F2121AB2FBF9F20EFB01225A
:10AA7000DAE700BF00ED00E098190020002878D048
:10AA80002DE9F0473B4B3C4D00F1FF3810264FF0CD
:10AA9000E0204FF47A7C01276A68C2F30802002A9A
:10AAA00053D1EFF31182002A4FD11A6884691968D3
:10AAB0008A42FAD159688C42F7D899680CFB01FE9A
:10AAC000AEEB040EBEFBF1FE0CFB02EE6A68C2F3B5
:10AAD0000802EAB9EFF31182D2B91A6884691968D9
:10AAE0008A42FAD159688C42F7D8D3F808900CFB07
:10AAF00009F1091BB1FBF9F10CFB0212A2EB0E02EA
:10AB0000B2F57A7FE2D3B8F10108C5D2BDE8F0878B
:10AB1000EFF3118286F3128884690169C90344BF87
:10AB2000C3F85C778469D3F800A0D3F85C17D2B27D
:10AB300082F31188D3F8089051440CFB09F2121BE0
:10AB4000B2FBF9F20CFB0122D8E7EFF3118186F397
:10AB5000128884690269D20344BFC3F85C778469B0
:10AB6000D3F800E0D3F85C27C9B281F311887244AE
:10AB7000A3E770479819002000ED00E030B50C46BF
:10AB800083B00546D8B1036803F13F4303F57E0364
:10AB90009B0A0C4A134493F854044FF05FFFC4F32C
:10ABA0004112C4F30013CDE90032C4F38103A98834
:10ABB000286804F0030251F083FF03B030BD4FF06A
:10ABC000FF33E6E75008060800B1D7E7704700BF3B
:10ABD00070B50E4C94F8C865B6B104F581640025D3
:10ABE00004E00135B54204F120040DD0237F002B91
:10ABF000F7D0E0680028F4D0217D0135FFF7BEFFD3
:10AC0000B54204F12004F1D1012070BD0400001010
:10AC100070B5002486B0CDE90144CDE903440DF1BF
:10AC2000040CC0E93D44C0E93F44C0F80441054676
:10AC300000F5847EBCE80F00AEE80F00CEF80040BF
:10AC400095F82131059444F23B36A5F84C610BB9D7
:10AC500006B070BD1C09013C052C03F00F032BD876
:10AC60001A4E06EB4402B2F8F40340FA03F2D2079C
:10AC700022D5012202FA03F3013B2644184055F085
:10AC80003FFC96F8EC2D124B024403EBC20429461C
:10AC90002623104DE380204641F80C5F51F0A0FEC2
:10ACA0000D49A2880868B2FA82F24FF00043D340FF
:10ACB00003430B6006B070BD2946064B41F80C3FBC
:10ACC000002006B0BDE8704051F08ABE500806086A
:10ACD000901A0020E1B00008003C014048B1828891
:10ACE0000449B2FA82F208684FF00043D3400343AC
:10ACF0000B607047003C014038B50409013C052C4D
:10AD00001AD80F4D05EB440200F00F03B2F8F4031C
:10AD100040FA03F212F0010210D0012202FA03F30A
:10AD2000013B1840254455F0EBFB95F8EC3D054AF6
:10AD3000034402EBC30038BD002038BD104638BDC7
:10AD400050080608901A002008B514F069FA052882
:10AD500007D8054BD3F8F8380344187BBDE8084002
:10AD6000CAE7002008BD00BF9819002008B51D20C3
:10AD7000FFF7C2FF10B190F9063053B11E20FFF764
:10AD8000BBFF10B190F9063003B108BD5523C38055
:10AD900008BD5523C380F1E7F8B5037D85690268D6
:10ADA0001F2B04464BD95068203B20219940084274
:10ADB00037D0D16010219940D1605168D940CE0779
:10ADC0007FD4EFF31183502282F312882A6C11682A
:10ADD000C90757D4516889B291B9D5E9096086424B
:10ADE0004DD0AF699CBF0E462969074494BF081A2D
:10ADF000301A80B20021D760AE6285F864105060CE
:10AE0000116841F00101DBB2116083F3118895F8FC
:10AE10006430002B3DD1237D22681F2B194614D9A5
:10AE2000203B506808219940084200D0D16050680A
:10AE3000042101FA03F3184200D0D360F8BD16686C
:10AE40002020984006420DD11946106808238B40F7
:10AE5000184200D09360106804238B401842EDD054
:10AE60009360F8BD10219940906091601168D940BD
:10AE7000C807A6D5012101FA03F39360A1E70122D7
:10AE800085F86420DBB283F3118895F86430002BD9
:10AE9000C1D095F87230002BBDD195F87100FFF745
:10AEA0002BFF2A6E938923F008031B0401211B0C3E
:10AEB000938185F872100028ADD02021FFF75EFE47
:10AEC000A9E7012101FA03F3D3607AE708B54CF052
:10AED00071FB1B20FFF710FF08B12923C3801C2042
:10AEE000FFF70AFF08B12923C3800C4B93F801290F
:10AEF000022A01D0012008BD93F80829012AF9D1BE
:10AF00000748C3F80C0900F120014C304EF032FE26
:10AF1000044B002083F8230008BD00BF98190020CF
:10AF2000C001002000ED00E010B58078FFF7E4FEDE
:10AF300078B1084AD2F810390446013341218171B1
:10AF4000C3712021C2F81039FFF718FE2368A288C8
:10AF50001A8310BD9819002043680B4A23F04073F0
:10AF600023F4807343F48073436083681A4042F093
:10AF700002028260C36A0139C9B223F4700343EA52
:10AF80000153C362704700BFFDF7FFC0704700BFA9
:10AF90000020FDF763B800BF0120FDF75FB800BFD8
:10AFA0000220FDF75BB800BF10B1036882881A83E6
:10AFB000704700BF10B1036882885A83704700BF92
:10AFC000F0B5056890F888606B688488012285F880
:10AFD00024201A8822F040021204120C1A802A89B6
:10AFE000A24255D1017BAA7A8A420BD01A8822F05C
:10AFF00003021204120C1A801A8892B2002944D05B
:10B000001A80A9721A882F7B92B242F040021A80ED
:10B010002B6A9A6892B34FF0000C2F4C1433E6461B
:10B0200053F8101C964401EA040221B1B2F1805F8A
:10B0300027D06A692AB353F8142C143302EA0401A6
:10B0400012B1B1F1805F1CD053F80C2C0CF1010C43
:10B05000002AE5D1AFB1A6B1BCF1010F0AD8BEF10B
:10B06000070F07D80CEB8C0C4FEA8C022B6A1344A9
:10B070001B7B33B9BDE8F04046F02ABD0FB1002E6E
:10B08000F4D1BDE8F04046F0A1BF42F00302B7E7BB
:10B090001A88124922F0380212048B424FEA1242F7
:10B0A00017D001F580618B4213D02146B1F5807F26
:10B0B000A8BF4FF480710229B8BF022191FAA1F113
:10B0C000B1FA81F1013942EAC10292B21A802C81AF
:10B0D00088E76108EAE700BF0000FFFF0038004092
:10B0E00038B52C4AD0F8E0305268D0F8D810044671
:10B0F00073B1501A83420BDC94F8D030C4F8D820D6
:10B10000012B10D0D4F8D4300133C4F8D43038BD7A
:10B11000D4F8E430C4F8D8200B44C4F8DC3094F8F8
:10B12000D030012BEED16168201D04F1E805EFF36A
:10B13000118C102383F3128863681B6A0BB3D4F855
:10B14000F0302A461BB1D3691432002BFBD10B6AB5
:10B150006BB1996839B9934209D0196829B15B6814
:10B1600099680029F7D01433F3E7C3E900055FFAC3
:10B170008CFC8CF31188D4F8D4300133C4F8D4306B
:10B1800038BD0D625FFA8CFC8CF31188FFF718FF55
:10B19000B8E700BF001000E02DE9F041826992F8A5
:10B1A000DC30012B8AB005464CD0023B012B54D831
:10B1B00092F84C31D2F89C202E4C63F07F03137030
:10B1C0008769D7F8A030D7F8108003F1010E0FCCB3
:10B1D000EC46ACE80F00D7F89C30CDE9003E0FCC30
:10B1E000ACE80F0094E8030007F110068CE80300B8
:10B1F000EFF31180102383F312883B691B6A002B45
:10B200002FD0029B6A461BB1D3691432002BFBD1AD
:10B21000D8F8203073B1996839B99A420AD01968C0
:10B2200029B15B6899680029F7D01433F3E71E60F1
:10B23000C3F804D0C0B280F31188AA6911690B6AFF
:10B24000002BFCD1D2F8A0305A8852BAEA819A88F1
:10B2500052BA2A82DB885BBA6B8201200AB0BDE851
:10B26000F081C8F820D0C0B280F311883046FFF7D3
:10B27000A7FEE2E7441606082DE9F04190F8DC301D
:10B28000D0F8A050012B8AB0044673D041D9023BBC
:10B29000012B6BD890F84D31D0F89C205E4E63F0B6
:10B2A0007F031370D0F8A030D0F8108003F1010EA6
:10B2B00000F110070FCEEC46ACE80F00D4F89C303C
:10B2C000CDE9003E0FCEACE80F0096E803008CE815
:10B2D0000300EFF31180102383F3128823691B6AA4
:10B2E000002B00F08F80029B6A461BB1D369143299
:10B2F000002BFBD1D8F820302BB3996839B9934291
:10B3000021D01968E1B15B6899680029F7D014333E
:10B31000F3E7D0F89C304FF0FF321A605A609A6021
:10B32000DA60D0F8E0300522B3F57A7FC0F8F0207B
:10B330003BD8032380F8DC3001200AB0BDE8F0815F
:10B340001F60C3F804D0C0B280F311882269136A69
:10B35000002BFCD16B885BBAA4F8D030AB885BBA09
:10B36000A4F8D230EB885BBAA4F8D43001200AB03C
:10B37000BDE8F08190F84C2190F84D319B1A5B109C
:10B380000133DBB205EB430235F813305BBAA0F8AA
:10B39000D03053885BBAA0F8D23093885BBAA0F85B
:10B3A000D43001200AB0BDE8F08103691A7B2AB3CA
:10B3B0005B691BB390F8983003B390F84C31D0F828
:10B3C0009C20C4F8A40063F07F03137090F84C1124
:10B3D00090F84D31D0F8A0201048C4F804015B1A51
:10B3E00007330121C4F8FC30D4F89C3084F80011F4
:10B3F0000A44C4E93D3284F8DC10B7E7022384F83C
:10B40000DC30B3E7C8F820D0C0B280F311883846EA
:10B41000FFF7D6FD9AE700BF4416060839800008FA
:10B42000D3B2012B1DD8104B02EB420210B54FEAEC
:10B43000820E0EF1080403F5137C02E01C33634511
:10B440000DD01A788242F9D15A788A42F6D11A5927
:10B45000002AF3D00EF1040E03EB0E0010BD002005
:10B4600010BD0020704700BF6C16060810B40C4CCD
:10B47000002304F6141C01E0152B0CD003EB43024F
:10B4800001331CF802108142F6D1144494F91609D4
:10B490005DF8044B70474FF0FF305DF8044B704788
:10B4A00098190020D3B2022B22D870B502EB4202C9
:10B4B000104C4FEA820E23460EF10C05002204E0E8
:10B4C0000132172A03F12C0310D01E68B042F7D1C5
:10B4D00093F804C08C45F3D15E59002EF0D02C2196
:10B4E0000EF1080301FB0233E01870BD002070BDAF
:10B4F0000020704750080608002839D030B51D4D8F
:10B5000090F804C0002305F6141401E0152B2DD08B
:10B5100003EB43020133A15C6145F7D11544046894
:10B5200095F9163990F805E0DAB2022A1ED803EB35
:10B53000430311484FEA830C0CF10C05034600222B
:10B5400004E00132172A03F12C030FD019688C4252
:10B55000F7D119797145F4D159590029F1D02C212D
:10B560000CF1080301FB0233184430BD002030BD4C
:10B57000704700BF98190020500806080348D0F80B
:10B58000B0300BB1A0301847704700BF88010020D1
:10B590000348D0F8D4300BB1C4301847704700BF0F
:10B5A000880100200348D0F8F8300BB1E830184784
:10B5B000704700BF880100200348D0F81C3113B148
:10B5C00000F5867018477047880100200348D0F8BE
:10B5D000403113B100F5987018477047880100207A
:10B5E0000348D0F8643113B100F5AA7018477047CA
:10B5F000880100200348D0F8883113B100F5BC70F1
:10B6000018477047880100200348D0F8AC3113B1C7
:10B6100000F5CE7018477047880100200348D0F825
:10B62000D03113B100F5E070184770478801002051
:10B630000348D0F8F43113B100F5F27018477047A1
:10B64000880100200348D0F8183213B100F50270C9
:10B6500018477047880100200348D0F83C3213B1E6
:10B6600000F50B7018477047880100200348D0F898
:10B67000603213B100F5147018477047880100203C
:10B680000348D0F8843213B100F51D701847704795
:10B69000880100200348D0F8A83213B100F52670C5
:10B6A00018477047880100200348D0F8CC3213B106
:10B6B00000F52F701847704788010020094B0A4A8F
:10B6C000013800EBC00003EB80030848D3F8A0303A
:10B6D000116B834214BF4FF480034FF400130B43EC
:10B6E0001363704788010020003802400060024068
:10B6F00070B501383C4C3D4D00EBC00C04EB8C0C9C
:10B700009646DCF8A0603A4AAE4214BF4FF480057A
:10B710004FF40015166B35431563CCF8B010CCF818
:10B72000B8303449DCF8A4308B424FEAC0023ED036
:10B7300001F580618B423AD0A1F57A718B4247D0F6
:10B7400001F580618B4243D0A1F57A718B4241D0E3
:10B7500001F580618B423DD0A1F57A718B4235D0E5
:10B7600001F580618B4231D0A1F57A718B4233D0E3
:10B7700001F580618B422FD0A1F57A718B422DD0DB
:10B7800001F580618B4229D0A1F57A718B4227D0D7
:10B7900001F580618B4223D0A1F57A718B4221D0D3
:10B7A000154D01F580618B4218BF002500E0134D57
:10B7B000131804EB8303CEF38711C3F8C05093F83A
:10B7C000B500BDE87040002251F0E6B80C4DEFE73F
:10B7D0000C4DEDE70C4DEBE70C4DE9E70C4DE7E7C1
:10B7E0000C4DE5E7044DE3E78801002000600240CE
:10B7F00000380240106002400080002820800010C5
:10B800000080001800880010008020102080002098
:10B8100000880020008020202DE9F04F924A92F805
:10B820006539012B85B021D0022B15D00023009360
:10B830008E4F4FF0000807F1780A3B78022B17D0A3
:10B8400008F10108B8F1030F07F128070AF1050A0A
:10B85000F3D105B0BDE8F08F92F85A3933B192F8C0
:10B860005639083B18BF01230093E1E70093DFE757
:10B870009AF903307E4D0297591C15BFDBB20023A5
:10B880009B464FF0010B1E46DAB2012A00F2D98026
:10B8900006EB460189007300764C019308315FFA8C
:10B8A00088F703E01C34AC4200F0CB802378002BF7
:10B8B000F8D16378BB42F5D160580028F2D011F07E
:10B8C00049FA009B814623B1A0F10901072940F202
:10B8D000BD807A1CD2B21421484611F027FA002804
:10B8E00000F0AF80DDE90137334404EB830409F154
:10B8F000FF33E068604C594203EBC30201F00701DB
:10B9000003F0070358BF4B4204EB8201A03404EB61
:10B910008202C1F8AC003A61484681F8A830FFF7CE
:10B92000CDFE9AF904305A1C00F09980DEB23246FE
:10B93000CDE902974E4DF3B29346012B61D806EB49
:10B940004601890073004B4C019308315FFA88F976
:10B9500002E01C34AC4254D02378012BF9D1637837
:10B960004B45F6D160580028F3D011F0F3F9009B55
:10B9700007461BB1A0F10901072946D909F10102C7
:10B98000D2B21321384611F0D1F9002839D0019AEA
:10B99000DDF808903244BB4604EB82040BF1FF3221
:10B9A0005142E068344C039F02EBC20501F00701ED
:10B9B00002F0070258BF4A4204EB8501A03404EBB1
:10B9C0008505C1F8AC007D61584681F8A820FFF7D5
:10B9D00075FEB9F1000F3DD0BBF1000F1BD028461A
:10B9E000FCF750FD3869FCF74DFD3846FCF71AFDB1
:10B9F00000231A4621495846FFF77AFE01233B737C
:10BA00001EE70136F3B29B4597D2DDE90297B9F103
:10BA1000000F1FD01A4C09F1FF33242202FB034010
:10BA2000002438617C61FCF72DFD3846FCF7FAFCF8
:10BA30002346144922464846FFF75AFE01233B732A
:10BA4000FEE60136F2B25A457FF61FAF029F4FF075
:10BA5000000966E700220023C7E90423F0E601237A
:10BA60001A46002664E700BF98190020182300201A
:10BA7000B81806086C1606088801002055A10008B1
:10BA800028020020CDA10008800AA0F580105228CD
:10BA900008D8054B034493F800340D2B02D8034A11
:10BAA000D056704700207047500806086883060883
:10BAB000064A136851690B4003F00103536123B137
:10BAC000034BD3F89807036818477047003C0140C0
:10BAD00098190020064A136851690B4003F00203CD
:10BAE000536123B1034BD3F89C0703681847704791
:10BAF000003C014098190020064A136851690B4028
:10BB000003F00403536123B1034BD3F8A007036888
:10BB100018477047003C014098190020064A1368F6
:10BB200051690B4003F00803536123B1034BD3F871
:10BB3000A407036818477047003C0140981900208B
:10BB4000064A136851690B4003F01003536123B197
:10BB5000034BD3F8A807036818477047003C01401F
:10BB600098190020F8B50C4B1D685A69154005F46A
:10BB700078755D617DB1094F0126B5FA85F4C4F190
:10BB80001F0407EB840306FA04F4D3F8980703684C
:10BB90009847A543F1D1F8BD003C01409819002019
:10BBA000F8B50C4B1D685A69154005F47C455D617C
:10BBB0007DB1094F0126B5FA85F4C4F11F0407EBE6
:10BBC000840306FA04F4D3F8980703689847A5435A
:10BBD000F1D1F8BD003C014098190020F0B50546B0
:10BBE00083B0A0B307681D4B144607F13F4202F52E
:10BBF0007E0203EB92230E4693F854044EF02EFF80
:10BC0000A988B1FA81F3C3F11F03C3F3CC0207EB98
:10BC1000820203F00703156A4FF00F0C9B009C4053
:10BC20000CFA03F325EA03031362136A1C4314623C
:10BC3000C6F30013C6F34112CDE900323846C6F30D
:10BC4000810306F0030250F03BFF03B0F0BD034B4D
:10BC500093F853044EF002FF2B68FFDE50080608ED
:10BC600000B1BBE7704700BF2DE9F047684E06EB17
:10BC70000013D3F8084A002C76D093F8107A0546C2
:10BC80004FEA001838464EF0E9FE07F01F027F0920
:10BC90000123032F03FA02F372D0042F6BD0022F7B
:10BCA00064D006EB0803013593F80C0AFFF724F87B
:10BCB000EDB2824610B11223C571837106EB080301
:10BCC00093F80D0AFFF718F8814610B11323C571D8
:10BCD000837106EB080393F80E0AFFF70DF8074689
:10BCE00010B11423C571837106EB0803504693F815
:10BCF0000F5A4A212A46FFF7B3FF2A4648462A210F
:10BD0000FFF7AEFF2A460A213846FFF7A9FF414B4D
:10BD10009C423AD0404B9C4242D0404B9C424AD03D
:10BD20003F4B9C4252D03F4B9C425AD03E4B9C4290
:10BD300062D0A38823F003031B041B0CA380238879
:10BD400003F4415343F4457343F003032380A38B6F
:10BD500023F400631B041B0C0722A3832282238885
:10BD60009BB243F040032380BDE8F0872F4A516A1D
:10BD70000B43536295E72D4A11690B43136190E71A
:10BD80002A4A116A0B4313628BE703F584335A6A1C
:10BD900042F480525A625A6A22F480525A62C8E7C8
:10BDA00003F500331A6A42F480421A621A6A22F4D6
:10BDB00080421A62BDE703F5FE331A6A42F400427C
:10BDC0001A621A6A22F400421A62B2E703F5823359
:10BDD0005A6A42F400525A625A6A22F400525A6273
:10BDE000A7E703F568435A6A42F480125A625A6A16
:10BDF00022F480125A629CE703F564435A6A42F4C3
:10BE000000125A625A6A22F400125A6291E700BF85
:10BE1000981900200030014000380040003C0040EC
:10BE200000340140005001400054014000380240FD
:10BE3000431C00F02E812DE9F04FDFF84C8300EB1E
:10BE4000800308EBC30387B0D3F80C90820005464B
:10BE50000192B9F1000F04D05C692CB194F906305D
:10BE600013B107B0BDE8F08FAB002B4408EBC30360
:10BE7000D3F818A0BAF1000F03D09AF90630002BBE
:10BE8000EFD1AB002B44B94ED9F80470DB00183366
:10BE9000F0180022691CF250C9B2C0E90122C26048
:10BEA000002C00F083811523E171A37199F828001B
:10BEB000BAF1000F00F06A8116238AF807108AF899
:10BEC00006304EF0CBFDBB882268A08823F4407377
:10BED0001B041B0CBB80DAF800301083BAF8042076
:10BEE0001A8311212046FEF749FE11215046FEF724
:10BEF00045FE09264FF0330B2CB9C4E0BBF1010B12
:10BF000006D04FF05FFE2268A18810690142F5D08B
:10BF100051834FF0B3FE2368A2881A834FF0AEFE20
:10BF2000013EE7D1002C00F0DE80332603E0013E25
:10BF300006D04FF047FE2268A18813691942F6D057
:10BF400051834FF09BFEBAF1000F00F0F480DAF855
:10BF50000030BAF804205A834FF090FE2368A2887C
:10BF60001A834FF08BFEDAF80030BAF804201A83F7
:10BF70004FF084FE2368A2881B691A4240F08A8031
:10BF8000019B2B4408EBC303997F1A7F002940F0E3
:10BF90008D8020461221FFF721FE1221019B2B44A8
:10BFA00008EBC3035A7F5046FFF718FE704B9F42C1
:10BFB00000F014816F4B9F4200F01B816E4B9F423B
:10BFC00000F02281019B2B4408EBC3034FF47A72EB
:10BFD0001C8CBB8823F440731B041B0CBB803B8868
:10BFE0009BB243F001033B80BD8802A802FB04F42E
:10BFF00025F03F054AF066FF0499604B2D04A3FB32
:10C0000001232D0C45EA9345BD803A8822F00102B8
:10C010001204120C3A805A4A980C944203464BDCA4
:10C020006200B1FBF2F292B20133042A38BF04225B
:10C030003B84BA833B889BB243F001033B803B883F
:10C0400023F4816323F002031B041B0C4FF4804193
:10C0500043F480633B8039813B8823F080031B04D9
:10C060001B0C00223B8099F82A00114650F094FCEA
:10C07000002299F82900114607B0BDE8F04F50F0B2
:10C080008BBC4FF09FFDBBF1010BFAD14FF0F6FDD9
:10C0900044E77047019BDAF800202B4408EBC30308
:10C0A00012699A7F002A00F0BA801A7F3221204656
:10C0B000FFF794FD322171E704EB4404B1FBF4F186
:10C0C0008AB2C1F30B0109B942F001022D494FF4C4
:10C0D000967300FB03F3A1FB03139B09013342F4A6
:10C0E00000423B84A5E7332401E04FF06BFD013CA7
:10C0F000FBD14FF0C3FDBAF1000F00F09680DAF8E3
:10C100000030BAF804205A834FF0B8FD4FF0B6FD66
:10C11000DAF80030BAF804201A834FF0AFFD019B23
:10C120002B4408EBC3039A7F002A18BF32215A7FA1
:10C1300008BF122137E74FF0A1FD2368A2881A83B8
:10C140004FF09CFD4FF09AFD2368A2881B691A42AC
:10C1500072D1019B2B4408EBC303997F1A7F0029FE
:10C1600079D020463221FFF739FD1FE7A4190020BE
:10C170000054004000580040005C004083DE1B4338
:10C18000A0860100D34D6210981900204EF066FC85
:10C19000BB88A28823F440731B041B0CBB8023685C
:10C1A00011211A832046FEF7E9FCA2E699F828003F
:10C1B000BAF1000F54D016238AF806308AF8071017
:10C1C0004EF04CFCBB88BAF8042023F440731B04E7
:10C1D0001B0CBB80DAF800301A8386E603F5F233D5
:10C1E0001A6A42F400121A621A6A22F400121A62DF
:10C1F000E8E603F5F0331A6A42F480021A621A6A1A
:10C2000022F480021A62DDE603F5EE331A6A42F484
:10C2100000021A621A6A22F400021A62D2E61A7F37
:10C2200020461221FFF7DAFCB7E64FF027FD4FF06A
:10C2300025FD4FF023FDB9E6019B2B4408EBC3031A
:10C2400020469A7F002A18BF32211A7F08BF122188
:10C25000FFF7C4FCAAE620461221FFF7BFFCA5E6C3
:10C260004EF0FCFBBB8823F440731B041B0CBB800B
:10C270003FE600BF2DE9F8430746FEF717F8DFF861
:10C280004C8007EB8709044608EBC90542F20F769C
:10C2900004E0FEF70BF8001BB0420BDC95F82530EC
:10C2A000002BF6D108EBC90898F8240080F00100B3
:10C2B000BDE8F883B8F8383A013338469BB2A8F89D
:10C2C000383AFFF7B5FD0020BDE8F8839819002043
:10C2D000B0F1FF3F6DD02DE9F04F022883B0044646
:10C2E00014DC354E984600EB800306EBC305DB00FB
:10C2F000D5F810A00093BAF1000F07D0894695F841
:10C300002510934601F0FF02019219B1002003B0FD
:10C31000BDE8F08FFDF7CAFF009B019A2033074666
:10C320004FEA490106F10C00C9B200EB030C85F895
:10C3300026104FF0010E0C9985F827B085F82920BA
:10C3400085F82AE0C150CCF8041085F8288085F8DB
:10C3500025E085F82420BAF8043099051DD4BAF8F0
:10C360000030DA0512D442F20F7504E0FDF79EFFAB
:10C37000C31BAB4213DCBAF800309B05F6D4BAF805
:10C3800000309BB243F48073AAF80030BAF804304E
:10C390009BB243F44073AAF804300120B7E7B6F823
:10C3A000383A01339BB22046A6F8383AFFF740FDF1
:10C3B000ACE70020704700BF98190020E0B5294E77
:10C3C00000EB800306EBC30384B0DA685568AA8AE1
:10C3D00092B20392039A12F4706F1CBF012283F889
:10C3E0002420039B13F4E06F4FEA80070DD1AB8A42
:10C3F000074423F4706306EBC7061B041B0C0022E2
:10C40000AB8286F8252004B0E0BD2B8BAB8823F4EB
:10C4100080631B041B0CAB80039B9A05E7D42B881D
:10C420009B05E4D42B88D9050FD52B88DA05FCD4DD
:10C430002B889BB243F400732B802B889B05FCD484
:10C440000190FFF7F5FC0198D1E72B889BB243F4EC
:10C4500000732B80AB8823F440731B041B0CAB8050
:10C46000C5E700BF981900200020A7E70120A5E735
:10C470000220A3E770B590F871301C09013C052C2F
:10C480000FD81A4E06EB44020546B2F8F40303F047
:10C490000F0340FA03F2D20703D595F87220012A60
:10C4A00001D0012070BD9A40013A1040264454F05A
:10C4B00027F896F8EC3D0E4A034402EBC30452F809
:10C4C0003320A38810691840ECD0EB6E002285F869
:10C4D000722093F8212002212046FFF77FFB2A6E6D
:10C4E00093899BB243F008039381DAE7500806086A
:10C4F000901A0020F8B50E4C94F8C8759FB104F559
:10C50000BA64C7F109070925013D0ED0A668307944
:10C51000FEF7F2FB217DF27908B1FFF75FFBAF4236
:10C5200004F18C04F0D10120F8BDAB68FFDE00BF40
:10C5300004000010094BD3F83C2AD3F8401A40F20B
:10C540002A40002350604B620B889BB243F00103EA
:10C550000B80136843F001031360704798190020A3
:10C5600010B41D4B1D48196C1D4A41F08051012427
:10C5700085B0196404625321FF24CA2054625062BA
:10C5800051625B6FDB0017D416480423002102912F
:10C590000290029A1A440292029A04331C2B1160F0
:10C5A000F5D103910390039B0393039B0E4A1A60FA
:10C5B00005B05DF8044B70470A4B002201920193CD
:10C5C000019B0193019A084B12689A42DCD105B095
:10C5D0005DF8044B704700BF0038024000000E4277
:10C5E0000028004050280040316665422DE9F041A6
:10C5F000046ED0F80880A38923F400531B04074677
:10C600001B0C90B0A38143793D79C3F380001903DB
:10C6100005F001061B0215F002054FEA00304FEA53
:10C62000860203F4806318BF42F0080203431A43F2
:10C63000238A9BB201F4005123F440530B4323821D
:10C64000A38923F4B05323F00C031B041B0C1A43DF
:10C65000A281A38A23F440731B041B0CA38201A8AC
:10C660004AF030FC6B4B9C4205D003F580639C4242
:10C6700001D0039B00E0049BA2896749A0891204B2
:10C6800003EB83034CBF4FEA48084FEA880803EBEB
:10C690008303B3FBF8F3A1FB03C252094FF0640C10
:10C6A00000040CFB12334FEA021200F19A801B01C6
:10C6B0003233A1FB0313C3F3431313439BB2238110
:10C6C00097F9380097F80580FEF73EFB30B1036814
:10C6D000828818F0010F14BF1A835A8318F0080FCC
:10C6E000A38A78D09BB243F00803A382A3899BB2AC
:10C6F00043F40053A381002E2FD0FE6B002E7DD07B
:10C700000023CDE90833CDE90C33CDE90E33049392
:10C7100006937B6C0193FB6D0293FB6805937B6929
:10C7200003934FF480714FF48033CDE90A13304600
:10C730004FF4806307934AF027FC01A930464AF082
:10C74000B9FC336843F001033360A38A9BB243F022
:10C750004003A38273689BB27B65002D33D03E6C8F
:10C76000002E46D0BB6C0193BB6D02933B690593D1
:10C77000402304934FF48033002530460B934FF44D
:10C7800080630793CDE90855CDE90C55CDE90E55E9
:10C79000039506950A954AF0F7FB01A930464AF041
:10C7A00089FC736943F080037361336843F01603B7
:10C7B00033607560A38A9BB243F08003A382E36871
:10C7C00043F04003E360A3899BB243F40053A38189
:10C7D00010B0BDE8F08123F008031B041B0CA382FA
:10C7E00084E7DB003233A1FB0313C3F3421313438B
:10C7F00064E7E36843F08003E360E0E74FF6DF734C
:10C800002380E36843F02003E360E36843F0100310
:10C81000E360A2E7001001401F85EB51BFF34F8F8B
:10C820000549064BCA6802F4E0621343CB60BFF3CC
:10C830004F8F00BFFDE700BF00ED00E00400FA05E8
:10C8400008B5002103204AF0B7FC72B6FFF7E6FFF7
:10C85000294C08B5D4F8443A94F84A0A002B3CD144
:10C860001420FEF70BF9002000BFD4F8443A5BB166
:10C870001A689B88116994F84A2A0B4012B91BB1B7
:10C88000FFF7DEFF002BFBD02268D4F86436D31A02
:10C89000322B12DCD4F84C3AD31A002BE4DDD4F856
:10C8A000643733B199881B685D69294214BF598385
:10C8B00019833232C4F84C2AD6E794F86037D4F89A
:10C8C000642703F001031AB1116892881BB90A8327
:10C8D000C4F84C0AC8E74A83FAE719689A880B69D2
:10C8E000134020B1002BBBD10B691340FAE7002B9A
:10C8F000B6D00B691340FAE79819002008B572B654
:10C90000FFF78CFF00B583B00D4900220092009123
:10C91000009B0C330093009B1B68012B02D003B0DB
:10C920005DF804FB01920191019B06490C330193D0
:10C93000019B1A600B6883F308884B689847FEE7F1
:10C94000502800400000FF1F38B5FFF709FEFFF731
:10C95000D9FF01204AF040FC6D4A936823F003039D
:10C960009360936813F00C0FFBD113686849A0B96A
:10C9700043F00103136041F2883302E0013B00F011
:10C98000C5800A689507F9D5624C00220823C4F8CF
:10C99000502AC4F8543A02251EE043F48033136051
:10C9A00041F2883302E0013B00F0B0800A68940352
:10C9B000F9D5584C584B594DB0FBF5F5B0FBF3F099
:10C9C000B5EB400F18BF28464FF48003C4F8503A27
:10C9D000C4F8540AB5FBF0F50220C4F8585A4AF0DE
:10C9E000FBFB03280DD84E4B03EBC0039988DA8874
:10C9F000C4F8601A5B88C4F8642AB3FBF5F3C4F882
:10CA00005C3A434B47491A6C42F080521A640A68F8
:10CA100042F440420A609A689A609A6842F400427E
:10CA20009A609A6842F4A0529A60D4F8501AD4F8E6
:10CA3000542A0A43D4F85C1A42EA8112D4F8641AE0
:10CA400042EA0162D4F8601A4908013942EA014217
:10CA50005A601A6842F080721A601A689201FCD516
:10CA6000314A40F205711160996821F00301996023
:10CA7000996841F00201A2F580629960936803F021
:10CA80000C03082BFAD12949D823B3FBF5F39B01FA
:10CA900043F000530120C2F884308866FBF78EFF14
:10CAA000234D1B4B234AEA60234A596FAA605A6BF5
:10CAB000224922F080025A635A6F42F080725A670C
:10CAC0001A6B42F4CE021A635A6B5A639A6B9A63DA
:10CAD0001A6C0A431A64596C194A0A435A64FCF7DF
:10CAE00021FE184AD4F8F430A2FB03239B09013B32
:10CAF000B3F1807F09D24FF0E022F0205361002192
:10CB0000072385F823009161136138BD014CC7E705
:10CB1000003802409819002080841E0040420F0017
:10CB2000B818060800700040003C02400000474270
:10CB300000ED00E00005FA0500000020FFC9FE3608
:10CB4000335F0700D34D62100C4B0D49DB68DB43AC
:10CB5000C3F30223C3F104030122DBB202FA03F39D
:10CB600001EB000C1B0103F0F0038CF800334309C8
:10CB700000F01F00824041F82320704700ED00E0E4
:10CB800000E100E030B5154C154D85B001390023AA
:10CB900089B2A042ADF80C30ADF806308DF80E30F9
:10CBA0000291D5F8F4300FD00E4988420CD001F52F
:10CBB0008041884208D001F58061884204D001F5A7
:10CBC0008061884218BF5B08B3FBF2F301A9013B07
:10CBD000ADF804304AF010FB05B030BD0004014050
:10CBE000981900200000014001490248FDF7E8B80B
:10CBF000901D00200000014010B5064C064804F5C9
:10CC00007E71FDF7DDF804F284510448BDE8104060
:10CC1000FDF7D6B8981900200000014000440140FB
:10CC200002494FF08040FDF7CBB800BFBC1D00208B
:10CC300001490248FDF7C4B8E81D00200004004087
:10CC400001490248FDF7BCB8141E0020000800404E
:10CC500001490248FDF7B4B8401E0020000C004016
:10CC600001490248FDF7ACB8C41E00200004014091
:10CC700010B5064C064804F22C51FDF7A1F804F556
:10CC8000C1610448BDE81040FDF79AB8981900202A
:10CC900000040140001C004001490248FDF790B823
:10CCA000F01E00200040014001490248FDF788B80D
:10CCB000481F00200048014001490248FDF780B8A4
:10CCC000741F00200018004001490248FDF778B8A1
:10CCD000CC1F00200020004010B50C2935D8DFE81B
:10CCE00001F091343434633434340734343435004F
:10CCF000038C5488B2F80CE023F480731B041B0CE3
:10CD00000384038CB0F804C0818B21F073014EEAD8
:10CD1000040E0904148823F40073090C1B04214336
:10CD2000764C1B0C43EA0E23A0421FFA8CFC9BB2EC
:10CD300000F0948004F58064A04200F08F80926837
:10CD4000A0F804C08183C263038410BD038C54889F
:10CD5000B2F80CE023F480531B041B0C0384038CF7
:10CD6000B0F804C0818B21F4E6414EEA040E0904B8
:10CD7000148823F40053090C41EA04211B045F4C7E
:10CD80001B0C43EA0E33A0421FFA8CFC9BB289B203
:10CD90007ED004F58064A0427AD09268A0F804C0E6
:10CDA00081830264038410BD038C5488B2F80CE0C4
:10CDB00023F010031B041B0C0384038CB0F804C085
:10CDC000018B21F4E6414EEA040E0904148823F095
:10CDD0002003090C41EA04211B04484C1B0C43EAC4
:10CDE0000E13A0421FFA8CFC9BB289B26CD004F5E2
:10CDF0008064A04268D09268A0F804C00183826376
:10CE0000038410BD038C5488B2F80CE023F00103B6
:10CE10001B041B0C0384038CB0F804C0018B21F0AD
:10CE200073014EEA040E0904148823F00203090C6E
:10CE30001B042143314C1B0C43EA0E03A0421FFA92
:10CE40008CFC9BB22CD004F58064A04228D0926860
:10CE5000A0F804C001834263038410BDD489B2F8F2
:10CE600010E023F4006343EA0423548A2CF4405C6A
:10CE70004EEA040E4CEA0E1C94884FF6FF3E03EA7D
:10CE80000E0E4EEA042E1FFA8CFC1FFA8EF356E7A4
:10CE9000148A2CF4804C4CEA841C1FFA8CFC7CE72E
:10CEA000D489B2F810E023F008032343548A2CF409
:10CEB000407C4EEA040E948823F004034CEA0E0CE6
:10CEC0001FFA8CFC2343C2E7D489B2F810E023F0A8
:10CED000800343EA0413548A2CF4406C4EEA040E97
:10CEE0004CEA8E0C94884FF6BF7E03EA0E0E4EEA93
:10CEF000041E1FFA8CFC1FFA8EF37CE70000014031
:10CF00002DE9F04FB14BDFF8DC8293F866E9B04CC5
:10CF1000B04D93B00EF1FF37FBB200930023CDE983
:10CF2000013EC246DFF8C0B2DBF80070BB0AA3F5D1
:10CF30008013522B00F20B81234493F800340D2B05
:10CF400000F2058115F90390029B012B00F0068188
:10CF5000029B022B02D1B9F1080F33D100263146D2
:10CF6000484611F025F811F0AFF890F9003013B1F0
:10CF7000542B40F0EB820436B6B2102EEFD1019B59
:10CF80000021002B00F0A38042460CE0234493F8DC
:10CF900000340D2B0ED8EB564B450ED002F58072A7
:10CFA000524500F09180906803689B0AA3F58013B6
:10CFB000522BEBD900234B45F0D143799BF8050068
:10CFC0009842EBD1844B0BF11C0B9B45ACD1019BE0
:10CFD0000133042B01930AF5807AA3D1DFF80C9278
:10CFE00099F8C835013309F5816A04934FF0010BB4
:10CFF000049B5B4565D0DAF80C30744A9AF810103F
:10D0000092F8682A01930291002B5AD01968D9F836
:10D0100004009B88039101F13F4505F57E0500283A
:10D020004FEA9525009340F3A780002303E00133E6
:10D03000834200F09E801C0258F80410A942F6D1E9
:10D040004444009A029B8AF81030B2FA82F6019B9F
:10D05000CAF80C30C6F11F054FF00301CAF804509E
:10D06000CAF81840997183F807B0E16C606C6B00E6
:10D07000012203279F4002FA03F3194399F8003075
:10D08000E164384302FA05F56064276DD4F8A00026
:10D09000A9B2002B00F060823D432565039D009BF3
:10D0A0002B83FBF73FFA20460BF1010BFBF780FBCC
:10D0B00040F20113BBF1090FAAF81C300AF1200A53
:10D0C00096D113B0BDE8F08F00297FF47BAF5846AE
:10D0D000FBF7EEF9C3B2022B9BF805E000F2778272
:10D0E00000F1010C3A4A0CEB4C0C4FEA8C0C02F5A7
:10D0F0007D7003E02C32904200F0698213689F42F9
:10D10000F8D113797345F5D152F80C30002BF1D0DA
:10D11000324842689A424FF0000108D0013110298C
:10D1200000F124003FF44EAF42689A42F6D14B1C06
:10D13000DBB22B4A013B03EBC30302EB830393F9FE
:10D14000BC30002B7FF43EAFCAF808B03FE7009B2D
:10D15000012B7FF637AF4FF00009FFE6B9F1010F61
:10D160003FF4FCAE1C4B0BF11C0B9B457FF4DCAE7B
:10D170002DE7042B00F0FC8109EB0023010205914F
:10D1800019690691002900F016826C1C0792E4B21E
:10D190004FF054029D6083F8042183F80541069BFB
:10D1A00001305E79C9F8040018461D680896FBF73F
:10D1B0007FF9C3B2022B00F20A82471C07EB470734
:10D1C000034B079ABF000021B44617E098190020CE
:10D1D0005008060868830608D419060828020020AB
:10D1E000880100200C000010D81806080400001068
:10D1F0000131172903F12C0300F0E9811E68B542C3
:10D20000F6D11E796645F3D1DE59002EF0D02C23DD
:10D2100000EB400001FB03F3BB49BC4F03EB800371
:10D220000B4438461969059B0A914B44C3E90661D2
:10D230004368B3424FF0000108D00131102900F1DA
:10D2400024003FF43EAF4368B342F6D14B1CDBB23F
:10D25000AF49013B03EBC30301EB830393F9BC101C
:10D2600000297FF42EAF83F8BD40059CA948E11149
:10D2700001EB242101EB011100EB810C0599CDF8A4
:10D280001CC08C24091204FB01F100F54C7000EB6A
:10D2900041000599099049440998C1F8F440039C5C
:10D2A000CC605424C1F8F00083F8BC409A48C1F81F
:10D2B000A8C03323C1F8AC30984B0599D3F8F430AB
:10D2C000854208EB01040FD095498D420CD001F541
:10D2D00080418D4208D001F580618D4204D001F576
:10D2E00080618D4218BF5B08062A00F06181072A21
:10D2F0008C488D4A8D4918BF11468D4A18BF024689
:10D300000598B3FBF2F2B3FBF1F3013A09EB00012C
:10D3100092B2013BA1F8B030A1F8682000F15401AD
:10D320000023A4F85C30284648F80130A265414447
:10D3300049F062FF0023ADF838302B8808999BB282
:10D3400043F080032B802B8823F001031B041B0C6C
:10D350002B80784B0D934FF0020E4FF48073CDE984
:10D3600010E328460A230DAA0F93FFF7B5FC069B8E
:10D370001879002840F006812B889BB243F0010306
:10D380002B8000237A68964203F1010300F0F780B6
:10D39000102B07F12407F5D14FF0FF3300205C4A32
:10D3A0006549664F03EBC30302EB8303644AD3F87A
:10D3B000A0308B4214BF4FF480034FF40013116B65
:10D3C0000B431363089A0C2A9BBF5E4B03EB42038B
:10D3D0000021B3F88C10059B4B449982002306E092
:10D3E000954200F0EF800133042B00F0ED8057F8F8
:10D3F0003320002AF4D1D9F8F02E0132C9F8F02EEA
:10D4000009EBC302DB00C2F8F45E3B4400259A88B6
:10D410001143998090224C492346FEF769F93368FD
:10D42000059A039843F010033360079BE3660A9B59
:10D43000636602F1640104234FF40032C4E923233C
:10D4400040233322C4E91C3200F118024FF48067F4
:10D45000A2664FF480504FF48042C4E92002414458
:10D460003046C4E92555A567C4F88850C4F89C50D7
:10D47000E76749F01FFE3068E061706920627068FC
:10D480000A9B6062B068A062F068C4F8AC30042304
:10D49000C4F8D830099BE062C4F8B4300398059A08
:10D4A000C4F8C4704FF44033C4F8D4308C23C4F8AB
:10D4B000BC3000F1100302F1AC01C4F8B0304FF4FD
:10D4C00080424FF40063C4F8C830C4E93755414482
:10D4D000C4F8CC20C4F8B850C4F8C050C4F8D05038
:10D4E000C4F8E450304649F0E5FD336823637369BE
:10D4F00063637368A363B368E363F36823643368A7
:10D5000043F0100333609CE5500806082802002011
:10D510008801002004240020000401409819002004
:10D5200000000140D0DD060044950800105522009F
:10D5300040771B006000010000600240F80E001000
:10D5400000380240481906086D850008019B01213A
:10D55000002B7FF419AD35E5C6F12F06B2403A43F2
:10D560002265039A009D55831A46FAF7DBFF9AE578
:10D57000184A032382F8693A13B0BDE8F08FD8B295
:10D58000431E0CE7FDF7B8FB0B9038B1069B022158
:10D59000DA79FEF723FB0B9B5422DA80B5F844308E
:10D5A0006FEA43436FEA53439BB2A5F84430E3E686
:10D5B00009490A4AA4E6074A022382F8693A13B0E5
:10D5C000BDE8F08FDB0020E700239B88FFDE00230F
:10D5D0005B68FFDE98190020882A1100A0BB0D00AF
:10D5E0000C2911D8DFE801F02310101019101010C9
:10D5F000111010100700838B23F400631B041B0C15
:10D6000043EA02239BB283837047838B23F0080392
:10D610001B041B0C1A4382837047038B23F40063A3
:10D620001B041B0C43EA02239BB203837047038B4A
:10D6300023F008031B041B0C1A430283704700BF2E
:10D640002DE9F04FDFF85CB39BF804719BB01FB974
:10D6500000201BB0BDE8F08F00222F21384610F0CB
:10D6600087FD80460028F3D0DFF83C930568C9F8B1
:10D67000405AFDF741FF0028EAD0D0E90143019369
:10D68000C9F83C4A002CE3D0BA4E0022314601E0F2
:10D69000102ADDD04868844201F1240102F1010220
:10D6A000F6D1D2B2DFF804A3013A02EBC2020AEBD0
:10D6B000820292F9BC100029CAD138462F27A2F85D
:10D6C000BC70FDF719FBCBF8080128B1C78098F8AA
:10D6D00007202A21FEF782FAA74F002207F6E4402E
:10D6E00050F832108D4200F0128101320E2AF7D12B
:10D6F00000204DF0B3F92988D9F8F42021F0010178
:10D700000904090C29809D498D4200F0E880A1F5AB
:10D7100080618D4200F0E38001F580418D4200F090
:10D72000DE8001F580618D4200F0D98001F58061D5
:10D730008D42934900F00A81B1EB520F4FEA52003B
:10D7400040F2F88001220021B0FBF2F2ADF80C109B
:10D750008C498D48120AA1FB02121109A0FB01019C
:10D760004908ABF80E11490000271209ABF80C115B
:10D77000284603A90492ADF81470ADF80E708DF828
:10D78000167049F039FD98F80630ADF81C7060222B
:10D7900006929A07CDE908770A9798F8057040F144
:10D7A000A380DB0003F008034FF00408ADF8263037
:10D7B000ADF81C8006AA39462846FFF78DFA0822E4
:10D7C0003946FFF70DFFB5F844206FEA42426FEA91
:10D7D000524292B2A5F844202A8892B242F08002C6
:10D7E0002A802A8C08FA07F39BB292B222EA03023B
:10D7F0002A842A8C92B213432B842B889BB243F049
:10D8000001032B803246002351688C4202F124022E
:10D8100003F1010376D0102BF6D14FF0FF3303EB69
:10D82000C3030AEB830A594ADAF8A03058498B42FD
:10D8300014BF4FF480034FF40013116B0B431363B9
:10D8400000237268944206F1240603F101035CD0C0
:10D85000102BF6D100204F4960220023FDF748FF2E
:10D86000204649F091FB236823F001032360204602
:10D8700049F08AFB019B0B9305F134033B440C9365
:10D8800040F22A430F934FF480631193424B0D9360
:10D8900040230E934FF480504FF480430026CDE98F
:10D8A00012030BA94FF440332046CDE91666CDE9AB
:10D8B000186610961496159349F0FCFB0C2F04D8AB
:10D8C000364B03EB4703B3F88C60AB899BB2334311
:10D8D000AB81236843F0100301202360B9E6284997
:10D8E0008A4219D2002131E75B0003F00203ADF850
:10D8F00024304FF001084FF48073ADF81A80ADF872
:10D90000283057E7DBB2013B89E7D8B2A3E707EB42
:10D91000C20797F8E80CECE6214802F1B77101F56F
:10D920005851A0FB0101890D013989B2481CB2FB95
:10D93000F0F20BE71A4900F1B77202F55852A1FB59
:10D940000221890D013989B24A1CFDE68A4204D2BE
:10D9500001200021B2FBF0F2F8E6114802F1B771A4
:10D9600001F55851A0FB0101890D013989B2481C0C
:10D97000F0E700BF2802002050080608000401401C
:10D98000006CDC02598B4F01ABAAAAAA00380240F6
:10D9900000600240058800089C77002048190608AE
:10D9A000819F5E16902A002098190020880100208F
:10D9B0002DE9F04FDFF8709299F8003089B01BB96B
:10D9C000012009B0BDE8F08F934B1C68FCF796FC72
:10D9D00099F8C8350393002B00F012828F4BA3FBFC
:10D9E00004328F4B5209A3FB0213DB0803EB8303C2
:10D9F000A2EB4303D9F8042B821A049209F6083BE0
:10DA0000DAB207920BEB830309F5C66409F6E85214
:10DA1000029200279846019432E0304649F0B4FA69
:10DA20008C2303FB0793002583F824569AF805A05E
:10DA3000204651462A46FFF7D3FD019C2246FFF7B8
:10DA40004BF951460822FFF7CBFD402344F83C3CFC
:10DA5000A4F14801304649F02DFB04F18C030193F9
:10DA6000029B14330293336843F010033360039B2B
:10DA700001379F420BF15C0B08F15C0800F0D68087
:10DA8000049A002A05DB019B53F8083C934200F3FB
:10DA9000A2818C23019A03FB079352F858AC93F8A8
:10DAA0002436166ADAF80040002BB6D07568A389D0
:10DAB000ADB2114632F8542CC5F116059BB223EADB
:10DAC0000203072DA381A8D9D9F8F03D8A6A013352
:10DAD000C9F8F03D0021CDE90572106896468C46E4
:10DAE000012315E0BCF1140F1EDC12F1080748BF3A
:10DAF00002F117073A110CEB271C571E01FA02F22C
:10DB000001210B4401FA07F79D4247EA02010BD3BA
:10DB100002465EF8040F9D42A0EB0202E2D8CCF16F
:10DB200015024FF0150CE8E7BCF1150FDDE90572A1
:10DB300066D13C4DC1F38423C1F3441005EB83034C
:10DB400005EB8000D3F8A830D0F8A8001B0243EA08
:10DB5000001301F01F0005EB8000C1F3C43105EB99
:10DB60008101D0F8A800D1F8A810034343EA01339B
:10DB700083EA132181EA111101F00F010F293FD12E
:10DB8000C3F30F134FF6FF718B4239D0B3F5606FBB
:10DB900000F02581029A93819BF8582007988242D1
:10DBA00014D0D8F80810DBF80020521ACBF8002067
:10DBB000D8F83010DBF80420521ACBF804200022E9
:10DBC000C8F80820C8F830208BF85800DBF800208F
:10DBD0000132CBF80020D8F808200132C8F808201C
:10DBE0004FF6FF7293427FF418AFDBF80430013335
:10DBF000CBF80430D8F830300133C8F830300CE7B7
:10DC0000D9F8EC3D0133C9F8EC3D002F00F0D98084
:10DC10004FF6FF73C0E700BF981900201F85EB5136
:10DC2000CDCCCCCC4819060804000010D9F8D81582
:10DC3000C9F8045B012389F8EC3E0A68487999F831
:10DC4000E015890748BF0423118C83409BB289B239
:10DC500021EA03011184118C89B20B431384039BC5
:10DC6000012B3FF4ADAED9F864261368517999F8C9
:10DC70006C26970754BF012204228A40198C92B265
:10DC800089B221EA02011984198C89B20A431A84E3
:10DC9000039B022B3FF494AED9F8F0261368517918
:10DCA00099F8F826960754BF012204228A40198C5D
:10DCB00092B289B221EA02011984198C89B20A430D
:10DCC0001A84039B032B3FF47BAED9F87C2713689F
:10DCD000517999F88427950754BF012204228A407C
:10DCE000198C92B289B221EA02011984198C89B285
:10DCF0000A431A84039B042B3FF462AED9F8082828
:10DD00001368517999F81028940754BF012204220E
:10DD10008A40198C92B289B221EA02011984198CC5
:10DD200089B20A431A84039B052B3FF449AED9F804
:10DD300094281368517999F89C28900754BF0122C0
:10DD400004228A40198C92B289B221EA0201198414
:10DD5000198C89B20A431A84039B062B3FF430AE18
:10DD6000D9F820291368517999F82829920754BFC6
:10DD7000012204228A40198C92B289B221EA02015E
:10DD80001984198C89B20A431A84039B082B7FF4E7
:10DD900017AED9F8AC2999F8B4191368507911F075
:10DDA000020F18BF0422198C08BF0122824092B2D0
:10DDB00089B221EA02011984198C89B20A431A84B2
:10DDC000FEE511461248582252F0AEFADAF8004049
:10DDD0004FF6FF73E0E6002009B0BDE8F08F0D4973
:10DDE00091F88E2002EB420201EBC2023A4492F813
:10DDF0009D200D2A7FF4CEAE029980228A77CBE651
:10DE0000012389F8EC3E039BC9F8043BD8E500BF29
:10DE1000980E0010981900200B4B93F82421D3F88A
:10DE200014313AB113B11A689B885383074B00220F
:10DE30001A827047002BF9D01A689B881383034B12
:10DE400000221A82704700BF902A00200010004074
:10DE50000B4B93F82421D3F814313AB113B11A685B
:10DE60009B881383074B00221A827047002BF9D03E
:10DE70001A689B885383034B00221A82704700BFA5
:10DE8000902A00200014004037B590F85F38032B2B
:10DE900004462FD10023204D8DF807309DF8073020
:10DEA00094F860289A4201D803B030BD9DF807303D
:10DEB00005EBC30393F82C318BB181F0010383B1DF
:10DEC0009DF8073005EBC303D3F82801FDF76CF884
:10DED0009DF807300133DBB28DF80730DEE70B46E3
:10DEE000EDE79DF8073005EBC303D3F82801FDF7F4
:10DEF00061F8EDE7D0E910039B7903F00103994243
:10DF000004D003B0BDE83040FDF74EB803B0BDE823
:10DF10003040FDF74FB800BF902A002038B50446C6
:10DF200000790D4650B1FCF7E7FE08B10323C3802A
:10DF3000E2792946BDE83840FDF792BE38BD10B5FC
:10DF400004462221FFF7EAFF6379216802229B0839
:10DF500002FA03F3DB439BB20B8263798889D340D7
:10DF60009A40024392B28A8110BD10B50446012145
:10DF7000FFF7D4FF206861798389890802229BB268
:10DF80008A4023EA0203838110BD38B510F8133CA0
:10DF9000A0F664041BBB94F850388BBBD4E909236A
:10DFA0009A421CD05A1CA169A262CB5C21695B0019
:10DFB00043F40073A4F854380A2384F85238012338
:10DFC00084F8503894F85F388A4228BF0022012B29
:10DFD000A26201D0042B02D1606CFFF7C6FF94F857
:10DFE0004C38002B6DD194F84D380133DBB2092B3E
:10DFF00084F84D3825D12046BDE83840FAF784BC76
:10E0000094F952586DB1B4F854184B08A4F8543828
:10E0100001F001012046013DFFF736FF84F8525818
:10E02000DDE7D4E909239A4284F85058D7D194F80F
:10E030005F38012B01D0042BD1D1606CFFF77FFF3B
:10E04000CDE70A2B3DD194F84F382BB9B4F85638A8
:10E0500043F00103A4F856382379D9070AD5B4F858
:10E060005608820501D4C30718D4B4F85C380133CC
:10E07000A4F85C38012284F84C2894F84F28002337
:10E08000012A84F84D381CD1617984F84F38606CCE
:10E0900001F00101BDE838404CF09EB9E36AC0F3DD
:10E0A000470013B1216B9847E4E7E3696269D054F4
:10E0B000E369E2680133B3FBF2F102FB1133E36180
:10E0C000D8E738BD1648174A174938B5174C184DC8
:10E0D000121A52F029F9D4F88820164B164842F447
:10E0E0007002C4F888201A68002142F001021A6008
:10E0F00099601A6822F0847222F480321A605860A3
:10E100001A6822F480221A600C4AD960521B2846F1
:10E110000B4952F009F9A560BDE83840FAF74EBC4A
:10E120000000001004000010BB38070800ED00E0FC
:10E130000000002000380240103000248801002038
:10E1400000000008144BD3F8F430B0EB930F14D256
:10E15000B0EBD30F13D2B0EB131F12D2B0EB531F9F
:10E1600011D2B0EB931F10D2B0EBD31F0FD2B0EB94
:10E17000132F0ED24FF48070704702207047042096
:10E1800070470820704710207047202070474020BB
:10E1900070478020704700BF98190020154A08B5C5
:10E1A000D2F8BC366BB119689B88086992F8B91629
:10E1B000034021B12BB1002382F88C3608BD002B1F
:10E1C000F9D092F88C36032B0ED892F880360133B2
:10E1D000DBB2072B82F88036EDD81368C2F87C36A4
:10E1E000012382F88C3608BD0348FFF7ABFFA2F885
:10E1F000C406EAE798190020801A06002DE9F041CC
:10E20000334C0546884617461E4694F88C0604286B
:10E210000BD0082807D1D4F88436AB4244D0FBF7A2
:10E2200077F90228F1D001203AE094F88236002BE9
:10E2300038D169021820FBF7B7F8C0B2B0BB94F828
:10E240008C36082B30D0FE21224BD4F8C02683F820
:10E250006811214B117BC3F8088351B1526942B157
:10E2600094F84827002A14BF4FF400724FF48072CC
:10E2700001E04FF4807219481949C3F8102343F0A4
:10E28000C3FB01220623C4F86886C4F86C56C4F8A0
:10E290007476C4F8786684F8702684F88C3600208A
:10E2A000BDE8F0812946C5E7FC21CDE7D4F8C026BA
:10E2B000136A002BFCD14DF085FCD4F8C83613B19D
:10E2C0001A689B881383FFF769FF0320E8E700BF04
:10E2D00098190020902A0020880100205820002052
:10E2E0006804002070B5224E96F88C36042B054643
:10E2F0000C4609D0082B22D1D6F8843683421CD094
:10E30000FBF706F902281AD100213720FBF74CF859
:10E3100021461720FBF748F8C0B2C0B996F88236FC
:10E320007BB969021920FBF73FF880B9082386F80A
:10E330008C36C6F88846C6F88456022070BD012087
:10E3400070BD29461920FBF72FF80028EED0D6F82B
:10E35000C026136A002BFCD14DF034FCD6F8C83629
:10E3600013B11A689B881383FFF718FF032070BD51
:10E3700098190020F0B503792E4C002B14BF012210
:10E3800000228BB084F8B82603D184F88C360BB009
:10E39000F0BD054604F5D86790F90010384643F003
:10E3A00063FBAE78002E38D1234B2448C4F8543791
:10E3B000C4F8C866FFF7C6FEA4F8C4064FF47A7026
:10E3C000FCF75CFBD4F8C83613B11A689B8813833A
:10E3D0001B4D0FCDEC46ACE80F000FCDACE80F00A5
:10E3E00095E803008CE803006946384643F00CFBCF
:10E3F000D4F8C026136A002BFCD11EB10921304687
:10E40000FCF7BCFB2168C4F87C160122002384F8C9
:10E410008C2684F880360BB0F0BD3046FCF76CFCDF
:10E4200006460028C0D01E23C3802821FCF7A6FB87
:10E43000BAE700BF9819002000200020801A0600CB
:10E44000701A0608F0B59F4C94F8B86693B0002E89
:10E4500000F0DE8194F88C365A1E082A00F265819D
:10E46000DFE812F039007100BC006301340175016E
:10E470001A00630109004BF015FB002840F0A5824B
:10E48000D4F87C362268FA33934280F04B81FFF750
:10E4900085FE94F88C36DFE74BF004FB0028EFD0C4
:10E4A000D4F888260023012A84F8803640F29E8220
:10E4B000D4F88416013A01310823C4F88826C4F838
:10E4C000841684F88C36A3F10806B6FA86F6760927
:10E4D000304613B0F0BD00210846FAF765FFD4F8C6
:10E4E000C026C5B2136A002BFCD14DF06BFBD4F8EB
:10E4F000C83613B11A689B881383012D40F012812E
:10E50000002740F2AB11082084F88176FAF74CFF1F
:10E51000C0B2052800F0C581012800F0A381D4F81D
:10E52000C026136A002BFCD14DF04CFBD4F8C83642
:10E5300013B11A689B88138394F88136002BC0D0DE
:10E54000022384F88C3694F88156A5F10205B5FAB9
:10E5500085F56D090021AD073720FAF725FF29461B
:10E560002920FAF721FFD4F8C026C5B2136A002B80
:10E57000FCD14DF027FBD4F8C83613B11A689B883C
:10E580001383002D40F0CE8094F88136022B00F0EA
:10E59000D0810021092084F88256FAF705FF00286F
:10E5A00000F084810025D4F8C026136A002BFCD12A
:10E5B0004DF008FBD4F8C83613B11A689B88138352
:10E5C000002D00F0AF8000210A20FAF7EDFEC0B266
:10E5D000002840F09E81032384F88C36102103A884
:10E5E000FAF752FF002840F09D809DF80C30BDF8EE
:10E5F0000D209DF80F1063F307009DF8193052BAF3
:10E600001B01A4F894269DF81A20DBB243EA1213EA
:10E6100003F5FA63A4F8A23602F00F0384F8A436D7
:10E620009DF81030D4F8C02661F30F2063F3174033
:10E63000BDF812109DF81130A4F89A16DDF81510E7
:10E6400063F31F609DF81430C4F8960609BAC4F845
:10E650009C16190903F00F0384F8A01684F8A1365C
:10E66000136A002BFCD14DF0ADFAD4F8C83613B1C3
:10E670001A689B88138394F88236ABB94FF4007103
:10E680001020FAF791FED4F8C026C5B2136A002B09
:10E69000FCD14DF097FAD4F8C83613B11A689B88AC
:10E6A0001383002D7FF4F3AE0748FFF74BFD0022E4
:10E6B0000423A4F8C4063046C4F8882684F88C36AF
:10E6C00013B0F0BD9819002040787D01D4F8680699
:10E6D0004FF40071FAF7D8FE012800F09E8002285E
:10E6E00000F0A280F0B9D4F8C026136A002BFCD148
:10E6F0004DF068FAD4F8C83613B11A689B881383B2
:10E70000D4F874560423002084F88C3684F88006EC
:10E71000002D3FF4DDAED4F87836D4F86826D4F86E
:10E720006C16A84794F88C365A1ED2B2022A0AD820
:10E730002268D4F87C16521AC82A7FF6C4AEFFF7B6
:10E740002DFD94F88C36042B7FF4BDAEC0E6D4F8D2
:10E75000C026117B136A002946D05269002A43D093
:10E7600094F84827002A3FD0B3FA83F35B09002BC3
:10E77000D8D002A9002303910221CDE904310DF183
:10E78000070101220991B948ADF8083003A9CDE984
:10E790000733CDE90C33CDE90E338DF818308DF801
:10E7A0002C3011930A928DF8402043F02DF9D4F8C3
:10E7B000C0361D6A002DFCD19DF8073003F01F0301
:10E7C000052B00F0EB80FFF7E9FCD4F87476002FFE
:10E7D0003FF440AED4F87836D4F86C162A460120BF
:10E7E000B84794F88C3637E6D4F8683694F8700653
:10E7F00003EB00204BF00AF994F870360133DBB2DA
:10E8000084F87036A3F10203B3FA83F35B09AEE731
:10E81000304684F88C6613B0F0BDD4F87C3622689C
:10E8200064339342BFF47EAFD4F8C026136A002B42
:10E83000FCD14DF0C7F9D4F8C83613B11A689B88DB
:10E840001383FFF7ABFCD4F87456002D3FF402AEEF
:10E850000022D4F87836D4F86C161046A84794F8FD
:10E860008C36F9E502ABCDE9037380488DF818705A
:10E87000042303A9CDE90777CDE9097705938DF83E
:10E880002C500C9743F0C0F8D4F8C026136A002B24
:10E89000FCD19DF80B30AB2B04BF022384F88136EA
:10E8A0003FE6D4F8C02684F881563AE67048102135
:10E8B000FAF7EAFD00287FF475AE94F8B73613F046
:10E8C00001033FF46FAE94F8A826921100F0A280E5
:10E8D000012A7FF467AE94F8AF26664F9200D2B259
:10E8E00016210225C5F108038B4228BF0B46C3F150
:10E8F00008052A419840C91A40EA02004FF0000575
:10E9000017F8012FEED101308302C4F89036354656
:10E9100049E6D4F8C026136A002BFCD14DF052F919
:10E92000D4F8C836002B3FF4B2AD1A689B88138325
:10E93000ADE529463A20FAF737FD02ABCDE903539E
:10E9400004230593C7B2012348488DF82C3003A94E
:10E95000CDE90755CDE909558DF818500C9543F0D0
:10E9600053F8D4F8C0361A6A002AFCD17FB91A6A63
:10E97000002AFCD14DF026F9D4F8C83613B11A6834
:10E980009B881383029D2DBAC5F3807501E61A6A30
:10E99000002AC3D01A6A002AF9D1BFE7D4F8745606
:10E9A0002268C4F87C26072384F88C36002D3FF4B7
:10E9B0008AADD4F87836D4F86826D4F86C160120DD
:10E9C000A84794F88C365A1EAFE6D4F8C026136ACE
:10E9D000002BFCD14DF0F6F8D4F8C83613B11A6804
:10E9E0009B881383042384F88C3671E565D0042357
:10E9F000D4F8C02684F88C36136A002BFCD14DF075
:10EA0000E1F8D4F8C836002B3FF48CAE1A689B8826
:10EA1000138387E694F8AD06DFF85CC0114600F07A
:10EA20000F0294F8B10680019340C0B20325062777
:10EA3000C7F10802AA4228BF2A46C2F10807384196
:10EA40009140AD1A41EA00014FF000071CF8010F98
:10EA5000EED194F8AEC6DFF824E04FEA8C1C023108
:10EA60005FFA8CFC0C2006220BE000BF582000202F
:10EA70004020002047200020492000204620002080
:10EA80000022C2F10802824228BF0246C2F10807F2
:10EA90004CFA07F79540801A1EF801CF45EA0705A2
:10EAA000EED1013505FA01F2D817A2FB033102FBC2
:10EAB00000125B0A43EAC25327E7FAF729FD02284E
:10EAC0007FF430AED4F8C0361A6A002AFCD196E73B
:10EAD0002DE9F04F013B9FB2B44BDFF8D8C2D3F819
:10EAE000F4400B6883B06345BDF830609DF8345046
:10EAF0003AD0DFF8BCC2634536D00CF5804C634594
:10EB000000F042810CF5806C634500F03D810CF50E
:10EB1000806C634500F038816408B4FBF2F41A8815
:10EB2000013CB3F1804FA4B292B200F03781DFF81C
:10EB300088C2634500F032810CF5806C634500F0BB
:10EB40002D810CF5806C634500F02881DFF86CC2E4
:10EB5000634500F06481DFF868C2634540F01A81C4
:10EB60001A80DF621C850DE0B4FBF2F41A8822F4EF
:10EB70005C721204120C013C1A80A4B20022DF6203
:10EB80001C851A8601229A824C798A790DB182F00D
:10EB9000010212F0020C62D0D2004FF0000E02F01F
:10EBA00008074FF4806201924FF0400CF346CDF815
:10EBB00000E0F24672464FF0040975460C2C35D839
:10EBC000DFE804F0B73434348B343434073434346D
:10EBD0005E001C8CDFF8D8C124F480742404240C5B
:10EBE0001C841C8C24F4007424042A43240C9D8867
:10EBF00044EA02249A8B22F073021204120C634539
:10EC0000ADB242F0600200F0EB800CF5806C634521
:10EC100000F0E6809D809A83DE631C849A8B22F04C
:10EC200008021204120C42F008029A83B3F844203E
:10EC30006FEA42426FEA524292B2A3F844201A8825
:10EC40001C4692B242F0010224F8342B4A79436008
:10EC5000A11800230160A35003B0BDE8F08F4FF46A
:10EC600080655200CDE9005C02F002024FF4805E44
:10EC70004FF4804B4FF4807A6746E14601259DE7CB
:10EC800015431A8C4A4F22F480521204120C1A8433
:10EC90001A8C22F400521204120C42EA05329D88AA
:10ECA0009C8B24F4E6442404240CBB42ADB244F40F
:10ECB000C04400F0AF8007F58067BB4200F0AA8037
:10ECC0009D809C831E641A849A8B22F40062120435
:10ECD000120C42F400629A83A8E71C8CDFF8D0E0A3
:10ECE00024F010042404240C1C841C8C24F0200424
:10ECF00024042A43240C9D8844EA02141A8B22F42B
:10ED0000E6421204120C7345ADB242F4C04259D02F
:10ED10000EF5806E734555D09D801A839E631C84CA
:10ED20001A8B22F400621204120C42F400621A835D
:10ED30007CE71C8CDFF878C024F001042404240C48
:10ED40001C841C8C24F0020424042A43240C9D8877
:10ED500014431A8B22F073021204120C6345ADB2F5
:10ED600042F0600249D00CF5806C634545D09D802F
:10ED70001A835E631C841A8B22F008021204120CA0
:10ED800042F008021A8351E7B4FBF2F2541E1A88CB
:10ED9000A4B292B222F4407292B2E1E622F45C7222
:10EDA00092B21A80DF621C85ECE600BF9819002041
:10EDB0000000014000040140000400400010004039
:10EDC0000014004024F0800444EA0714009F25F456
:10EDD000406524F040042F434CEA04043D469BE781
:10EDE00024F4006444EA0724019F24F4806425F499
:10EDF00040553C434EEA05050CE74FF6F37C04EA28
:10EE00000C0C25F440754CEA070C45EA0A054CEA5F
:10EE10000904ACE725F480454BEA050550E7ACF85A
:10EE20000020CCF82C70ACF82840ABE6274A92F8CA
:10EE3000F83A7BB3D2F8381A884237D0012B29D060
:10EE4000D2F8501A814235D0022B23D0D2F8681A5A
:10EE5000884231D0032B1DD0D2F8801A88422DD0A1
:10EE6000042B17D0D2F8981A884229D0052B11D03C
:10EE7000D2F8B01A884225D0062B0BD0D2F8C81A87
:10EE8000884221D0072B05D0D2F8E01A814208BF72
:10EE900007230CD003EB430102EBC10103F1010C8A
:10EEA000C1F8380A82F8F8CA184670470023DBB266
:10EEB000184670470123FAE70223F8E70323F6E731
:10EEC0000423F4E70523F2E70623F0E7040000102B
:10EED000024BD3F860361B6A184700BF9819002010
:10EEE0000A4AD2F8BC3673B119689888096992F851
:10EEF000B93608401BB1B0FA80F0400970470038BD
:10EF000018BF012070470120704700BF98190020EA
:10EF1000034BD3F8600608B183691847704700BFF8
:10EF2000981900200378022B12D00F494368026918
:10EF3000D1F8480810B41840D1F84048D1F83C182E
:10EF4000931E400A04FB030008445DF8044B70471D
:10EF5000054B4268D3F83418D3F8300800EB410071
:10EF600000EB5220704700BF546900202DE9F04F9C
:10EF700012F0020A8E4E83B09B4601D0002853D077
:10EF8000D6F83858002D3AD14FF0FF3C894C8A4FC3
:10EF9000CDF804C0E046E646002300922268A57B37
:10EFA00090424DD025B303F5B179012D07EB091936
:10EFB0000ED199F80750EA070AD415F07E0F07D151
:10EFC000ED0940F0A780A568AE4584BFAE469846DF
:10EFD00001330B2B04F11004E0D1BCF1000F009AB7
:10EFE00080F2C280019B002BC0F2A480019B2BE029
:10EFF0009C4601330B2B04F11004CFD1EDE7D6F87A
:10F000004048D6F83C3804FB05339842BCD396F808
:10F01000E43713B9012386F8E437674B01225A70AD
:10F02000002003B0BDE8F08F96F8E437A6F58054D1
:10F03000002B7BD001230220637003B0BDE8F08F6A
:10F04000009A002D40F092805B4CD6F8C85604EB35
:10F05000031C41F2186E01354CF80E0041F21C6E93
:10F0600003F5B1774CF80E504FEA071CC6F8C856A6
:10F0700044F80C5004EB07154FF0000CC5F804C021
:10F0800004EB0715AD79042D4CD80FF2080C5CF891
:10F0900025F000BFA9F00008D9F0000821F0000811
:10F0A000D9F00008DFF0000812F001056DD104EB83
:10F0B00007104FEAE20C90F807E0BBF1030F6CF386
:10F0C000C71E80F807E05ED94FF6FF70584528BF8D
:10F0D000584604EB0715A880BAF1000F30D150074D
:10F0E00005D504EB0715E87940F00100E871D20678
:10F0F00008D504EB0717FA79C2F34500013060F335
:10F100004602FA712D4A012002EB43220A6003B045
:10F11000BDE8F08F019301330B2B04F110047FF451
:10F120003DAF5AE796F8E437002B83D1012386F8E8
:10F13000E4377FE7B8F1000FA8BF434684DA6FE7F2
:10F14000D6F8C806D6F8CC5601300135C6F8C80640
:10F15000C6F8CC5604EB031541F21C66A85104EB2B
:10F16000071004258571BAE763466DE7D6F8C856DF
:10F17000114C03F5B1774FEA071C013544F80C50E8
:10F18000C6F8C8567CE72846A3E70C490C4A01EBB1
:10F1900043210C4BD3F860369D680023A847002814
:10F1A0003FF43EAF04EB07170223BB7138E700BF03
:10F1B000546900206C6F0020545900206C590020C5
:10F1C000E99500089819002070B5104E3378022B8D
:10F1D0000F4B0BBF020AC0F3D412C4B200F07F047D
:10F1E000D3F8300882B010440D460023032201A951
:10F1F000FFF7BCFE012807D13378019A022B0CBF20
:10F2000022F8145042F8245002B070BD5459002026
:10F21000546900202DE9F04FDFF820910D4699F850
:10F2200000102B68032985B0164640D0022966D10C
:10F230004FEA132A5FFA83F84FF4807B421E012ABB
:10F2400024D801249E421CD901288CBF002201220F
:10F25000394F0192D7F8A8271AB1D7F8C4179942A5
:10F2600050D0D7F8300800235044092203A9FFF7F3
:10F270007DFE012824D0022815D020B12B689E42A3
:10F28000E8D82E60032005B0BDE8F08FB8F1000F7C
:10F2900014D0294B93F8E42712B9012283F8E4270C
:10F2A000012389F80130022005B0BDE8F08F4FF04E
:10F2B000800BC3F3D41A03F07F08BFE75C46C1E7B5
:10F2C00099F80010022916D00329ECD1039B53F8BA
:10F2D000282022F07042019BD5F800C0B2FA82F2D9
:10F2E00052099A4220D0A0440CEB0403D8452B606D
:10F2F0001DD20229EAD1039B33F81820EBE74FF423
:10F30000807BD6E7D7F84018013A02EB4122490248
:10F31000B2FBF1F21344B3FBF4F204FB12320AB174
:10F3200023449B1A2B60AAE76645ACD8A9E70AF1EB
:10F33000010A4FF00008A2E7546900205459002048
:10F340002DE9F04FDFF850910B6899F800C017468F
:10F3500009F58052BCF1020FD2F8305883B08B46C9
:10F36000824640F08180DEB2A6EB030805EB132550
:10F37000B8444FF480729044BB4208F1FF38B8FBA8
:10F38000F2F843D2A844BCF1030F06EB0704A4EB48
:10F39000030414BF4FF4807280229442A8EB05034B
:10F3A00028BF1446B6BB944234BF0B220A2201A9DF
:10F3B0002846FFF7DBFD012829D199F800C0DBF8CA
:10F3C0000000BCF1020F00F1010325D0A64210D2CB
:10F3D000019906F18042013A01EB8202043901EB06
:10F3E000840142F8043F8A4203F10103F9D1DBF8BA
:10F3F0000000A31B0344BAF1010FCBF8003023D067
:10F400009F4205F101054FF00006BCD8012003B072
:10F41000BDE8F08F0B22CAE7A642EAD2019906F1B5
:10F420000042013A01EB4202023901EB440122F8A9
:10F43000023F8A4203F10103F9D1A31B0344BAF14D
:10F44000010FCBF80030DBD1BB42D9D1BCF1020FA8
:10F45000019B18D004F18044013C4FF0FF3243F887
:10F460002420DBF80030CBE703F07F06C3F3D4128F
:10F47000BCF1030FA6EB03081544B84414BF4FF4C6
:10F480008072802277E704F10044013C4FF6FF725E
:10F4900023F814200120BAE75459002030B504465F
:10F4A000C06983B010B9012003B030BD0D46002300
:10F4B000032201A9FFF75AFD0128F5D1B4F9202054
:10F4C000002A19DB019B012D4FEA421103EB421286
:10F4D00003D0022D1BD1E5205854A368D3612378B3
:10F4E000032B04D10023137753779377D377636A81
:10F4F00053831B0C9382D6E7064A92F8E41709B9A6
:10F5000082F8E407044B01225A700220CCE7E3683A
:10F51000E4E700BF54690020545900202DE9F0436E
:10F52000022383B004460F4694F83C20042A7DD879
:10F53000DFE802F02F0371504000434EDFF81091D6
:10F540004FF6F77806F5805518E0C44561D84AF0C3
:10F5500033FA01284FF00001034637D1206BFFF743
:10F5600033FE0128034631D10198D5F844182063B1
:10F57000421E8A4228BF0A46C5F844283078226BCA
:10F58000032801A910461FFA82FCDED14A45DED9C4
:10F590003FE0790001F0FE012046FFF77FFF0128E0
:10F5A000034643D1626B002A14BF0222012284F871
:10F5B0003C20B9E794F82830042B04BF002384F8DA
:10F5C0002830A36B0BB1204698470123184603B09F
:10F5D000BDE8F0831D48E26AD0F8C437C0F8C427FC
:10F5E0009B1AD0F8402802FB03F3D0F8A82702EBBF
:10F5F0004322C0F8A827D0F8AC2702EB4322C0F87A
:10F60000AC27002100F5F460FFF748FF012803460E
:10F610000CD10422CBE7626B04F130010020FFF72C
:10F620008FFE0128034601D10322C0E7022BCDD172
:10F6300094F82820042A08BF0022184608BF84F83E
:10F64000282003B0BDE8F0835459002054690020FD
:10F65000F7FFFF0F38B5044694F83430052B58D81F
:10F66000DFE803F0372B2319100394F82830082B18
:10F6700004BF002384F82830274B012283F8E527B4
:10F68000022038BD94F82830082B04BF002384F8EA
:10F690002830012038BD00212046FFF7FFFE012859
:10F6A00037D1042084F83400D6E7D4E90B01FFF702
:10F6B0008BFD01282DD10320F4E7206B4FF0FF31A3
:10F6C000FFF782FD012824D1E36A002BF3D002204A
:10F6D000E8E7114DD5F8382804F130010120023255
:10F6E000FFF798FD012805D00238C0B2012810D8D4
:10F6F0000520D7E7E368D5F84018226BC5F8442801
:10F7000003EB4123C4E90332E36A002BCAD16262EE
:10F71000C8E7002038BD00BF54690020F8B5044692
:10F72000022094F83830032B07D8DFE803F01F17C6
:10F730000B0200212046FFF7B1FE431EDBB2012B76
:10F740003FD9F8BD626B04F130010120FFF7F8FDED
:10F750000128F2D1032384F83830E2E71E48002163
:10F76000FFF79CFE0128E8D10223F4E71B4AE56875
:10F7700002F580531278D3F84018032A14BF4FF4CF
:10F780008072802202FB01F105EB4126D3F8C457B9
:10F79000C4E90365D3F8A867A6EB4126C3F8A867B8
:10F7A000D3F8AC67AF1AA6EB41212A44C3F8C427AB
:10F7B000C3F8AC17E36A2563626353B9656201233A
:10F7C000C9E794F82830062B04BF002384F82830BA
:10F7D000F8BD2763F3E700BFF47000205459002000
:10F7E0002DE9F0434368C3F308020A44B2F5007FF1
:10F7F00083B005460C4605D223446B60012003B05C
:10F80000BDE8F08390F91A20501C0AD0444902F553
:10F81000B17201EB0212D17921F00101D171FF2205
:10F82000AA7695F91B20511C0FD03D4802F5B17204
:10F8300000EB0210FF26C279C2F34501013921EA2B
:10F84000E17161F34602C271EE762A78022AD3D0C2
:10F85000DFF8CC8008F58057D7F84028B4EB422F6A
:10F860004FEA42292CDCD7F848681E407242A24277
:10F8700026DCA2194A45286913D32A7E12072BD504
:10F88000D7F8C427411C8A421CD300D100214B4425
:10F890009B1BA4EB0909686109EB060429616B60F5
:10F8A00008460028AAD098F80020032A33D080B256
:10F8B0004FF6F7729042A1D81A4614446C609DE747
:10F8C00000209CE797F8E4270ABB012387F8E43778
:10F8D00088F801306B68DAE701A94AF06DF8012871
:10F8E000EED16B68297828696861A4EB0904994412
:10F8F000A9EB060301986B600229344428611A467B
:10F90000CFD1D7F85018B3EB412FD6D376E70122E9
:10F9100088F80120BBE7034A90423FF66FAFCBE780
:10F9200054590020F7FFFF0F2DE9F047044682B03D
:10F9300094F83830032B00F2A980DFE803F0981721
:10F940000C02236C002084F8280003B198470220A1
:10F9500002B0BDE8F087236C002284F828200BB1A8
:10F9600020469847012002B0BDE8F08723786668FA
:10F97000474F022B1CBF464BD3F84838204618BFD0
:10F980001E40FFF7CFFAC6F34F26361A0546B6B229
:10F99000A7F5805811E0D7F84038013B994557D278
:10F9A000FFF71EFF40B997F8E43713B9012387F832
:10F9B000E437012388F80130013506EB050C0222FB
:10F9C00001A9002328461FFA8CF9FFF7CFFA012876
:10F9D0004FF400724FF00001BAD1019850F0FCFCD6
:10F9E000E3694FF400712046002BD4D06368002BEC
:10F9F000D1D1019B4FF020324FF02E0C4FF0100E62
:10FA0000C3F80120C3F80520A3F8092083F800C03B
:10FA100042F62E6AD4F824C0A3F820A083F80BE0A5
:10FA2000C3F82220C3F8262083F82A20E26BA3F82B
:10FA30001AC05A872CFA0EFC83F82BE022FA0EF239
:10FA4000A3F814C09A86D7F84038013B9945A7D34C
:10FA5000C3EBC35359022046FFF7C2FE28B997F8FB
:10FA6000E4377BB10B4B01225A70022007E020469D
:10FA7000FFF7F0FD012802D0022807D1032084F807
:10FA8000380055E7012387F8E437EBE700205FE70C
:10FA900054690020545900202DE9F041B1F9043097
:10FAA0000F2B82B00E460446174632D02046FFF791
:10FAB00039FA94F91B80B8F1FF3F3BD05C4B41F21F
:10FAC000186203EB08118A58904211D1183303EBE6
:10FAD0004825B38801331BB205EB4315B38020469C
:10FAE0003D60FFF71FFA3060012002B0BDE8F081F1
:10FAF00003F5805292F8E41700295CD001225A7075
:10FB00002378022B4CD02269002A60D100233B606D
:10FB1000EAE74FF40071FFF763FE002847D04FF685
:10FB2000FF73B3802046FFF7FDF994F91B80B8F10D
:10FB3000FF3FC3D12378022B41D02269002AE5D0B0
:10FB40003B4B1B78032B69D093B24FF6F7718B4276
:10FB500094BF00230123002BD6D138B9354B93F83D
:10FB6000E427002A4DD0324B01225A700023112283
:10FB700001A9FFF7FBF9012810D1019D2E4BEB1ACB
:10FB800048BF03F2FF13B3F5B05F4FEA63222DD2F3
:10FB90004FFA82F884F81B80002D9AD12378B0E7C1
:10FBA000244A6368D2F85028B3EB422FAED200202B
:10FBB00002B0BDE8F081012182F8E4179EE71D4BF9
:10FBC000D3F850286368B3EB422FC6D39EE7184B97
:10FBD0001B78032B19D093B24FF6F772934294BF60
:10FBE00000230123002B91D10020E1E7114B93F872
:10FBF000E42712B9012283F8E4270D4B01225A7041
:10FC0000C8E7012283F8E427ADE70C4B9A4294BF82
:10FC100000230123002B7FF479AFE5E7074B9A42DD
:10FC200094BF00230123002B7FF46EAF95E700BF44
:10FC300054590020546900206C590020F7FFFF0F31
:10FC40002DE9F043044689B094F83030042B11D8E4
:10FC5000DFE803F04B135C035500237E9A0640F166
:10FC6000E480E0690023112205A9FFF77FF901284C
:10FC700000F0DB8009B0BDE8F083CA4D01AE04F1AD
:10FC80001C07324639462846FFF706FF012800F0D8
:10FC9000E5800228EED1C44A02F5805595F9023874
:10FCA0005F1C0AD003F5B17302EB0313D97921F07D
:10FCB0000101D971FF2385F8023895F903385E1CDC
:10FCC0000FD003F5B17302EB0313DA79C2F34501E8
:10FCD000013921EAE17161F34602FF21DA7185F809
:10FCE0000318042384F83030AEE7AE484CF044F8F3
:10FCF0004FF6FF720123228484F83030A4E70020FD
:10FD0000E36A207009B0BDE8F0431847A74D95F8A5
:10FD10001038002BAED104F11C0701AE05F5FD68CB
:10FD2000324639464046FFF7B7FE012840F0EE80E4
:10FD3000DDF80490B9F1000F00F0C48099F80030AC
:10FD4000E52B01D0002BEBD1994AB9EB020248BF59
:10FD500002F2FF12B2F5B05F4FEA622380F0158124
:10FD6000914A1B0193490B44997B04290CD0D5F887
:10FD7000C8160131C5F8C816596004219973D5F821
:10FD8000CC360133C5F8CC3695F90238581C0AD068
:10FD900003F5B17302EB0313FF2185F80218D9793B
:10FDA00021F00101D97195F90338591C0FD003F5E1
:10FDB000B17302EB0312FF21D37985F80318C3F363
:10FDC0004501013921EAE17161F34603D371202233
:10FDD0000021484650F000FBD4F83130D4F83520EB
:10FDE000C9F80420C9F80030B4F8393094F83B2041
:10FDF00089F80A20A9F80830637E89F80B3005A835
:10FE000001F028FFBDF81430002B40F0098144F2C6
:10FE100081720321A9F81020A9F80E30A9F8182042
:10FE2000A9F8163084F830100EE720464BF0A4FFF6
:10FE30002369002B71D0237E03F0F70213F0040333
:10FE4000227677D1122A00F08C80E36A00222046C5
:10FE500084F8282009B0BDE8F0431847DDF8048095
:10FE6000B8F1000F00F0A88098F80030002B00F0E7
:10FE7000A38098F80B9019F0080F7FF402AF0B22C3
:10FE800004F13101404650F0E4FA00287FF4F9AE65
:10FE9000637E89EA0303DF0640F1F980424A02F5F6
:10FEA000805595F902385E1C3FF407AF03F5B17336
:10FEB00002EB0313FF2185F80218D97960F30001E2
:10FEC000D971FAE695F8E837022B4FF009023FF4B2
:10FED00008AF95F81038002B7FF403AF85F8203871
:10FEE000C5F82438C5F8283885F81C38D5F8FC370B
:10FEF000C5F814382B48D5F8443885F81028C5F8CB
:10FF00001838FFF711FD01283FF40AAF02287FF4EB
:10FF1000B1AE042384F8303096E6237E1B0794D5D7
:10FF2000224B93F8C827002A7FF4A4AE072283F857
:10FF3000C8278AE7A568E66A002384F8283029469E
:10FF40002046FFF74DFC002840F09B8094F82830B5
:10FF5000002B7FF48FAE0223C4E90B6584F82830B0
:10FF600088E6626AE16AA163042084F828002046DA
:10FF7000C4E90B22C4E9023384F83C306363636252
:10FF800009B0BDE8F0434BF0F7BE95F8E43713B97C
:10FF9000012385F8E437044A012353706FF00F03FF
:10FFA000E0E600BF3C710020545900205469002055
:10FFB0006C5900206C6F0020554A02F5805595F968
:10FFC0000238581C0AD003F5B17302EB0313D97938
:10FFD00021F00101D971FF2385F8023895F9033822
:10FFE000591C0FD003F5B17302EB0313DA79C2F396
:10FFF0004501013921EAE17161F34602FF21DA711D
:020000040801F1
:1000000085F80318237EDB067FF56BAE41484BF085
:10001000B3FE4FF6FF720223228484F8303013E6D9
:100020003D4B05A8B3F96C5101F04EFD4FF47A72C7
:1000300000234EF0ADFC3C2305FB030192B24FF4CC
:100040007A700023C1FB002302A801F073FD9DF824
:100050000A309DF80B209DF80E1042EA4312BDF8BD
:100060000830A3F2BC7342EA43229DF80D305B01D5
:1000700043EA51039DF80C1043EAC12392B29BB2AC
:10008000C7E6002E3FF4F6AD204633463AE6B8F810
:100090001420B8F81A30214D43EA02436362D5F8C0
:1000A0004028D8F81C30A3605202B3FBF2F102FBE7
:1000B000113109B113445B1AE36084F8199095F982
:1000C0000238134A581C0AD003F5B17302EB03132C
:1000D000D97921F00101D971FF2385F8023895F90A
:1000E0000338591C0FD003F5B17302EB0313DA790F
:1000F000C2F34501013921EAE17161F34602FF21B2
:10010000DA7185F80318032384F830309CE500BFCA
:10011000545900203C710020902A0020546900208E
:1001200070B50378017E023B012B044602D911F021
:10013000060F5BD18D063BD494F91A30581C0AD0B7
:10014000304A03F5B17302EB0313FF20DA7922F092
:100150000102DA71A07694F91B305A1C0FD029489D
:1001600003F5B17300EB0310C379C3F34502013A01
:1001700022EAE27262F34603FF22C371E2760B07C2
:100180000DD5214B93F8C827072A05D093F8E4270B
:100190009AB31C4A01215170002283F8C827E26AF1
:1001A0000023237084F82830FAB1BDE8704010476E
:1001B00000231648E5691A018258954206D001339A
:1001C0000B2BB9D01A0182589542F8D10D4803F58E
:1001D000B17300EB0310C379C3F34502013A22EA7D
:1001E000E27262F34603C371A6E770BD0121FFF717
:1001F00055F90128F9D1217E9CE7012283F8E427F3
:10020000C7E700BF54590020546900206C6F0020DC
:1002100038B5184D05F58054014694F8100820B9FA
:1002200061B191F8283013B138BD002038BD04F514
:10023000FD60442250F078F8012038BD44220E4879
:1002400050F0CAF82B78D4F84C18C4F80C180322D4
:100250004FF6FF70022B18BF1346A4F8020884F86B
:100260000028054884F8E837102284F801284BF06C
:1002700083FDE1E7545900203C7100204FF0FF3C22
:100280002DE9F041344A35486446002304E0013347
:100290000B2B02F1100216D011780429F7D103F5C7
:1002A000B17100EB0111C979CE07F0D4651C52F889
:1002B0000A1C01D08C45EAD91C4601330B2B8C4615
:1002C00002F11002E8D1002C02DA0120BDE8F08131
:1002D000224D04F5B17705EB0713998801BBDFF8D0
:1002E00088802601D8F86026AB19D2F810801C4E01
:1002F00041F2186206EB442198581A4A0023C0477D
:10030000D8B102280AD106F6E87605EB0715D6F82B
:10031000CC360122013BC6F8CC36AA710020D5E7C5
:10032000DFF8448005EB0413D8F8602641F218602A
:10033000D268185826019047D4E706F6E87605EB10
:100340000715D6F8CC360321013B0122C6F8CC367E
:10035000A97186F8D026E1E77A6F00205459002071
:100360006C5900205D960008981900202DE9F04393
:1003700090F82830013B83B00446082B0BD8DFE807
:1003800003F0393D1F24052A0A2F34000121FFF70D
:10039000C5F8012802D003B0BDE8F0832378216CB2
:1003A000002284F82820002BF5D0D4E901038342F1
:1003B0004FF0030238BF0346A36084F82820E162AF
:1003C000204603B0BDE8F043AAE6002103B0BDE833
:1003D000F043FFF7A3B803B0BDE8F043FFF79EB9C1
:1003E00003B0BDE8F043FFF735B903B0BDE8F04313
:1003F000FFF79ABA03B0BDE8F04321E4534F4268D7
:10040000D7F84858036BD7F8401894F800E0154027
:10041000E818B0EB412F4FEA412644D3A7F58059A5
:100420004FF6F778BEF1020F14D021690846002973
:1004300064D16068A368E26A834238BF0346002142
:10044000A36084F82810002AA5D0204603B0BDE898
:10045000F0431047D7F850186068B0EB412F35D201
:100460002069217E09073BD5D7F8C41700F1010C9C
:10047000614531D297F8E417002950D1012387F85C
:10048000E43789F8013094F800E06268236B9B1B25
:100490002B443244521B9E42C4E904C06260236371
:1004A0004FF00005BED9BEF1020F0ED02169002920
:1004B000BFD027480078032843D089B24FF6F770A1
:1004C0008142B6D898186060B4E76068D7F85018D1
:1004D000B0EB412FF6D3ADE7D9D14FF0000CD6E702
:1004E00001A949F069FA01287FF455AF2069DDF8C8
:1004F00004C094F800E06268236BC8E799F800C074
:10050000BCF1030F11D01FFA81FCC44594BF4FF01A
:10051000000C4FF0010CBCF1000FC8D1A1E7012184
:1005200089F8011094F800E0B1E7DFF828C06145D0
:1005300094BF4FF0000C4FF0010CBCF1000FB6D18E
:100540008FE7044881423FF674AFBBE7546900204F
:1005500054590020F7FFFF0F00B501EB020E714563
:1005600016D001390EF1FF3E41F2210C11F8013F86
:10057000082280EA032003B2002B4FEA4000B6BFF6
:100580008CEA430380B298B2013AF4D18E45EDD1A2
:100590005DF804FB704700BFD0ED007AD0ED016A32
:1005A00030EE677AE6EE877AB0EE670AC0ED007A41
:1005B000704700BFD0ED017AD0ED026A30EE677A65
:1005C00090ED000AE6EE877A37EEC07AC0ED017A48
:1005D000A6EE870A80ED000A704700BF90ED017A11
:1005E000D0ED036AD0ED027A30EE470AA6EE807AAB
:1005F00090ED000A80ED017A37EE676AE6EE867AC2
:1006000037EEC07AC0ED027AA6EE870A80ED000AC6
:10061000704700BFD0ED056AD0ED017A90ED066A13
:10062000D0ED025A90ED035AC0ED066AB0EE407A62
:1006300026EEA70AD0ED007A80ED057AA7EE870AAC
:10064000D0ED077AA5EE860A90ED086AD0ED045A3F
:10065000C0ED087AA5EE670AA5EEC60A80ED070A86
:10066000704700BFF0EE406AD0ED007A90ED050AC9
:1006700090ED067A90ED016AD0ED035AA7EEA60A36
:10068000A6EE267AD0ED047A90ED026A67EEC07A83
:10069000A5EEC07AE6EE267A80ED057AC0ED067A00
:1006A000704700BF2DE9F047DDF820A055460F4602
:1006B00015F8011B002B064614460CBF4FF020090D
:1006C0004FF0300939B3002A2BDD2B4600E09CB1F6
:1006D00013F8012BA046013C002AF8D1A8F102082A
:1006E00054B1444649463046B847013CFAD29AF8DC
:1006F000001008F1010459B13046B8472B4615F8EF
:10070000011B0029F8D1A4EB0A041819BDE8F087F1
:100710002046BDE8F087002A02F1FF38E1DC0846F8
:10072000F4E70024E8E700BF03685A1C0260197070
:10073000704700BF10B500F100440246013C04E0E0
:10074000B3EB0E0015D1A24214D012F8013BA3F175
:100750004100192811F8010BA0F1410C98BF20337A
:10076000BCF1190F00F1200EEAD91B1A04D10028A0
:10077000E9D110BD002010BD184610BD884210B54B
:100780004FF001043ED301FB04F4B0FBF4FC8C45B4
:10079000F9D2CCB122BB08E0A14203F801EBB4FBD3
:1007A000F1F211D8B0FBF2FC1446BCF1090F0CF1C8
:1007B000570E0CF1300204FB1C00EDDCA14203F8E3
:1007C000012BB4FBF1F2EDD900221A7010BDA14249
:1007D00003F801EBB4FBF1F2F6D8B0FBF2FC1446DF
:1007E000BCF1090F0CF1370E0CF1300204FB1C00B8
:1007F000EDDCA14203F8012BB4FBF1F2EDD90022AC
:100800001A7010BD8446002AEAD1CEE7002870B5E0
:1008100003DA2D2301F8013B4042092886464FF0B8
:10082000010307DD03EB83035B00B0FBF3F2092A4E
:10083000F8D8E3B10F4CA4FB0320BEFBF3F2092A66
:1008400002F1570602F130054FEAD00007DD092B0F
:1008500001F8016B03FB12EE09D90346EBE7092B04
:1008600001F8015B03FB12EE01D90346E3E7002325
:100870000B7070BDCDCCCCCC0378202B024600F1A0
:100880000100F9D0092BF7D02D2B28D02B2B03BF3B
:100890005378B7EE000A0246B7EE000AA3F1300122
:1008A000C8B209289FED567A10D8F2EE046A07EE16
:1008B000901AF8EEE77A12F8013FE7EE267AA3F1F4
:1008C0003001C8B20928B0EE677AF0D92E2B5ED07D
:1008D00003F0DF03452B07D020EE070A704753785B
:1008E000BFEE000A0246D9E710B451782D2978D01E
:1008F0002B296AD0A1F13003092B02F101026BD838
:100900000024002303EB830301EB430312F8011FD0
:10091000A1F130000928A3F13003F3D9B3F59A7F90
:100920001A4628BF4FF49A72072B66D9DFED356A55
:100930001346F7EE007A083B072B67EEA67AFAD843
:1009400002F00702DAB1F2EE046A012A67EEA67A33
:1009500015D0022A67EEA67A11D0032A67EEA67A8E
:100960000DD0042A67EEA67A09D0052A67EEA67A8A
:1009700005D067EEA67A062A18BF67EEA67A6CB392
:1009800087EE277A5DF8044B20EE070A704753780C
:10099000A3F13001C8B2092802F1010298D8F2EEA1
:1009A000046AF0EE665A07EE901AF8EEE77A12F84B
:1009B000013F87EEA66AA3F13001C8B2092866EEAE
:1009C000A56A37EE067AEED982E79178A1F1300375
:1009D000092B02F1020293D9F7EE007A27EE277A6B
:1009E000D0E79178A1F13003092B02F1020288BF10
:1009F000F7EE007AC4D8012483E7F7EE007AA1E786
:100A00000000000020BCBE4CF0B5067906F0E00303
:100A1000402B03D145794FF0FF3406E0602B4FF0B7
:100A20000105F8D1447905FA04F40023012006F009
:100A30000706AB4200D1F0BD052E0FD8DFE806F067
:100A40000308101D242448B1C85CD75C78400FE02F
:100A500020B1C856D756C71B784278410133E8E722
:100A60000028FBD031F8130032F81370784080B2C0
:100A700020420CBF01200020F0E70028EED031F921
:100A8000130032F91370E6E70028E7D051F823008D
:100A900052F82370DAE7F8B50C4E337805468BB977
:100AA000F8BD25B12388C3F30B039D4204D0D4E9DC
:100AB0000201A2884FF038FC1C34BC42F1D3002361
:100AC0003370EDE7024C034FF7E700BF4888002082
:100AD00060150708741E0708037903F01803102B2C
:100AE0001CD003D833B9B0F80B007047182BFAD0DC
:100AF00000207047104BB0F80B0093F90030591CE0
:100B000006BF0E4B1B78DBB203EB430203EB820301
:100B100003EBC30300EB430080B27047064BB0F811
:100B20000B0093F901305A1C06BF044B5B78DBB213
:100B300000EB4310F0E700BFA8050020002C0020C8
:100B4000032870B516D80C4BC60003EBC000C94390
:100B5000057A427A01F0010181EA0504A24209D036
:100B600042682AB190881268A94214BF108350834A
:100B700033445C7270BD00BF488800200379062BA7
:100B80000FD1C9B20D2998BF074BC26894BF5956FF
:100B9000002101238B40134214BF08464FF0FF3061
:100BA0007047481C704700BF68830608092900D0B9
:100BB00001B9704701394A0002F00802930001F0C0
:100BC0000301A3EB9203C1EB0111C3EB0313C1EBD0
:100BD000011100229B0089000260818043807047E0
:100BE000B5EEC00ADFED347AF1EE10FACCBF30EE8C
:100BF000270A30EE670ADFED317A20EE270A30B59A
:100C0000FDEEC07A87B017EE904A054684EAE4709C
:100C1000002303A9A0EBE470CDE90033029347F071
:100C200035FC002CB4BF2D23202303A88DF8003001
:100C30004DF050FA012829D0022833D003281DD0C6
:100C400003A968464FF0D0FB68464DF043FAC41E36
:100C5000E4B22246694628464FF066FB00232B5536
:100C600028464DF037FA2E232B5401300DEB0401AA
:100C700028444FF0E6FB284607B030BD302303A9D7
:100C800068468DF801304FF0AFFBDDE743F23002EC
:100C9000302303A96846ADF801208DF803304FF0EA
:100CA000A3FBD1E743F2300303A96846ADF8013056
:100CB0004FF09AFBC8E700BF6F12033A00007A4476
:100CC0000BF0E4BD38B5054658B14C1E14F8011FB1
:100CD000284619B9BDE838400BF0ECBD0BF0D6FD45
:100CE000F4E738BD70B50546B0F8090046F064F881
:100CF000054B1E7804462846FFF7EEFE16B1E36862
:100D0000184470BDA368FBE74888002038B5054645
:100D10000C46FFF7E7FF2A7902F0070302F0E00232
:100D2000602A29D1052B0CD8DFE803F0030B0F0B49
:100D30001B1B6A7901239340DBB2027814B1134381
:100D4000037038BD22EA0303FAE76A79012393406E
:100D50009BB2028814B113430380F2E722EA030333
:100D6000FAE76B7901229A40036814B113430360D8
:100D7000E7E723EA0203FAE7052BE2D8DFE803F00E
:100D80000303050507070470DBE70480D9E7046067
:100D9000D7E708B520214FF036FB0346184623B1AC
:100DA0000278202A03F10103F8D008BD08B5CB076B
:100DB00001D4FBF7A3FD08BD2DE9F341124D134FFC
:100DC000002305F8243F044600EB8106B44203D11A
:100DD0000F4802B0BDE8F081394628464FF004FBC9
:100DE000214668464FF02DFB4FF000082021684651
:100DF0004FF009FB28B9694628464FF0F5FA04344C
:100E0000E4E780F80080F1E74888002051FF0608F9
:100E10006C8800202DE9FF47914604468A461E460D
:100E2000FFF7ACFE421CBDF83070DDF8348005469B
:100E30001FD0B9F1FF3F1FD0CDE90009144A236844
:100E400031463846C0474A4620795FFA8AF1FAF7B8
:100E5000E7FA024600B10288D3B20393C2F3032338
:100E6000120BCDE90052029323680A4A31463846F4
:100E7000C04704B0BDE8F0877B06FAD40C90236825
:100E8000054A31463846C44604B0BDE8F0476047DD
:100E900090F306089DF30608C1F306082DE9F04318
:100EA000154685B06A1C8946BDF830600D9F19460D
:100EB00025D04FEA101800F00F0408F14008CDE9E2
:100EC0000045164A43463046B847A8B199F8051080
:100ED000D9F800002A46FAF7E5FA68B103880278E3
:100EE0000392C3F303221B0BCDE900430292434656
:100EF0000B4A00213046B84705B0BDE8F0837306C1
:100F0000FAD40309074A00F00F000C904033304632
:100F1000BC4605B0BDE8F043604700BFD0F306080B
:100F2000E2F306080BF406082DE9F04387B0070941
:100F3000DDF8388091461E46403700F00F0439B383
:100F40000CF0D4FFC379174ACDE9004305463B4670
:100F500049463046C047C0B12868FAF795FDAA79DE
:100F60006B79114912F0020F4FEA93030F4A18BF31
:100F70000A46E97900940133CDE90321CDE9010363
:100F80000B4A3B4600213046C04707B0BDE8F0831E
:100F9000084A0E943B4649463046C44607B0BDE871
:100FA000F04360471FF4060880F706086509070844
:100FB00031F4060853F406084840082341B24000C3
:100FC0000029C0B2B8BF5040013BF7D1704700BF05
:100FD00030B505688D42044618D901F1FF3E681E00
:100FE00000231EF801CF082183EA0C034FFA83FC8B
:100FF0005B00BCF1000FDBB2B8BF53400139F5D143
:101000007045EED16A1C22602B7030BD00236A1C33
:1010100022602B7030BD00BF10B52DED028B08EEA5
:10102000101AB8EE488ADFED7E7ADFED7E0A28EEF0
:10103000008A044628EE278AB0EE480A4EF06AFC81
:101040009FED797AB4EEC70AF1EE10FAF0EE407A2D
:1010500040F3BD809FED736ADFED746AB0EE677A8E
:10106000B4EEE67AF1EE10FA77EEC67AF6DC9FED92
:10107000707AF4EEC77AF1EE10FA40F3C5809FED76
:101080006A7A77EE677A27EEA76ADFED6A5ADFEDB4
:101090006A6A9FED6A7A9FED660ADFED620AE6EE04
:1010A000256A67EE865AA6EE267A38EE000AE5EE45
:1010B000877AB0EE678A4EF02DFCDFED5B7AB4EEF6
:1010C000E70AF1EE10FA5BDDDFED566A9FED577A25
:1010D000F0EE407AF4EEC77AF1EE10FA30EE660ADE
:1010E000F6DCDFED537AB4EEE70AF1EE10FA62DDDA
:1010F000DFED4D7A37EEC00AF7EE007ADFED504AA9
:10110000DFED4C5A9FED4C7AC4ED097AB0EE675A88
:10111000A8EE245A0023A36160EE006A87EE856A78
:1011200063612362E361A6EEA57A9FED445AA6EEC1
:10113000875A20EE264AF0EE675AA4EE050AE8EE3A
:10114000645ABDEC028BB6EE007AF8EE006A77EED8
:10115000C07A26EE077A66EE266A27EE277A66EED2
:10116000806A67EE867A25EE866A84ED007AC4EDA1
:10117000017A84ED027AC4ED036A84ED046A10BD3D
:10118000DFED307AB4EEE70AF1EE10FAA9D5DFED23
:10119000256A9FED2D7AF0EE407AF4EEC77AF1EEF3
:1011A00010FA30EE260AF6D4DFED217AB4EEE70A23
:1011B000F1EE10FA9CDCDFED257AB4EEE70AF1EEF1
:1011C00010FA44BFDFED1F7A37EEC00A94E79FEDB7
:1011D0001D7AB4EEC70AF1EE10FA7FF548AF9FED25
:1011E000116ADFED196AB0EE677AB4EEE67AF1EED5
:1011F00010FA77EE867AF6D49FED0D7AF4EEC77A80
:10120000F1EE10FA3FF73BAF9FED107AF4EEC77A9C
:10121000F1EE10FA44BF9FED0B7A77EE677A32E772
:1012200027D4D236DB0FC940DB0F4940E4CB16414F
:10123000DB0FC93F92E741B99730083C15A82ABE99
:10124000F304353FDB0F49C0E4CB16C1DB0FC9BF48
:1012500008B5DFED2D0A4EF05DFBDFED2C7AB4EE24
:10126000E70AF1EE10FA28DDDFED276A9FED287A14
:10127000F0EE407AF4EEC77AF1EE10FA30EE660A3C
:10128000F6DCDFED247AB4EEE70AF1EE10FA2FDD9A
:10129000DFED1E7A37EEC00A20EE007A9FED1E6A5F
:1012A000DFED1E6ADFED1E7AE7EE066A20EE076AC2
:1012B000E6EE877AA6EE270A08BDDFED1A7AB4EECD
:1012C000E70AF1EE10FADCD5DFED0F6A9FED167A32
:1012D000F0EE407AF4EEC77AF1EE10FA30EE260A1C
:1012E000F6D4DFED0C7AB4EEE70AF1EE10FACFDCBB
:1012F000DFED0E7AB4EEE70AF1EE10FA44BFDFED4F
:10130000097A37EEC00AC7E7DB0FC940DB0F494057
:10131000E4CB1641DB0FC93F92E741B99730083C57
:1013200015A82ABEDB0F49C0E4CB16C1DB0FC9BF2D
:10133000B0EEC07AF0EEE06AF4EEC76AF1EE10FAB1
:10134000B4BFF0EE475AF0EE665AF5EE405AF1EEB1
:1013500010FAF0EE407A44D0F4EEC76AF1EE10FADB
:101360008CBFB0EE475AB0EE665A85EE256A9FED07
:101370001E2A9FED1E3A9FED1E4ADFED1E4ADFED4D
:101380001E2ADFED1E3A9FED1E5AA6EE423AE6EE09
:10139000223AA6EE034AF7EE005AE6EE044AE6EEDB
:1013A000235AA6EE245A85EE250AF4EEC76AF1EE1A
:1013B00010FA48BF9FED137AF5EEC00A48BF37EE2A
:1013C000400AF1EE10FA48BF9FED0F7AF5EEC07AB1
:1013D00048BF37EE400AF1EE10FA48BFB1EE400ABE
:1013E00070479FED070AE0E739094E3DE3B59E3EA1
:1013F00088FA163E45FE7F3F99FB243F69A2163EC0
:10140000A7DFA834DB0FC93FDB0F49402DE9F04FC0
:10141000144689B08846217801320392002900F0F1
:101420001681002507461E46A94609E03846C047F2
:10143000039C01352178631C0393002900F08F8001
:101440002529F3D16078A31C3028CDE9033923D0B6
:10145000A0F13003DBB2092B4FF0000A26D96C282B
:101460002AD078287FD8572878D9A0F15803202B84
:1014700079D8DFE803F0BD7878787878787878786C
:101480007882AF787878787878787878AA78787869
:10149000789E788A7878BD00A078E31C0393A0F149
:1014A0003003DBB2092B4FF0010AD8D804AA03A9F4
:1014B00047F00EF96C28D4D1039C22780134782AA5
:1014C0000394B7D8572A40F28E80A2F15803202BFC
:1014D000B0D801A151F823F00F1601083514010806
:1014E00035140108351401083514010835140108B4
:1014F00035140108351401083514010835140108A4
:10150000351401087D1501082B1601083514010852
:101510003514010835140108351401083514010883
:101520003514010835140108351401083514010873
:10153000CD150108351401083514010835140108CA
:1015400035140108B5150108351401083B160108CA
:1015500035140108351401080F16010828B928466A
:1015600009B0BDE8F08F039C64E72528FBD1039CFC
:1015700025213846C04701355CE7039C56F8041B1B
:101580003846C9B2C047013554E70DF1140B56F87F
:10159000040B039C5B4600220A21FFF7EFF8049A34
:1015A000CDF800B0534641463846FFF77BF8054476
:1015B00040E7039C56F8043B0093049A00234146FD
:1015C0003846FFF76FF8054434E7039C56F8043BB0
:1015D0001D602FE70DF1140B56F8040B039C5946C0
:1015E000FFF714F9DBE7002AB9D0252AC0D021E79C
:1015F000A0F15802B2FA82F20DF1140B56F8040B66
:1016000052095B461021FFF7B9F8039CC7E7A2F126
:1016100058020DF1140BB2FA82F256F8040B52097B
:101620005B461021FFF7AAF8B9E70DF1140B56F845
:10163000040B5946FFF7EAF8B1E70DF1140B56F821
:10164000040B5B4600220A21FFF798F8A7E70D4636
:1016500085E7F8B5104C0746A06C0D461646A0B1BC
:101660000E49FFF72FFBA06C3946FFF72BFB0C4907
:10167000A06CFFF727FB0B49A06C33462A46FFF707
:10168000C5FE0949A06CFFF71DFB94F84C3013B15F
:10169000012384F84D30F8BD4888002065F4060821
:1016A000660E0708C10C010872F406080EB400B5F6
:1016B00084B005AB019053F8042B0649039301A8AD
:1016C000FFF7A4FE019B00221A7004B05DF804EB42
:1016D00003B0704729070108F7B5114E0746304699
:1016E000002300F84E3F0C460E4B0F49002F18BF49
:1016F000194615464EF078FE0C4F04EB45054E3664
:10170000AC4202D10A4803B0F0BD394634F8022B8E
:101710006846FFF7CBFF694630464EF065FEEFE7BF
:101720004888002076F406087FF4060888F4060846
:1017300096880020F7B50C4E0C4F002306F87F3F2B
:10174000044600EB4105AC4202D1094803B0F0BDAC
:10175000394634F8022B6846FFF7A8FF6946304641
:101760004EF042FEEFE700BF488800202DF7060844
:10177000C7880020F8B5084F4E1E054601F11F042A
:1017800016F8012F28463946FFF790FFA64205F1CB
:101790000205F5D1F8BD00BF8DF406080246531CC2
:1017A000084605D1034B1A681B790A600B71704714
:1017B00001497BE7CBF306082EF7060810B5013187
:1017C00014460CF093FB28B9054B1A681B7922606C
:1017D000237110BDC27903492046BDE8104065E77A
:1017E000CBF306082CF4060803685A1C0260197033
:1017F0000368090A5A1C02601970704710B4026825
:101800001346511C016013F8021B0360D31C54786B
:10181000036093781B0443EA0423141D0460D0780A
:101820005DF8044B0B4343EA00607047A0F13003BE
:10183000092B07D920F02000413819288CBF00203F
:101840000120704701207047303809288CBF0020E4
:1018500001207047413819288CBF002001207047B3
:10186000613819288CBF002001207047202805D03E
:10187000093804288CBF00200120704701207047E0
:10188000A0F14103192B98BF20307047A0F16103EC
:10189000192B98BF2038704702B310B584468418BE
:1018A00003E0981A15D1A44514D01CF8013BA3F10C
:1018B0004100192811F8010BA0F1410E98BF203307
:1018C000BEF1190F00F12002EBD91B1A04D1002838
:1018D000E9D110BD002010BD184610BD104670475C
:1018E00070B5044608460D464CF0F4FB064602E08F
:1018F00014F8013F43B1324629462046FFF7CCFF9A
:101900000028F5D1204670BD1C46204670BD00BFA2
:101910002DE9F043064686469EF800C0BCF1200F34
:101920007446ACF109050EF1010EF5D0042DF3D982
:10193000BCF12B0F64D0BCF12D0F26D10127102A4A
:1019400094F801C004F1010423D04FF0FF35B5FB3A
:10195000F2F502FB05FE6FEA0E0E5FFA8EFE904670
:10196000002014F801CBBCF1390F4CF02009ACF188
:10197000300C29D85FFA8CFC944528DAA842264618
:101980001ED81BD000FB08C0EBE7102A4FF0000761
:10199000DBD1BCF1300F0AD16078A0F14105192DDF
:1019A00098BF2030661C78280CBF023434466FF094
:1019B00070454FF00F0E4FF01008D1E7F445E1D914
:1019C0004FF0FF301F40CCE7B9F1600F0AD801B1EA
:1019D0000E6067B923B16FF00043984228BF1846E4
:1019E000BDE8F083A9F157095FFA89FCC4E723B188
:1019F000B0F1004F28BF4FF000404042BDE8F083F7
:101A000000279CE773B50E4610490546FEF792FE87
:101A100018B93070012002B070BD2C78602C8CBFDA
:101A2000613C413C082C0FD8013501230A2201A951
:101A30002846FFF76DFF019BAB4205D00F2803D866
:101A4000013440EA0410E4E70020E4E7CBF30608A1
:101A500001230A2200215BE770B50D461446FFF70B
:101A600098F90646A0B1FFF7F3FF40F63403984219
:101A7000A8BF1846B0F5617FB8BF4FF46170A0F5FC
:101A800061731922B3FBF2F32B70237801332370B7
:101A90003046FFF77EF90646A0B1FFF7D9FF40F6C2
:101AA00034039842A8BF1846B0F5617FB8BF4FF421
:101AB0006170A0F561731922B3FBF2F36B702378A8
:101AC00001332370304670BD10B402888378174C00
:101AD00002F0030101EB4101013B03EB8103A2F59D
:101AE000FA62C17834F813305DF8044B920840F282
:101AF000B55C0CFB02334A1E13440179427990F81D
:101B000006C0008903EB430301EBC301C1EB0111E4
:101B1000074B02EB8102C2EB0212634403EB820328
:101B200000214FF47A72C3FB02017047D8230608E4
:101B300080436D382DE9F04116461F46044639466C
:101B400030464FF47A7200234CF022FF3C4D3D4B5F
:101B5000054483FB05602844E917C1EB601183FB52
:101B600001030B44384EC817C0EB631086FB003CE2
:101B7000C317364EC3EBAC0386FB03764FEAE37E16
:101B8000CEEBE61EC1EB0116A5EB860CC0EB0015F3
:101B9000A1EB8501617103EB4301A0EBC10040F2B1
:101BA000B55101FB1E33B3F5896F84F806C020716F
:101BB0004FEA8E0633DA40F2DA218B4237DCB3F596
:101BC000B77FB4BF4FF0000E4FF0010E204F0EEB69
:101BD0004E0107EBC1017546C88A4FEA4E0808EB73
:101BE0000E0C07EBCC0C0CF1160C0B2101E03CF8B1
:101BF000020D984210DD0139F9D1F044012137F886
:101C00003800A170013306F5FA6E1B1A7544E370B3
:101C100022812580BDE8F0810131C9B2F1E70325B9
:101C20000B4F40F29650AE464FF00608D7E702251C
:101C3000074F40F22940AE464FF00408CFE700BFFF
:101C400080BC92C789888888ABAAAA2A73B06D160F
:101C5000D82306080C4B10B5D3E92A4354EA0302F3
:101C600009D1014640F201130020C1F80230887109
:101C70000880088110BD054A1268121943F100035B
:101C8000FFF758FF012010BD488800209819002058
:101C90002DE9F041044694421546084609D2B4FBAA
:101CA000F2F6154B05FB16441B5D00F8013BBDE841
:101CB000F081B4FBF2F69642B6FBF2F70CD20E4B73
:101CC00005FB176705FB1644DA5D00F8012B1B5D69
:101CD00000F8013BBDE8F081BA42B7FBF2F807D942
:101CE000054B05FB187813F8082000F8012BE7E7EF
:101CF0004046FFF7CDFFF3E77883060870B5884CC0
:101D0000B4F8DC34B4F8E024B4F8E414B4F8E6042D
:101D1000B3F57A7F88BF4FF47A7382B088BFA4F896
:101D2000DC34B4F8DE34B3F57A7F84BF4FF47A73D1
:101D3000A4F8DE34B4F8E234B2F57A7F84BF4FF40D
:101D40007A72A4F8E024B3F57A7F84BF0023A4F864
:101D5000E234B1F57A7F50D94FF47A718842A4F811
:101D6000E4145CD89A429CBF0023A4F8E03481427A
:101D70009CBF0023A4F8E434B4F8F434B4F8F2249B
:101D8000684D9A4284BF0023A4F8F234664B1B8846
:101D900003B36979654E0129B27848D9062A55D925
:101DA0003179002940F096809FED617A61490A7887
:101DB00007EE903A06EE902AF8EEE77AB8EEE66A79
:101DC000B379C6EE276A002B7CD1B4EEE67AF1EE49
:101DD00010FA49DC6A78032A1DD8574B03EB4213EB
:101DE0002A78C4F8FC34032A0ED8544BEA2102FBAB
:101DF0000133534A136002B070BDB0F57A7F84BFDF
:101E00000020A4F8E604ADE700224C4B2A704C4AAF
:101E1000136002B070BD0022474B6A70E0E70021FA
:101E20009A42A4F8E614A7D8A4F8E014A4E7B1797C
:101E30000029B3D0072A61D0B3F57A6FAED93D49F6
:101E400008780228B8BF02200870A7E73D4901EBD7
:101E5000820191ED187A31790029A7D0531F032B05
:101E6000B8D9002AB6D03BE027EE277AFCEEC77A35
:101E7000CDED017A9DF8043007EE903AF8EEE77A5E
:101E8000B4EEE77AF1EE10FAC4BF0133DBB29BB3D4
:101E9000102BA8BF1023DBB2934238BF13460B7040
:101EA00098E73279002A95D122499FED277A0A785E
:101EB00007EE903A06EE902AF8EEE77AB8EEE66A78
:101EC000C6EE276A37EE077AB4EEE67AF1EE10FA3C
:101ED00080DDC9E7053A032A7FF67CAF9FED147ACF
:101EE000B7EE000A80EE070A4DF046FD33888342C4
:101EF00028BF034633806DE70123CCE70622B3F504
:101F00007A6FB270CDD90B4930790A78022AB8BFFE
:101F100002220A7000287FF45DAF9FED0B7A46E73E
:101F200048880020002C002028130010EC220020FC
:101F30006F1203383C2D0020F8880020788900209B
:101F4000442D0020D823060817B7D1382DE9F04FCB
:101F50009D4B83B01B78A3F11702022A00AF00F259
:101F60009F829A4E9A4C04F2345994F808357B605B
:101F7000CB4604F5B1684FF0000AB14619E09BF971
:101F80000420142A2FD028464EF0BAFAAB031ED5EF
:101F9000012828D0082826DC16B18E4B1D4204D11A
:101FA000796828464AF01EFEE8B10BF10C0BD845C3
:101FB00013D0DBF8005015F00106E0D028464EF0B3
:101FC0009FFA0AF1010AAB035FFA8AFAE0D401280A
:101FD000E0DC0BF10C0BD845EBD10AF1FF32022A01
:101FE0004E4605D900E04E467B497C4844F0FAFE57
:101FF0000023022084F88C350DF04EF894F89035CB
:10200000774A022B156800F0ED82002800F0398332
:10201000DFF8E491734B94F8E9C5C7F804C003F501
:102020006A7B4FF47A7A4FF0000E4FF0640833F871
:10203000082CB2F57A7FB3F8462088BF23F808ACA5
:10204000B2F57A7F33F8062C88BFA3F846A0B2F524
:102050007A7F33F8042C88BF23F806AC33F8061CCB
:10206000B2F57A7F84BF002223F804EC9142B3F8E2
:102070005A10B3F85C2098BF23F806EC914293F80D
:102080006B2088BFA3F85AE0013A632A93F86C20CA
:1020900088BF83F86B800132D2B2092A88BF83F8E7
:1020A0006CE003F16501002213F8320011F801CF52
:1020B0000132844538BF81F800E0032AF4D17A6800
:1020C000012A18BF83F886E0EA339B45AFD1DFF8D9
:1020D0002CA19AF80230042B00F0B28243B9BAF86E
:1020E0000030B3F5F07F84BF4FF4F073AAF80030EE
:1020F000FFF704FE3C4894F8FC15FEF757FD94F8F2
:102100001B161030FEF752FDB4F82A26B4F8283614
:102110001343B4F82C2613431BB213B10123A4F8C4
:102120002E36324B2B40002B00F0B882E80700F12E
:102130007382690400F1D3812A0740F141822C4A5D
:10214000274B15401D60D9F800301340C9F8003006
:1021500015F4004300F01982002384F80F3584F849
:102160001F35E80440F11B8294F83B36DFF8848089
:10217000022B04BF012384F83B3608F1780B434659
:1021800002E006339B450CD01A780A2AF9D19978D7
:10219000DA78914202D35A79002AF2D00A2025F047
:1021A000D9F800234FF4806084F88C350CF074FF6C
:1021B000002800F05A820F4979600D46687958B3BB
:1021C000297831B343461EE0842C0020D82306082A
:1021D00048880020BC0202007C8D002000180708FF
:1021E000C431002082890020548E00200960000242
:1021F000FE9FFFFD888E00202C2C0020EC2200206A
:1022000006339B4508D01A788242F9D15A79002AC0
:10221000F6D0084625F09EF80635AB45CED19AF8A3
:1022200002807968B8F1080F00F0CF8194F8E935A1
:10223000D9F80000B24DA3F10103B3FA83F35B09AF
:1022400084F8B83694F8EA35A3F10103B3FA83F3BE
:102250005B0984F8BE3694F8D934032B84BF00237D
:1022600084F8D934A74BC0F3C03293F80EC084F879
:10227000BB262B68A44A134002402B60C9F80020FB
:10228000BCF1000F00F0CA81A04DAB88002B40F0DC
:10229000B9819F4A1368B3F5000F24BF0023136070
:1022A000936823F4007323F0020313B140F2022376
:1022B00093601379013B042B84BF01231371A8F1B0
:1022C0000508944BB8F1030F93F8009040F24A814F
:1022D0000025B9F1000F27D0DFF868827D603E60ED
:1022E00045464E46894606E0A8F10608A8EB0A03D3
:1022F0009E4240F2F680A84615F8010F0028F3D060
:102300000BF01CFE0028EFD083799B07ECD57D688D
:102310003E68494601223DB19AF8113053B99AF806
:102320000530012B00D02AB19AF8063013B10023F2
:102330008AF80630784BDA8802F00F00042803D8B8
:10234000C2F30312022A02D94FF42062DA801A89FA
:1023500002F00F00042803D8C2F30312022A02D9A4
:1023600040F601221A8194F8D10694F8DD2694F8FB
:10237000D036904205D9002284F8D12653B1A4F872
:10238000D42694F8DC269A4204D2002384F8D0366E
:10239000A4F8D43694F8C63794F8D226DFF8A8C14A
:1023A0009A4284BF002384F8D2360CF1800A634637
:1023B00013F8032D02EB4202324492F8549192F842
:1023C000558192F856E113F8015F9879DA784D4516
:1023D000A8BF4D464045A8BF40467245A8BF7246BB
:1023E00063451D709871DA70EDD103F1200CD4456E
:1023F000DDD1D4F82C25002A00F01781002501201A
:102400000B782B2B07D14B78043300FA03F31342DC
:102410001CBF9A43012506318B45F1D10DB1C4F89B
:102420002C253E4D6E4605F108082B4601E043453C
:102430005CD013F8012F072AF9D9002305F8013FD2
:102440000133082BFAD1B4F8E225B4F8E0359A420A
:10245000B54602D3324BC4F8E035324B324DFF2241
:1024600084F8F82703F1540013F9082C142A05D036
:1024700053F80C1C35EA010100F0DF800C33984260
:10248000F2D12A4A5379012B04D0022B04D1284BD4
:102490001B790BB9002353710C37BD46BDE8F08F93
:1024A000244A12F8331081B9DB001A44224E5278C4
:1024B000002A3FF457AD334493F87C30002B7FF46F
:1024C00051AD1E4A182313704CE502EBC301DB002B
:1024D00049680029E9D1194817210170E5E7184A30
:1024E0002EE67D683E684946002214E788B0E9463A
:1024F0002022FF2148464DF06FFF084A2BE000BF25
:10250000C4310020002C0020BCD755180C2D002011
:102510004C2D0020D01100109C300020FE22002005
:10252000AE014A01888D00200100020094220020A3
:102530009C220020101C0608D8230608842C0020AA
:10254000F6DFFFFDF3220020FD880020424549F818
:1025500023303FF478AF12F8013F59F823100131CE
:10256000F4D06AE700238AF804300125B9F1000F9E
:102570007FF4B2AE9AF81130002B7FF4DBAE9AF8FC
:102580000530012B7FF4D6AECEE694F80F25002A55
:102590003FF4E7ADE80484F81F353FF5E5AD2906C3
:1025A0007FF5E2AD424B1A78182A04D8414BD3404C
:1025B000DA073FF5D9ADDFF8108108F1780BF0E5C7
:1025C000AB047FF5C5AD3C4ABAE59AF80630002B5E
:1025D0003FF42CAE9AF81130012B04BF02238AF885
:1025E000113023E600283FF413AD90F904904FF02A
:1025F000FF0A01E080F808A048460CF03DFD0028E5
:10260000F8D105E5287879600BF098FC7968002806
:102610007FF43FAEA8803CE6284A91E52848034372
:1026200002432B60C9F800202EE62B20796024F0AD
:1026300091FED4F82C257968E0E684F8F82720E7A5
:10264000204B25F480551D60D9F8003023F48053C9
:10265000C9F80030BAF82030B3F57A7FBFF448AD3E
:102660004FF47A73AAF8203042E5164A136823F033
:1026700000631360D9F8003023F00063C9F800301C
:1026800099E5104BDFF8449025F080051D60D9F8DE
:10269000003023F08003C9F80030BBE4D9F80030E3
:1026A00043F0080345F00805C9F8003047E500BFCE
:1026B000842C002000410001F6BFFFFDF79FFFFDC5
:1026C00000040500C4310020888E00202C2C00203E
:1026D0002DE9F04FDFF8EC816F4ED8F80C30DFF8C1
:1026E000E89103F2DC534E4583B0C8F80C3080F01B
:1026F000CF8001230193694BDFF8D0B106F11C05AF
:102700009F1C664B5988002900F0AD807A185A4505
:1027100080F0A9803C4608E0118814460A4400294C
:1027200000F0A1805A4580F09E80052940F29B80F0
:1027300035F81C3C6188C3F30B039942ECD16379F3
:102740009B07E9D155F8141C238894F804A0009342
:10275000304644F047FB35F81C1CBAEB113F00F043
:1027600088800023019335F8181C55F8140C55F88F
:10277000044CC1F30B0144F08DFB1C364E45206028
:1027800005F11C05BDD3464A464B474F474C1268DE
:102790001A60FFF7DBFB3878454D7A78454EEA2121
:1027A00004F5987300FB01332B6004F1B00303EBD5
:1027B0004213C4F8FC3423F09FFF4FF0FF33286826
:1027C00073602DF087FD24F00DFE04F5C86304F559
:1027D000D76102E00633994255D01A78002AF9D120
:1027E0009D78D878854202D358790028F2D094F8A1
:1027F0003836327203EB830303EB83039B00642BB5
:10280000B4F83C26B8BF6423C8F80430642303FB43
:1028100002F2642AB8BF64220023C8E90223C8F880
:102820002020254AA8F82430C8E90433C8E9063333
:1028300088F82630214B93622EF0A4FDB4F8FC07F3
:1028400094F8FE1725F0DCFB39F032FA16F054F854
:102850001B4A01981268C8F80C20012388F825301B
:1028600003B0BDE8F08F55F8141C304644F0BAFAB6
:1028700077E7009BA11D9A1F304644F0E9FA002833
:102880007FF471AF6DE7FA7B003A18BF0122AEE723
:102890000123019377E700BF601507080040000897
:1028A000C43100202C2C0020002C0020488800205F
:1028B000442D0020A80500201C170010708E002059
:1028C000981900205C2D0020741E07080080000865
:1028D0000121194A10B5032800EB010403461170C9
:1028E000E4B218D9FF2825D0144A002341F202414E
:1028F00000E034B10233402B22F8021B04F1FF3414
:10290000F7D10F4A1344FF2183F80018BDE81040A7
:102910000E200CF00FBD0B480B49EA2203FB02000E
:102920000A4A0B7010602DF0D5FC25F043FF26F00D
:1029300025F8D9E70023E4E7581700104890002055
:102940004888002078890020002C0020442D002099
:10295000054BD3F84428012142F4001283F84118B2
:10296000C3F84428704700BF48880020F8B5164DCA
:102970006B78BE2B26D1022229464FF6FF70FDF759
:10298000EBFD124FAC1C22884AB1A618BE4219D2E8
:10299000052A17D92146FDF7DFFD3446F3E7214626
:1029A0000222FDF7D9FD0222A118FDF7D5FD06345C
:1029B000074B641BA3F8484841F60F53C31A58420B
:1029C0005841F8BD0020FCE70040000800800008E6
:1029D000488800202DE9F0410768C7F30D0406463A
:1029E00088460CB3D8F8005044F092FB092840F018
:1029F0008580444C236923F440732361236943F4A5
:102A000000732361236943F0010323613D6044F0B7
:102A10007FFB2369092823F0010323616ED133680A
:102A20000433336000206BE0374B384A93422AD39B
:102A300002F58042934225D302F5804293424BD364
:102A4000334A93424AD902F58032934248D902F57B
:102A50000032934246D902F50032934244D902F53E
:102A60000032934242D902F50032934240D902F536
:102A7000802293423ED9B3F1016F3DD348F0ACFDC3
:102A800048F07AFB082444F043FB092821D11D4D6E
:102A90002B6923F440732B612B6943F400732B6182
:102AA0002B6923F0F8032B612B691C4344F00204CB
:102AB0002C612B6943F480332B6144F029FB2B6993
:102AC00023F002032B612B69092823F0F8032B6103
:102AD00088D04FF0FF3013E01024D4E71824D2E759
:102AE0002024D0E72824CEE73024CCE73824CAE7D6
:102AF0004024C8E74824C6E75824C4E76FF0020022
:102B0000BDE8F081003C02400040000800400008A1
:102B1000FFFF00082DE9F041594E3378B12B8AB000
:102B200073D1FFF723FF80F00104E4B2554B564DFB
:102B3000B3F86331554FADF8043004F00104BD42E1
:102B400065D3002C00F099800023CDE90733099369
:102B50004F4B05969B1B06934E4B1A69002A04DACD
:102B60004D4A5A6002F188325A6001228DF82520C0
:102B7000F322DA6001A9022205A84FF000088DF8BF
:102B800024804AF01BFB022201A94FF6FF70FDF7DB
:102B9000E3FC3D4D0446BD4247D3022202A905A8ED
:102BA0000025ADF808504AF009FB022202A9204690
:102BB000FDF7D2FC40BAC043ADF80C00022205A8D4
:102BC00003A94AF0FBFA089878B107ABC0F10402F8
:102BD000294618444DF000FC9DF9240018B907A9B6
:102BE00005A8FFF7F7FE8DF824009DF8253023B1E6
:102BF000284A136943F0004313619DF92400B0FA99
:102C000080F040090AB0BDE8F08101248EE7A98870
:102C1000AB69A868D3F80080C1F30B0144F03AF91E
:102C20001C35804518BF012489E7AE888DF81180D6
:102C3000C6F30B06B31DADF80C302B88C3F30B02A3
:102C4000ADF80E201B0B062203A905A88DF8103045
:102C50004AF0B4FA062203A92046FDF77DFCA968D4
:102C60000446324605A84AF0A9FAA9682046324629
:102C7000FDF772FC1C3504468DE70120C2E700BF5A
:102C800000400008D823060860150708741E0708CE
:102C900000800008003C024023016745F8B5184D4C
:102CA000184E194FFFF752F9EB68012203F2DC537B
:102CB000EB6086F84A280324FFF72CFF58B13B78D5
:102CC000B12B08D1FFF752FE013C0AD058B9FFF7EB
:102CD00021FF0028F3D1013CEED148F07DFC48F003
:102CE0004BFA0028F9D0094A1168E9600122002353
:102CF00085F8252086F84A3886F84B38F8BD00BF9D
:102D00005C2D002048880020004000089819002011
:102D100008B50B490B4A01230B709373FFF7BEFFF5
:102D2000FFF7D6FC084B41F20241FF22A3F800183E
:102D300083F80228BDE808400E200CF0FBBA00BF63
:102D400058170010002C00204888002090F892307E
:102D5000DFED6B6A6B4A07EE903A90F8963005EE1D
:102D6000103A90F8943004EE903A90F8953005EED1
:102D7000903A90F89830F8EEE77AB8EEC55A04EE3B
:102D8000103A67EEA67A25EE265AF8EEE44AF8EEF7
:102D9000E55AB8EEC44A25EE275A64EEA64A65EE17
:102DA000A65A24EE264AF0B5B7EE007A90F8917054
:102DB00064EE854A65EEA75A24EE274A00F16F06B5
:102DC000014602F11A050024B0EE476AB0EE473A18
:102DD000137807EE903AF8EEE77A67EE857A67EEB9
:102DE000867AFDEEE77A17EE903AFA2BA8BFFA231F
:102DF00023EAE3730B72537807EE903AF8EEE77A22
:102E000067EEA47A67EE867AFDEEE77A17EE903ADF
:102E1000FA2BA8BFFA2323EAE3734B72937803EEED
:102E2000903AF8EEE33A63EEA57A67EE877AFDEE24
:102E3000E77A17EE903AFA2BA8BFFA2323EAE37356
:102E40008B72938807EE903AF8EEE77A67EE847A11
:102E500067EE867AFDEEE77A17EE903AB3F57A7F61
:102E6000A8BF4FF47A7323EAE3738B812B68D5ED07
:102E7000007A002BF8EEE77A3FDD90F8973002EE0B
:102E8000903AF8EEE22AB0EE436AA2EEE66A63EE0A
:102E9000863A83EEA76AA2EEA66A013465EEA77AA7
:102EA00067EE877A67EE867AFDEEE77A17EE903A5C
:102EB000FA2BA8BFFA2323EAE373BC4206F8013FCA
:102EC00000DDF0BD012C13D190F8933007EE103ADD
:102ED00090F89B3006EE103AB8EEC77AB8EEC66AA4
:102EE00027EE267A26EE266A0435083208316FE787
:102EF000B7EE007AB0EE476AF6E7B7EE006ACCE7C5
:102F00000AD7233C3E25060890F899306BB3B0F8F9
:102F100064308BB190F89A2002EB82036421C3EBFA
:102F20000313B3FBF1F3A0F86430962312FB03F311
:102F3000B3FBF1F3A0F8663043884BB190F89A30B8
:102F400003EB8303C3EB03136422B3FBF2F343806D
:102F5000B0F850304BB190F89A30962213FB02F340
:102F60006422B3FBF2F3A0F85030704790F82130A0
:102F70004BB3438B83B190F82230FA2213FB02F259
:102F800003EB8303B3F57A7FA8BF4FF47A73642110
:102F90008383B2FBF1F24283838843B190F82230FD
:102FA000FA2213FB02F36422B3FBF2F38380C3889B
:102FB0004BB190F8223003EB8303B3F57A7FA8BFBF
:102FC0004FF47A73C380704770B50B4C002504F53D
:102FD0006A7694F8913013B12046FFF7B7FE204689
:102FE000FFF792FF01353046FFF7C0FF042D04F1D3
:102FF000EA04EED170BD00BF7889002010B5064C00
:103000004FF48072002104F64C004DF0E5F90023E6
:10301000C4F84C3910BD00BF48880020034BD3F8DA
:10302000500908B109F046BC704700BF488800202D
:1030300008B50B4605490246D1F8500928B10449A4
:10304000FEF7E4F9BDE80840E8E708BD488800203D
:10305000C10C0108024B0146D3F85009FDF732BEFE
:10306000488800200048F5E7630907080CB4C30648
:1030700007B500D561B9049805A90191FFF7D8FFFC
:10308000FFF7F0FF012003B05DF804EB02B07047DA
:103090000020F8E70FB407B504A951F8040B01911B
:1030A000FFF7C6FFFFF7DEFF03B05DF804EB04B0E7
:1030B00070470349034801F521610EC9EAE700BFE3
:1030C0000070FF1F92F4060870B5134C134D144E98
:1030D000002294F8FB3403F0010302B170BD002B11
:1030E000FCD001212846FFF7D5FF75202EF0E6FB26
:1030F00001463046FFF7CEFF1A202EF0DFFB0146D7
:103100000848FFF7C7FF1B202EF0D8FB01460648F2
:10311000FFF7C0FF0122DCE748880020A6F406087C
:10312000B2F40608C5F40608D8F4060808B5FFF797
:1031300091FFBDE8084095E710B504460348FFF746
:1031400089FF2046BDE81040F0E700BFEBF4060819
:1031500008B5034610460AB9002008BDDB0601D5B4
:103160000029FAD0FFF7E8FFF6E72DE9F04F0A460D
:103170008DB000218346FFF7EBFF714CDFF8CC9157
:10318000039004F1800A0025A37A99F80060AB420D
:1031900000F3938010345445F5D140F2162043F0EB
:1031A0000BFED0E902450DF1180A002E4FF0150272
:1031B0004FF00001504604BF254634464DF00CF94F
:1031C00000272E78002E3ED06978059130460AF00F
:1031D0008DFE95F90290049009F10102534253418A
:1031E000002C00F0A98005990022A05CB04240F0BC
:1031F0009F80224492F90280C14540F09780527826
:103200008A4208BF012301220AF8072003F00103C4
:1032100083F00101039A05935846FFF799FF059B38
:10322000039044B1474A0499CDE900B23046424682
:10323000FDF734FE059B444A0499CDE900B23046BF
:103240004A46FDF72BFE0137152F05F10305B8D1CE
:1032500084B3DFF8F080DFF8F090564604F13F07C2
:1032600016F801ABBAF1000F21D12078F8B194F92A
:10327000023001331BD061780AF038FE039A05460C
:1032800001215846FFF764FF94F90220039053464A
:1032900020782946CDE900B8FDF700FE2078534696
:1032A000CDE900B94FF0FF322946FDF7F7FD0334B1
:1032B000BC42D5D10DB0BDE8F08FE08843F07CFD75
:1032C000D0E90231627A207A002E08BF194605FB48
:1032D000002208BF33468F562BB39E56039A0493A1
:1032E000B74214BF0121002158460CBF4FF001081E
:1032F0004FF00008FFF72CFF049B039043B1114BE4
:103300003246CDE900B3294643462046FDF782FD0B
:103310000D4B2946CDE900B33A4643462046FDF71A
:1033200079FD013530E74FF0FF36D7E700236AE734
:1033300003323F2A7FF459AF4FF0FF3868E700BFF0
:10334000B4050020C93401086D3001084888002008
:1033500010B508460749FDF7EDF9002815BF01240F
:10336000002405480548FFF7E7FE2046BDE8104069
:103370000BF0DFBEF0F40608F9F4060820F50608A5
:103380002DE9F04F07468BB040F216200C4643F073
:1033900013FD2246054600213846FFF7D9FE424B71
:1033A000D5E902451B78002B08BF254606464FF09D
:1033B00015024FF0000104A808BF1C464DF00CF8A0
:1033C00005F13F03039395F80090B9F1000F31D058
:1033D00095F801A0002C65D02246002311784945BC
:1033E00058D128336B4492F80180012203F8182C3D
:1033F000D045324614BF0121002138460CBF4FF0A2
:10340000010B4FF0000BFFF7A3FE064654B1B8F1D5
:10341000000F07D0254B00935A463B46414648468D
:10342000FDF782FD224B00935A463B4651464846E3
:10343000FDF77AFD039B03359D42C4D13CB3DFF811
:103440006C90DFF86CA0651C0DF11008403418F882
:10345000013BCBB915F8013CB3B116B13046FFF7CB
:103460006BFE297815F8010CCDF800903B46002240
:10347000FDF75AFD002215F8010CCDF800A03B46DF
:103480001146FDF751FD00260335A542DFD10BB0F3
:10349000BDE8F08F0133152B02F103029ED14FF0EE
:1034A0000008A5E7A046A3E748880020C934010822
:1034B0006D300108034B0146D3F8500908B109F0FB
:1034C000E5B97047488800200CB407B510F020001B
:1034D0000BD079B92320FFF7EDFF049805A90191DE
:1034E000FFF7A6FDFFF7BEFD012003B05DF804EB7A
:1034F00002B070470020F8E72DE9F04F914687B001
:103500000C461A4600218046FFF722FE4D4606462D
:103510000027B9F1000F66D02946062220464CF05C
:10352000DFFF0028324614BF0121002140460CBFB6
:103530004FF0010A4FF0000AFFF70AFE064628780E
:1035400015F0A2F98346F8B1687915F09DF9AB78CA
:10355000EA789BF805E095F801B04FF461714FF0FF
:10356000190C1CFB03131CFB0212297900B14079D2
:10357000CDE90410CDE90232CDE900EB1B4A3B4610
:1035800051464046FFF7A0FF207815F07DF98346AD
:10359000F8B1607915F078F9A378E2789BF805E046
:1035A00094F801B04FF461714FF0190C1CFB031338
:1035B0001CFB0212217900B14079CDE90410CDE95C
:1035C0000232CDE900EB094A3B4651464046FFF73F
:1035D0004DFD0137142F04F1060405F1060598D1BD
:1035E00007B0BDE8F08FCA46CEE700BF3CF506083D
:1035F0002DE9F04F904689B01A460C4600218146CD
:10360000FFF7A6FD3B4EDFF8F0B008F15403074684
:103610004546079394F904000BF02EFD00285DD079
:10362000B8F1000F63D029460C2220464CF058FF19
:1036300000283A4614BF0121002148460CBF4FF034
:10364000010A4FF0000AFFF783FD074695F90400D1
:1036500044F006FFEA7906EB82020346D2F88C2199
:1036600004922A7A06EB82025146D2F88C21039208
:10367000AA7906EB82024846D2F88C2102926A7936
:1036800006EB8202D2F88C2101922A6800925A46F7
:10369000FFF71AFF94F9040044F0E2FEE27906EB2A
:1036A00082020346D2F88C210492227A06EB82022F
:1036B0005146D2F88C210392A27906EB8202484649
:1036C000D2F88C210292627906EB8202D2F88C2128
:1036D0000192226800925A46FFF7C8FC079B0C35FE
:1036E000AB4204F10C0495D109B0BDE8F08FC2469D
:1036F000D0E700BFD823060855F506082DE9F04F9E
:1037000090468BB00C461A4600210746FFF720FD75
:103710004546099000264FF0190A4FF46179B8F137
:10372000000F4BD029460A2220464CF0D9FE002833
:10373000099A14BF0121002138460CBF4FF0010B3C
:103740004FF0000BFFF704FD2A890692EA880592E4
:103750002A790492EA780392AA7809901AFB0292D5
:1037600002926A781AFB029201922A7800923346FA
:10377000134A59463846FFF7A7FE22890692E28887
:10378000059222790492E2780392A2781AFB0292BF
:10379000029262781AFB0292019214F80A2B0092AC
:1037A0003346074A594638460136FFF75FFC1E2E5E
:1037B00005F10A05B3D10BB0BDE8F08FC346DCE7D5
:1037C00072F506082DE9F04F2DED088BDFF828A1E2
:1037D00095B0804691461E460C461546002794ED4E
:1037E000008AB5EE408AF1EE10FA7DD0D4ED019A50
:1037F00094ED029AD4ED038AB9F1000F49D0D5EDCA
:1038000000BA95ED01BAD5ED02AA95ED03AAB4EE82
:103810006B8AF1EE10FA6CD1F4EE4B9AF1EE10FADD
:1038200067D1B4EE6A9AF1EE10FA62D1F4EE4A8AE8
:10383000F1EE10FA0CBF0121002132468B464046C2
:1038400081F00101FFF784FCB0EE6B0A064611A877
:10385000FDF7C6F9B0EE4B0A07900EA8FDF7C0F9C8
:10386000B0EE6A0A06900BA8FDF7BAF9B0EE4A0A64
:10387000059008A8FDF7B4F90599069A079B0390EF
:1038800002910192009352463B4659464046FFF74B
:103890001BFEB0EE480A11A8FDF7A2F9B0EE690AC6
:1038A00083460EA8FDF79CF9B0EE490A06900BA8D6
:1038B000FDF796F9B0EE680A059008A8FDF790F9B3
:1038C000069B059A0390CDE900B302923B4652460F
:1038D000002140460137FFF7C9FB082F04F110040F
:1038E00005F110057FF47BAF15B0BDEC088BBDE88A
:1038F000F08F0021A1E700BF95F506082DE9F74FED
:1039000092460C461A4600218146FFF721FCDFF85B
:1039100070B0804656460025BAF1000F2ED03146D1
:10392000042220464CF0DCFD0028424614BF012151
:10393000002148460CBF01270027FFF709FC7388C8
:1039400001933AF82530009380462B465A46394673
:103950004846FFF7B9FD6388019334F8043B0093B0
:103960005A462B46394648460135FFF77FFB042D62
:1039700006F10406D0D103B0BDE8F08F5746EAE760
:10398000A9F506082DE9F04F89468FB017460021AA
:103990001A460646FFF7DCFBDFF874A00546002454
:1039A0000DF1240B59F82480CDF80880594602A85F
:1039B00044F004FD57B357F82430039398452A4642
:1039C00014BF0121002130460CBF4FF001084FF019
:1039D0000008FFF7BDFB04A9054603A844F0EEFC70
:1039E00004A900912346524641463046FFF76CFD3C
:1039F0002346CDF800B05246414630460134FFF729
:103A000035FB202CCED10FB0BDE8F08FB846EFE7E4
:103A1000BAF506082DE9F04F924685B00C461A46D5
:103A200000218146FFF794FBDFF874B080465546CD
:103A30000026BAF1000F31D02946042220464CF06E
:103A40004FFD0028424614BF0121002148460CBF0B
:103A500001270027FFF77CFBEB780293AB780193FB
:103A60002B880093804633465A4639464846FFF72E
:103A70002BFDE3780293A378019334F8043B009381
:103A80005A463346394648460136FFF7EFFA102EBC
:103A900005F10405CDD105B0BDE8F08F5746E8E744
:103AA000C4F506082DE9F04F85B0144602911A4678
:103AB00000210546FFF74CFB4FF0000806460623A1
:103AC00003FB08F7C0374FF00009029B13F807B05B
:103AD000002C7ED0E35D03939B45324614BF012149
:103AE000002128460CBF4FF0010A4FF0000AFFF7F3
:103AF0002FFB039B394ACDE90093064643465146C6
:103B00002846FFF7E1FCCDE9009B344A4346514685
:103B1000284609F10109FFF7A9FAB9F1060F07F1E3
:103B20000107D2D108F10108B8F1060FC7D1E42787
:103B3000029BA7F1E40913F807A0002C4BD014F85E
:103B400007B0DA45324614BF0121002128460CBFD8
:103B50004FF001084FF00008FFF7FAFACDE9009B9B
:103B600006461E4A062341462846FFF7ADFCCDE92E
:103B7000009A1A4A0623414628460137FFF776FA8B
:103B8000EF2FD5D1029B93F8EF70B4B194F8EF808A
:103B90004745324614BF0121002128460CBF0124AD
:103BA0000024FFF7D5FA002300930C4ACDF80480D7
:103BB000072321462846FFF787FC00230093074A86
:103BC0000197072321462846FFF750FA05B0BDE8C4
:103BD000F08FA24697E7A046C9E700BFD6F50608D2
:103BE0002DE9F04F0E46154689B01A4600210446CD
:103BF000FFF7AEFAB04681462F464FF0000B002D7E
:103C00007CD039460C2240464CF06AFC00284A46DB
:103C100014BF0121002120460CBF4FF0010A4FF0D4
:103C2000000AFFF795FA97F90B20049297F90A20FA
:103C30000392B7F908200292B7F906200192B7F96A
:103C4000042000928146384A5B4651462046FFF7E1
:103C50003BFC98F90B20049298F90A200392B8F9DA
:103C600008200292B8F906200192B8F904200092C7
:103C70005B462D4A514620460BF1010BFFF7F6F942
:103C8000BBF1080F08F10C0807F10C07B7D1DFF8FA
:103C90009C804FF0000B0C2303FB0BF985B300272E
:103CA00055F8090056F80920012303FA07FA4240A3
:103CB0003AEA020214BF1946002110EA0A0F07D09F
:103CC00000975B46424620460791FFF7FDFB0799A8
:103CD00056F809201AEA020F05D000975B464246C3
:103CE0002046FFF7C3F901370E2FD9D10BF1010B95
:103CF000BBF1080FCFD109B0BDE8F08FAA46A8E705
:103D00002F4656F80910012303FA07F20A4206D09B
:103D100000975B46424601212046FFF7A7F901378D
:103D20000E2FEED1E2E700BFEAF5060802F606081C
:103D30002DE9F04F89468DB0164600211A460746F8
:103D4000FFF706FADFF8DCA005460024C4EBC40345
:103D500009EB030259F8030091889279089040F327
:103D60000748ADF824108DF82620B8F1000F54D084
:103D7000002E55D0F218F058918893790A90ADF83A
:103D80002C1007220AA908A88DF82E304CF0A8FBA9
:103D900000282A4614BF0121002138460CBF4FF0ED
:103DA000010B4FF0000BFFF7D3F99DF82E3006936F
:103DB0009DF92D3005939DF92C3004939DF82B30FF
:103DC00003939DF92A3002939DF8293001939DF8C1
:103DD0002830009305462346524659463846FFF799
:103DE00073FB9DF8263006939DF9253005939DF9C8
:103DF000243004939DF82330CDE902839DF82130CF
:103E000001939DF820300093524623465946384688
:103E10000134FFF72BF9102C98D10DB0BDE8F08FCD
:103E2000B346DEE717F606082DE9F04F924689B053
:103E30000C461A4600210746FFF78AF9002607902C
:103E40005546B3464FF019094FF46178BAF1000FA7
:103E500028D02946062220464CF042FB0028079A2B
:103E600014BF0121002138460CBF4FF0010B4FF069
:103E7000000BFFF76DF96A79079019FB0282059232
:103E80002A7919FB02820492EA780392AA780292B4
:103E90006A7801922A7800923346124A5946384687
:103EA000FFF712FB627919FB02820592227919FB56
:103EB00002820492E2780392A278029262780192DE
:103EC00014F8062B00923346064A59463846013606
:103ED000FFF7CCF80A2E05F10605B7D109B0BDE809
:103EE000F08F00BF34F606082DE9F04F0F468BB077
:103EF000144600211A460646FFF72AF90546002C0B
:103F000000F0DD8022783B789A4218BF01210246FA
:103F100008BF002130460CBF4FF001084FF00008E9
:103F2000FFF716F923789E4A054641463046FFF7CB
:103F3000CBFA3B789A4A41463046FFF797F8002C77
:103F400000F0BF8062787B789A4218BF01212A4630
:103F500008BF002130460CBF4FF001084FF00008A9
:103F6000FFF7F6F863788F4A054641463046FFF77B
:103F7000ABFA7B788B4A41463046FFF777F807F17A
:103F8000C9030593A31C0693822307F1020A04F1D7
:103F9000CA0B07934FF000093B784B4500F3938021
:103FA000002C00F0F68097F8EA3094F8EA209A4264
:103FB00018BF01212A4608BF002130460CBF4FF030
:103FC00001084FF00008FFF7C3F894F8EA30764A8A
:103FD000054641463046FFF777FA97F8EA30724ACD
:103FE00041463046FFF742F8002C00F0D48004F13F
:103FF000EA0307F1EA0204F1FA014FF0010833F88D
:1040000002CF32F8020F844518BF4FF000089942E2
:10401000F5D188F001012A46C9B23046FFF798F879
:104020000821054604F1EC00FDF784FB5F4A0346D6
:1040300041463046FFF748FA97F8EA1007F1EC00DE
:10404000FDF778FB594A034641463046FFF70EF824
:10405000002C00F0A2804FF0FC094FF0010807EBA4
:10406000090104EB0900FCF765FB09F104090028CC
:1040700018BF4FF00008B9F58E7FF0D188F001012C
:104080002A46C9B23046FFF763F8082104F1FC0064
:10409000FCF792FE464A034641463046FFF714FAC3
:1040A00097F8EA1007F1FC00FCF786FE404A034649
:1040B000414630460BB0BDE8F04FFEF7D7BFA046F3
:1040C00037E7A04655E7079BFB180993002C5ED005
:1040D000079B0998E31819460893FCF72BFB059BEF
:1040E0005A789BF800309A42069A06BFB0FA80F8D8
:1040F0004FEA58184FF00008AAF10203023A0AF1F9
:104100000E0133F802CF32F8020F844518BF4FF08A
:1041100000088B42F5D188F001012A46C9B2304629
:10412000FFF716F86278069905469BF81800FDF728
:10413000D3FA02909BF800300193089B00931D4A2C
:1041400009F1010341463046FFF7BEF9059B7A7835
:10415000587E5146FDF7C0FA059A029012F8013FC9
:10416000019309F10109099B05920093114A4B46FD
:1041700041463046FEF77AFF069B10330693079BB5
:1041800009330AF1100A0BF1010B079304E7A0466B
:10419000DCE7A04621E7A0464EE7A04680E700BF47
:1041A0004DF606085FF606088DF60608A5F6060821
:1041B000BCF6060874F606082DE9F04F89B00F46E4
:1041C00090460021139A03930646FEF7C1FF87EA43
:1041D00008086FEA0803DFF8849006930446002578
:1041E00028460AF0E1FE129B184230D0069BDFF809
:1041F00070B0034014BF4FF0010A4FF0000A04935F
:1042000010EA07030CBF4A465A4628460593079210
:104210000AF0DCFE039B079A009080465146304628
:10422000FFF752F9049BB3FA83F12246490930465D
:10423000FEF78EFF059A039BCDF800800446002A06
:104240000CBF5A464A4651463046FEF70FFF01352D
:10425000172DC5D109B0BDE8F08F00BFD3F6060811
:10426000A3F506082DE9F04F0A4689B0002105465E
:10427000FEF76EFF384C059094F9000008F0FEFD43
:104280008146608842F098FD344BD0F808B01F7822
:1042900017B15F46D0F80CB0A379012B38BF0123CA
:1042A000069300262279637906FB02331BF803800C
:1042B000002F3BD0FB5C059A0793434514BF0121B7
:1042C000002128460CBF4FF0010A4FF0000AFEF70C
:1042D0003FFF079B0590013653B303F00F021B0904
:1042E0004033CDE9006302924B461D4A51462846B1
:1042F000FFF7EAF8B8F1000F24D008F00F034FEAF7
:104300001818029308F14003CDE90063144A4B46A4
:1043100051462846FEF7AAFE069BB342C2DC114B6B
:104320000834A342A8D109B0BDE8F08F3B46C2E7EC
:10433000002FDFD00C4A00964B4651462846FFF727
:10434000C3F8D7E76B06E7D4074A00964B465146B9
:104350002846FEF78BFEDFE7A425060848880020E4
:10436000DAF60608AC260608F0F606080FB407B51C
:1043700004A951F8040B0191FEF75AFE03B05DF851
:1043800004EB04B070472DE9F041037903F0E0023B
:10439000402A4DD009D83ABB03F00703052B1ED89D
:1043A000DFE803F0181D181D0910602A47D0802A85
:1043B00041D0BDE8F081D0F805102348BDE8F041B8
:1043C000FEF768BED0F8052051422048BDE8F04114
:1043D000FEF760BEB0F80720B0F80510F5E7B0F9B9
:1043E0000720B0F90510F0E74679194D194805EB9B
:1043F000C605FEF72FFE95F8D87200240123A742C8
:1044000003D8BDE8F041FEF72DBED5F8D46256F8CA
:1044100024204FEA84084AB113B90F48FEF71AFE68
:1044200056F808100D48FFF7A1FF00230134E6E716
:1044300041790B48C2E7827941790A48C6E7BDE86D
:10444000F0410948FEF726BE04F706081AF70608E9
:10445000D823060831F7060856F90608230E070880
:1044600042F7060853F706086AF7060830B52C48E5
:1044700085B0FEF7EFFD2B4B1B792BB92A4805B011
:10448000BDE83040FEF752BEFAF72AFD08B92748CA
:10449000F5E7FAF73DFD08B92548F0E7254B1B681D
:1044A000DB6998470028F7D0FAF712FD0268037D10
:1044B00081790446407C0290207C0190608A0090C3
:1044C00052081D48FFF752FFE51D0C3415F8010B8B
:1044D000FEF7F0FFAC42F9D1184C1948FEF7BAFDCF
:1044E0006378022B06D007D9032B10D11548FEF7AD
:1044F000B1FD0CE01448FAE704F580541348FEF7C8
:10450000A9FD94F8E437022B06D0032B06D005B0A2
:10451000BDE83040FEF7A6BD0D48E8E70D48E6E7E8
:1045200082F706089C2200208CF706089BF70608F5
:10453000A9F70608F81F0020B8F70608545900200C
:10454000E6F70608ECF70608F2F70608FFF7060894
:1045500005F806081EF806082DE9F04FBC4BBD49CA
:104560001A68BD4BB2FBF3F297B00746BB48FFF7A2
:10457000FDFEBB4BDFF8B4E30FCBDEF808C00AAD9D
:104580001CF0080F18BFDEF8044085E80F00B54B9B
:1045900005934FEA9C08B44B069318BFC4F38054AC
:1045A00016AB18F0020F18BF03EB8404CCF381069E
:1045B00003EB860618BF54F8442CAC4C08BFAC4A39
:1045C00056F8301CAB48AC4DDFF86483FFF7CEFEE5
:1045D000B4F854294FF47A73B2FBF3F103FB1122C0
:1045E0000A20B4F9563992B2B2FBF0F2A348FEF7B2
:1045F00051FDA34AA349A448FFF7B8FEFEF732FDD8
:10460000A24BA34A997BA34BA34805EB8101D31A84
:10461000D1F8C414B4F84828FEF73CFDFEF722FD9B
:104620009E48FEF717FD94F858199D48FFF79EFE27
:104630009C48FEF70FFD9C4B94F859191A889B482B
:1046400092B2FFF793FEFEF70DFD99499948FFF7E7
:104650008DFE4FF000094E46DFF8D8A294F8F734EB
:1046600003F00103B9F1000F00F06A81002E40F061
:104670009C819148FEF75AFDDFF8BC82D4F860991E
:10468000DFF8B8A2012608F1180B0123B34013EAA2
:10469000090F15D01AF8062058F826305BF82610B6
:1046A00053F822208548FFF761FE012E06D1844B86
:1046B00093F8211011B18348FFF758FEFEF7D2FCA2
:1046C0000136062EE1D18048FEF7C4FC7F4B1B6803
:1046D0001B0640F19E8194F88039032B8CBF7C48E7
:1046E0007C48FEF7B7FC94F89035022B40F06081CF
:1046F0007948FEF7AFFC94F88039042B00F28081F2
:104700007648FEF7A7FC94F89039002B00F07F81E3
:1047100005EBC303D3F860157148FFF727FEFEF7DA
:10472000A1FC704B70481E68704B1B7805EB83032F
:10473000D3F89415FFF71AFE26B1327A717A6C48D5
:10474000FFF714FEFEF78EFC49493846FFF78EFE50
:10475000FEF788FC67496848FFF708FE6749684824
:10476000FFF704FEFEF77EFCFEF77CFC654B664817
:1047700019684FF47A73B1FBF3F1FFF7F7FD07A85F
:10478000FDF768FA38B107A90EA849F055FA5F4855
:104790000EA9FFF7EBFDFEF765FCD4F81C8AB8F113
:1047A000000F00F03A8107EE908ADFED596AB8EE0B
:1047B000E77AC6EE877AFDEEE77A17EE903A554F24
:1047C00097F81C0130B1544A039392ED250A4BF03F
:1047D000D3F8039BD4F89C695EB107EE906ADFEDD5
:1047E0004C6AF8EEE77A86EEA77AFDEEC77A17EE06
:1047F000906A334AB2F870106429A8BF6421CDE9E9
:10480000000642464548464EFEF744FCB7F82021D4
:1048100044486423B2FBF3F103FB112297F83131D2
:1048200005EB830592B2D5F8A835009397F830319F
:10483000FEF730FC3C48FEF70DFCD4F84448012557
:10484000002C40F0EC80FEF70DFC17B0BDE8F08FB7
:104850008C1A002038F8060840420F0042F806087B
:104860008C28060854F8060859F8060848880020DD
:10487000650907085EF80608D823060866F80608E2
:10488000F0FF00100008000088F80608002C002047
:1048900000800008004000089AF80608B1F80608F1
:1048A000C3F80608CBF80608D0230020CDF8060888
:1048B000E1F80608E6F8060805F906083B060708C9
:1048C000581700100AF906080EF906082C2C0020CB
:1048D00014F9060820F9060830F90608850F0708BC
:1048E00069F906081431002085F906081031002006
:1048F0008EF9060898F90608B9F90608C7F90608F6
:10490000BA08070898190020D1F90608EBF906083B
:104910000024744940990020A8050020FEF90608EB
:1049200075F9060844FA060869FA060800380240D4
:104930002813001056F9060804290608340600203A
:10494000002B3FF493AE16B15046FEF783FB3B4875
:104950000121FFF70BFD94F85C39394805EB83031F
:10496000D3F8CC14FFF702FD98F8CE33DA0702D55E
:104970003448FFF7FBFC98F81831032B09D0324874
:10498000FFF7F4FC98F81831012B02D12F48FFF7FC
:10499000EDFCD8F84C305B7B0126B342B1467FF684
:1049A0005DAE2B48FFF7E2FC56E6FEF75BFB63E6E5
:1049B00002200AF091FB064608B9264899E690F9CC
:1049C000040043F04DFD804637F05CF905EB8000B4
:1049D0004146D0F88C212048FFF7C8FC94F8933565
:1049E000012B04D11D48FEF735FB1D4881E6B37944
:1049F0001C4805EB8303D3F88C11FFF7B7FCF4E7F1
:104A000094F892350BB918487BE6184879E61849AE
:104A100082E61848FEF71EFB81E64346CFE694FA8D
:104A2000A4F0B0FA80F005FA00F024EA00040AF0DD
:104A3000A1FA01463046FFF799FC01E7EBF80608BA
:104A400075F906085BFE0608F0F80608F8F806088F
:104A5000FDF8060836F9060840F9060850F9060878
:104A600055F906086EF5060859F9060890F7060884
:104A700030F8060879F906082DE9F04FDFF8708163
:104A800098F8033099B0002B00F094804F48504EB6
:104A9000DFF860B1DFF86091DFF860A1FEF746FB58
:104AA00000252F460BA9E8B214F0AEF99DF834307A
:104AB000002B53D0139C54B107EE904A9FED450A4A
:104AC000F8EE677A80EE270A4AF056FF04460B9A02
:104AD00029465846FFF74AFC109A002A6CD002FB80
:104AE00004F04FF47A73B0FBF3F30993DDF848C098
:104AF000BCF1000F62D00CFB04F142F21073B1FB69
:104B0000F3F198F80330082D18BF7F18002B57D009
:104B10001798079015980690169805900A231198F3
:104B20004FF47A7EB0FBFEFE0998CDF810E0B1FBA1
:104B3000F3FE03FB1E11CDE902E10999B1FBF3F18C
:104B400003FB1100CDE90010BCFBF3F321465046F6
:104B5000FEF7A0FA0023C6E90D33B3620135222D1A
:104B600006F140069ED198F8033003B31A4C1B4857
:104B7000D4E94D124FF47A73D208B1FBF3F3D4F8B1
:104B80003C11FEF787FA0A22154897FBF2F102FB67
:104B90001172FEF77FFA134B1B78432B04D1D4E933
:104BA00050211148FEF776FA0023C4F83C3119B0C1
:104BB000BDE8F08F0D486AE7099297E76146A0E7E4
:104BC00021464846FEF766FAC4E700BF7FFA0608AA
:104BD000DC9100208096184B4099002026FB0608A7
:104BE00046FB0608772200206AFB0608DDFA060865
:104BF000002C0020E7FA060809FE0608F6FA060867
:104C000010B586B0104B0493104B0393104B0293D6
:104C1000104B0193104B1149114A00930446114B5C
:104C20001148FFF7A3FBFEF71DFA10491048FEF7E5
:104C300031FA3CB10F4A1049104806B0BDE81040A7
:104C4000FEF728BA06B010BDD4FB0608D9FB06084B
:104C5000E3FB0608ECFB0608C7F906089EFB0608FE
:104C600094FB0608072C0020A9FB0608F8FB0608A1
:104C700000FC060811FC060821FC060826FC0608B4
:104C80000120BDE770B52348FEF7E4F9224B93F805
:104C90001C31002B38D0214B93ED250A4AF06CFED5
:104CA00001461F48FEF7F6F91E4C1F48FEF7D2F9E1
:104CB0001E4B94F821051E4A00280CBF10461846CA
:104CC000FEF734FA94F8213513B31A4C1A48B4F8A5
:104CD00006111A4E1A4DFFF749FB94F804010028FB
:104CE0000CBF30462846FEF721FAB4F808111548E3
:104CF000FFF73CFB94F8050100280CBF304628461E
:104D0000BDE87040FEF712BA0F48FEF70FFACBE786
:104D100070BD00BF63FC060840990020A805002074
:104D20007DFC0608488800208CFC06087FF70608F2
:104D300061140708581700109DFC06085CFC060863
:104D400053FC0608C4FC060882FC060838B50B4D67
:104D500005EBC0050C4695F9CC0108F08FF801462B
:104D60000748FFF703FB95F8D23133B1611C0548C2
:104D7000BDE83840C9B2FFF7F9BA38BDD8230608F4
:104D8000230E07082DF706082DE9F04F6B4B1B7813
:104D900087B0002B00F0CB80694D6A48A968FEF708
:104DA00079F969686848FEF775F9684B6848D3E98E
:104DB0000031C91A674B1A68B1FBF2F2FEF76AF9C3
:104DC000FEF750F96448FEF7B1F96448FEF7AEF912
:104DD0004FF00008624B1B785FFA88F4A34222D898
:104DE000FEF740F95F4D604E002455F8041F304631
:104DF0000134FFF7BBFA162CF7D1FEF733F95B4D00
:104E0000594E01242B4669681B683046C91A013483
:104E1000FFF7ACFA162C05F10405F3D107B0BDE895
:104E2000F04FFEF71FB9524B142603EB840306FB29
:104E3000045693ED450AB6F80E904AF09DFD96F89B
:104E40001EA01AF0010F0CBF2D2252221AF0020FE1
:104E50000CBF2D2354231AF0040F0CBF4FF02D0C60
:104E60004FF0560C1AF0080F0CBF4FF02D0E4FF0FC
:104E7000430E81B21AF0800F4FF03C0BB1FBFBF1F7
:104E800005914FF064010CBF4FF02D0A4FF0530A0B
:104E900080B201FB09F1671CCDE902A10490CDE9C4
:104EA00000CE34483946FFF761FAB37FDB073AD5C5
:104EB0005C23314A6343D118D05891ED010A70B197
:104EC000DFED2E7AB8EE400A20EE270A07EE900AB0
:104ED000F8EE677A80EE270A4AF04EFD00B26422AF
:104EE00090FBF2F102FB11022548FFF73FFA142173
:104EF00001FB075701FB0454F988628A0491218B56
:104F00000391E18A0291A18B0191A18A009102F0A3
:104F1000030319214B431B48218A9208FEF7BAF874
:104F200008F1010856E71848FEF794F8DFE717483C
:104F300007B0BDE8F04FFEF7F9B800BF040000105D
:104F4000EC0D0010E4FC0608F4FC0608000B001051
:104F50000BFD0608A019002038FD060894FD060880
:104F6000D0110010940E001044FE0608980E001098
:104F700058170010F0FD06080C0B001000401C46EE
:104F80000DFE060822FE060819FE060848FE060861
:104F90000EB403B503AA52F8041B0192FCF759FBA7
:104FA000064BD3F850291AB90549986CFBF78AFECD
:104FB00002B05DF804EB03B0704700BF48880020E2
:104FC000630907082DE9F04798460B7903F0E005DF
:104FD000402D81460F46164632D1644DDFF8A88138
:104FE000DFF8B091002416E03B7903F00703013BA2
:104FF000042B04D8DFE803F014171A1D2100315DDB
:105000005A48FFF7B3F97B79013BA34202DD4846DA
:10501000FEF720F801347B79A342E5DCBDE8F08798
:1050200031572846EDE736F81410FAE736F9141030
:10503000F7E756F824104046E3E756F82410F0E767
:1050400003F00703052B57D8DFE803F0031F2729D8
:105050002C3E3478602D55D02CD8002D75D1B7F862
:105060000550B7F8076041482146FFF77FF9AC4289
:1050700039DBB44237DCB8F1000FCFD032462946D5
:105080003B48BDE8F047FFF771B996F90040602D45
:1050900038D00FD8002D58D151E03488DAE7B6F96E
:1050A0000040F4E7D6F800A0202D54464DD034D966
:1050B000602D27D0802DB1D132782E4B2E48002A7A
:1050C00014BF3146194635E0202D34683DD0EFD865
:1050D00021462648FFF74AF9D7F80510A14202DB1E
:1050E0004B42A34221DDFDF7BDFF3A682349234629
:1050F0004846BDE8F0474BE7202D25D01ED9602D4E
:10510000D8D100247B7944FA03F3DB07BDE8F047EC
:105110004CBF1B481B48FFF729B951461A48FFF7F7
:1051200025F9D7F805108A45DDD8B8F1000F3FF40E
:1051300075AF1648BDE8F047FFF718B90024B7F976
:105140000550B7F907608EE700247A79104B03EB1E
:10515000C20393F8D822A242C5DDD3F8D43253F863
:105160002400BDE8F047FDF775BF00BF2EF7060825
:105170002DF6060815100708230E07086AFE060814
:105180007FF706086114070817F7060864FE06088B
:10519000D8230608CBF806082DE9F04F164685B04F
:1051A000CDE901011A4600213046FDF7D1FF314C0F
:1051B000009006F010034FF00009A2460393FDF79C
:1051C0002DFF2379029A03F01803934203D0002A9B
:1051D00044D1182B42D14FF00D0B0BFB09A3B3F8B0
:1051E000090041F0E9FD80462046FBF775FCD8E94F
:1051F00002210746024401442046FBF705FC80F0EB
:105200000101009A0546C9B23046FDF7A1FF039B94
:10521000009003B115BB0BFB09FBB3065AF80BB0AA
:105220000ED56DB914485946FFF7A0F8D8F80820F4
:1052300001982B463A442146FFF7C4FEFDF712FFC2
:105240000E485946FFF792F8D8F80C200198002331
:105250003A442146FFF7B6FEFDF704FF09F10109C4
:1052600040F26A23994504F10D04A8D105B0BDE8C8
:10527000F08F00BFE432060884FE060885FE0608AB
:1052800070B50546084616460C46FBF72BFD33461F
:10529000024621462846BDE8704093E60EB403B5A9
:1052A00003AA52F8041B0192FCF7D3F9044B0549F9
:1052B000986CFBF707FD02B05DF804EB03B0704794
:1052C00048880020630907080049E7E78FFE0608C1
:1052D00038B50C46054615492046FBF72BFA30B980
:1052E000FDF772FE1248BDE83840FDF71FBF1149B7
:1052F0002046FBF71FFAA0B90F4B83F8C10183F8D2
:10530000C90183F8AB0283F8B30283F8950383F8ED
:105310009D0383F87F0483F8870483F8F904074822
:10532000E1E72846BDE83840CEE700BF9EFE06080C
:10533000A4FE0608BFFE060848880020C7FE06082F
:105340000049ABE7E3FE06082DE9FF47074608469C
:105350000D4648F0BFFE082845D105F1FF3801AEE3
:10536000073531464246B14612F8010FFCF78EFA76
:10537000AA4201F8010BF7D10023DFF87CA08DF8D9
:105380000C30A84517D11B4948462BF053FF19484C
:105390001949082310F8012B11F8014B10326A4407
:1053A000013B02F80C4CF5D114488DF80C3001A9E2
:1053B000FDF770FE14E018F8010FFCF767FA06F825
:1053C000010B0446014650464BF01DF828B121461A
:1053D00030464BF018F80028D3D03846FFF774FF5A
:1053E00004B0BDE8F0870028D1D0384604B0BDE84D
:1053F000F047A5E7488D002098920608FAFE0608B7
:1054000007B5009313460A460249FFF747FF03B06A
:105410005DF804FB01FF06082DE9F04FDFF8A482D8
:105420008BB006460D46284648F054FE034638B970
:105430009649024601200BB0BDE8F04FFEF778BC5C
:10544000934905222846FCF727FA0446C8B9914D2E
:105450000146702205F5A4704AF0BEFFC5F8B841B8
:10546000C5F8C441C5F8D041C5F8DC41C5F8E841EC
:10547000C5F8F441C5F80042C5F80C420BB0BDE8D0
:10548000F08F042241462846FCF706FA044628BB62
:105490002846FBF77EFC81460028EFD048F01AFE34
:1054A000DFF824B282465BF8047B37B97A492A4692
:1054B00030460BB0BDE8F04FF0E65246394648465C
:1054C000FCF7EAF940B920462BF02EF87348744DEA
:1054D0003946FDF7DFFDA6E70134E4E7714907220D
:1054E0002846FCF7D9F9074600287AD1202128461A
:1054F0004AF089FF044670BB6B486C4DFEF736FFDF
:10550000214628460134FEF731FF0E2CF8D1FDF775
:10551000A9FDDFF8B891664FDFF8B4810025294670
:105520004846FEF723FF0C26DFF8A8A16E430024AF
:10553000F25960480123A34013420CBF4146514633
:105540000134FEF713FF0E2CF2D10135FDF78AFD71
:10555000082DE4D192E75849574D01AA4AF01FFFA0
:1055600002AC002848D0022F11D1029A072A07D88E
:10557000039C0D2C04D80378722B13D06E2B25D0EE
:105580004E49082300223046FFF73AFF76E7FCF742
:105590005FFA01AA44F8040B2946002001374AF0BB
:1055A000FEFEDEE73B490C2303FB02110123D1F889
:1055B000B811A3400B4337490C2000FB02123949B4
:1055C000C2F8B8313046FFF727FF57E7314B0C20C0
:1055D00000FB02330121D3F8B831A14023EA0103D3
:1055E000E9E728463449344F01AA4AF0D8FE02AD13
:1055F000002480B1082C03D13046FFF7A1FE3DE71F
:10560000FCF726FA01AA45F8040B394600200134BC
:105610004AF0C5FEEDE7082CEED1029B0F2B30D8E7
:10562000DDF80CE0BEF1070F2BD8DDF810C0BCF19F
:105630000D0F26D8059F07F16402C82A21D8069DC0
:10564000FF2D1ED8079864281BD80899642918D8FC
:10565000884216DA099C032C13D8C3EBC3020D4B06
:10566000134483F84D1183F848E10D4983F849C18B
:1056700083F84A7183F84B5183F84C0183F84E410B
:10568000A0E70F493046FFF709FEF7E6889A0020A9
:105690001AFF06084099002025FF060836FF060875
:1056A0006509070840FF0608240E070848FF06089A
:1056B000F89A00204DFF060851FF060853FF060820
:1056C00059FF060820FF0608942906082EF7060849
:1056D000FC0D070815F606082DE9F04F8FB00446BB
:1056E00002AA0846B1494AF05AFE054640B90346A7
:1056F0000246AF494120FEF7F7FB0FB0BDE8F08F3F
:10570000AC49FBF717F8064628BBA84902AA4AF09D
:1057100046FEFCF79DF90828054606D9A649082348
:1057200032462046FFF76CFEE7E7A44C94F8DC36DF
:1057300083420CDC84F8DC56DFE73146384635F02E
:105740007BFC013694F8DC36B342F6DCF2E7064621
:1057500004F2DC67F6E79A492846FAF7EBFF0646BB
:10576000E0B9924902AA4AF01AFEFCF771F908283A
:10577000054603D9934908233246D2E78F4C94F863
:10578000DD36834202DC84F8DD56B6E73046294632
:10579000013642F037FD082EF8D1F4E78A49284651
:1057A000FAF7C8FF064600BB804902AA4AF0F7FD97
:1057B0000028A2D0FCF74CF90828054603D98349F4
:1057C00008233246ADE77D4C94F8C637834209DDA5
:1057D000014604F2DC6035F073FC294604F2DC601B
:1057E00035F07CFC84F8C65787E779492846FAF7F4
:1057F000A1FF064618BB714BDFF8B09193F8C6774E
:1058000006AD0146102228464AF0E6FDA846BE42F3
:1058100002AA80F20A81494600204AF0C0FD10B970
:105820006C493A460AE1FCF713F9013628F8020BF5
:10583000EDE795E80F00684C84E80F005DE76749E5
:105840002846FAF777FF0646C0BB5C4BDFF85C9151
:1058500093F8C67706ADBE4202AA80F2F3804946AD
:1058600000204AF09CFD014610B95D493A46E5E04A
:10587000032228464AF0FFFDAA464FF000082846BA
:1058800048F028FC404502D801360435E3E79AF891
:105890000000FBF7FBFF08F101080AF8010BEEE737
:1058A000504DB6000446B4423FF427AF06AB191979
:1058B0002819032235F0AAFB0434F4E74A492846A4
:1058C000FAF738FF0746002840F0AC80DFF8EC809C
:1058D000364998F8DC6602AA4AF061FD00283FF4D8
:1058E0000CAFFCF7B5F8451E01D4AE4203DC3F49CE
:1058F0003346012215E72D4902AA00204AF04FFD48
:10590000014600283FF4F9AE0026082203A88DF8CE
:1059100014604AF0B0FD0DF10C0903A848F0DAFB61
:10592000B0421BD8214902AA00204AF038FD0028C5
:105930003FF4E3AE037898F8DDA601930026B14664
:1059400056451A4902AA4FF0000080F285804AF0BD
:1059500026FD834650B9264952466FE099F800006B
:10596000FBF794FF013609F8010BD6E7A6B99BF8BF
:105970000030303B092B0FD91E49FAF7DBFE38B156
:105980001D495846FAF7D6FE70B11C495A4655E0F3
:105990004FF001094FF0FF365846FCF759F8002840
:1059A00030DA17495A4649E0B146F3E751FF060895
:1059B000248F00206FFF060875FF06084888002026
:1059C00080FF060889FF060897FF0608A3FF060860
:1059D000B5FF0608A400070810900020DFFF0608A6
:1059E000C400070820900020090007080E000708DF
:1059F000E400070877F406081A00070821000708E2
:105A0000560007080EAB03EB4603013623F8200CC3
:105A100096E72049524611E033F8022B24F8022F72
:105A2000013730E01C492A4608E01C4900204AF0B2
:105A3000B6FC00283FF4FDAE19493A462046FFF770
:105A40002DFC5AE6154900204AF0A9FC00283FF435
:105A500027AF14493A46F1E74AF0A1FC0028D8D113
:105A6000114C05EBC50082302044082203A935F013
:105A7000CDFA0198FBF70AFF08EB050304EB0514C8
:105A800083F8A60706ABBE42C6DC454485F8BE9740
:105A900033E600BF6B0007088E00070851FF0608B9
:105AA000C1FF0608EBFF0608248F00202DE9F04116
:105AB000144B1B6888B00446F3B11A6804A9D56A70
:105AC00018466A46A847064688B1DFF8448004AC09
:105AD0006D46002735F8022B34F8021B404601378B
:105AE000FDF7D8FABE42F5DC08B0BDE8F081064902
:105AF0002046FFF7D3FBF7E7044908B0BDE8F041C3
:105B0000FFF7CCBB942D0020230107083B010708B9
:105B10000901070870B5054608460C4648F0DAFA50
:105B2000024670B10F2804D1094821464AF091FC81
:105B300038B12846064B074A0749BDE87040FFF7D1
:105B4000ADBBBDE8704002490448FDF7A3BA00BFF1
:105B500011FC0608420107084D01070877010708F4
:105B600070B5054608460C4648F0B4FA024670B1D6
:105B7000042804D1094821464AF06BFC38B1284674
:105B8000064B074A0749BDE87040FFF787BBBDE8F1
:105B9000704002490448FDF77DBA00BF21FC0608A9
:105BA000850107084D010708950107082DE9F04315
:105BB00007469BB008460C4648F08CFA2022064661
:105BC000002101A84AF008FC36B3402E08D03B491A
:105BD0004023324638461BB0BDE8F043FFF75EBBBA
:105BE00001AD04F140084FF0000902222146684649
:105BF0004AF041FC0023102209A968468DF8029062
:105C0000FBF786FE099B0DF10202934223D1023479
:105C1000A04505F8010BE8D109AC4122002120463E
:105C20004AF0DAFB264D002E3BD095F81862D6B12B
:105C3000202205F2192101A84AF052FC98B105F280
:105C400019212046FBF796FD1E4A1F492346384678
:105C5000FFF724FB04E01A781C493846FFF71EFBC7
:105C60001BB0BDE8F0831A4B1B78D3B9CEB9194EDF
:105C700001AB1A4603CAA24230607160134606F1B6
:105C80000806F6D101232046124985F83932FBF780
:105C900071FD1148FDF750FA10482146FDF7FAF959
:105CA000DEE795F839321BB995F81832002BF3D09E
:105CB00008492046FBF75EFDEEE700BFA801070894
:105CC00040990020E60107084D010708CA010708AE
:105CD00048880020599B0020F0010708FF010708B1
:105CE0002DE9F74F834608460C4648F0F3F9DFF8F4
:105CF00018810646D8F8007028B10246334920467C
:105D0000FBF7CAFD80B93946314842F02DFB3149D5
:105D1000314821EA070142F027FB3049304803B0FF
:105D2000BDE8F04F42F020BB23782D2B2D4B03BF55
:105D3000013406F1FF364FF0010A4FF0000A4FF030
:105D400000094FF0FF3553F8041B51B1324620468D
:105D50000193FBF7A1FD019B00280ABF4D460021DE
:105D6000012109F1010991B9B9F11D0FEBD11E49CA
:105D70002246584603B0BDE8F04FFFF78FBA3B43C9
:105D8000C8F8003019491A4B12E01A4913E0114AB9
:105D90000123AB401A40002AF7D007EA0302BAF108
:105DA000000FECD027EA0303C8F800301249134B68
:105DB000002A18BF1946124B124803EB8503D3F88B
:105DC0002C2603B0BDE8F04FFDF764B9E2FA0608EF
:105DD00037020708BCD75518410207084328AAE72D
:105DE0004D020708042A060825FF06082F020708A7
:105DF000280207080C020708180207081F020708F4
:105E0000D8230608A3F50608C43100202DE9F74F72
:105E1000019008460E461746984648F05BF904463E
:105E2000E8B93F483F4DFEF7A1FA204609F0BCF81B
:105E30003B68184206D0204609F0C8F801462846BB
:105E4000FEF794FA0134172CEFD13B6813B93648AA
:105E5000FDF700F903B0BDE8F04FFDF703B90246C6
:105E600032493046FBF718FD0546A8B93048FDF722
:105E7000F1F82C462F4D204609F096F810EA080F4D
:105E800006D0204609F0A2F801462846FEF76EFA31
:105E90000134182CEFD1DDE733782D2B03BF013609
:105EA00004F1FF34012500254FF0000948F4000BF0
:105EB000484609F08BF82246824601463046FBF7F9
:105EC000EBFC00BB484609F06FF81BEA000F1AD044
:105ED0008DB1B9F1170F1CBF3B6840EA03081648A3
:105EE000C7F80080FDF7B6F81248514603B0BDE888
:105EF000F04FFDF7CFB8B9F1170F1CBF3D688543D0
:105F00003D600E48EEE709F10109B9F1180FCFD154
:105F10000B490198324603B0BDE8F04FFFF7BEB918
:105F20005B02070874F9060865020708E2FA06082A
:105F30006C02070875F906081F0207082F020708F8
:105F400025FF0608014A40F202235FE7542D002096
:105F5000014B024A5AE700BFFFFF7F004C2D002093
:105F600010B5044601202BF0D5F928B92046054983
:105F7000BDE81040FFF792B9BDE810400248FDF7B8
:105F800089B800BF7702070886020708074B10B5DB
:105F90000446D3F83C0235F0EDFD28B9204604490B
:105FA000BDE81040FFF77AB910BD00BF409900204E
:105FB0009102070870B5054608461646FBF748FDEE
:105FC0000D4B041E1A780EDB944205DA0B4821466D
:105FD000FDF760F8204670BD2EB1FF2C03D10848B4
:105FE000FDF758F8F6E70749013A2846FFF756F952
:105FF0004FF0FF34EEE700BFD0110010A7020708F2
:10600000B8020708CB0207082DE9F04F074691B008
:106010008248834D0E46FDF73DF88249C5F840D2CF
:10602000002385F8443206220123097830464024B3
:1060300085F8454206F0F8FB0A20F4F71FFD95F8B5
:1060400044320C2BDAB240F2E4809DF80C60FE2E54
:106050002CD0FF2E15BF0F241524002501259442B6
:1060600040F0D780611EC9B268463BF017F804F1D2
:1060700040030DEB030414F8413C834240F0C4801C
:106080006A1E012A9DF80D3012D903F01F076137EF
:106090005C096548FCF7DEFF022D39D0013C042C79
:1060A00034D8DFE804F00B2D2F3331000225D6E77A
:1060B0009DF80E709DF80F401E46EAE75B48DFF83A
:1060C000C491DFF8C4A1DFF8C4B1FDF72FF8584838
:1060D000FCF7C0FF6C464FF0000814F8011B48465F
:1060E00008F10108FEF742F9B8F10C0F16D00AFBCF
:1060F00008F3B3F1553FF0D85846FCF7ABFFECE797
:106100004C48DCE74C48DAE74C48D8E74C48D6E73F
:1061100000238DF83F300DF11F00D0E7FCF7A2FF00
:10612000022D3AD06422B6FBF2F102FB11623B462B
:106130004448D2B2C9B2FCF7ADFF85F001035B421F
:10614000DBB2012B59D8404A404B9DF81010404813
:10615000404E00290CBF11461946FCF79BFF9DF8E5
:1061600011103D4B3D4800290CBF31461946FCF744
:1061700091FF022D41D19DF812403948FCF76AFF8A
:106180008CB1FF2C1FD00A23B4FBF3F103FB1142A7
:106190003448D2B2FCF77EFF08E033483A46314635
:1061A000FCF778FFCFE73046FCF7C0FF9DF81340BF
:1061B0002E48FCF74FFF44B1FF2C21D02C4821463C
:1061C000FCF768FF04E02B48EEE72248FCF7AEFF3F
:1061D000204E214FDFF89C800DF11305002415F8A7
:1061E000013F7BB1FF2B14BF3A464246214622486D
:1061F0000134FCF74FFF042CF1D111B0BDE8F08F52
:106200001C48E3E73246F1E71C493846FFF746F8F9
:10621000F3E71B48FCF78AFFEFE700BF110307080D
:1062200040990020D0110010220307082D03070811
:1062300053030708340307083C030708440307080F
:1062400030F8060865030708FA020708F102070894
:106250009C03070801030708350D0708B303070867
:10626000BA030708CE03070881030708D603070807
:106270002EF7060805030708E6030708F1030708D9
:10628000010407088DF40608ABAAAAAA151007088E
:106290002DE9F843DFF8A49007460C46204647F066
:1062A00019FF064658B91D4B1D481A781D4B03EBC4
:1062B0008203D3F8B815BDE8F843FCF7EBBE0246FD
:1062C00049462046FBF7E8FA60B1DFF86480002514
:1062D00058F8041BB1B9224638461349BDE8F843C3
:1062E000FEF7DCBF1148124C124DFCF7B3FE54F818
:1062F000041B19B12846FEF739F8F8E7BDE8F84362
:10630000FCF7B0BE32462046FBF7C6FA013500283E
:10631000DED1024B084C1D70C0E700BF842C00206A
:106320000A040708D823060825FF06086C02070898
:106330009429060875F9060865090708E2FA0608AF
:1063400038B50D4604461A4905222846FBF7A4FA3B
:1063500068B9184B93F84C2022B9012183F84C10EE
:1063600083F84D20BDE838401348FCF7DFBE1349E1
:1063700003222846FBF790FAA0B90E4D95F84C3051
:1063800063B195F84D304BB10D492046FEF786FFBD
:10639000002385F84C3085F84D3038BD0948FCF7AE
:1063A000C5FEF5E720460849BDE83840FEF776BF50
:1063B0008C0C07084888002014040708DE0D070825
:1063C0002A040708610407087504070870B5184C0B
:1063D00094F84C3005467BB194F84D3063B11549C3
:1063E000FEF75CFF28461449FEF758FF002084F8AA
:1063F0004C0084F84D0070BD104B93F83922AAB1BF
:1064000093F8182292B903F2192203F5127503F2D8
:106410003926106851682C4603C40832B24225461A
:10642000F7D1012283F8832208F030FB0120E2E754
:10643000488800202A04070884040708409900209F
:106440002DE9F04F80468BB008460D4647F042FEDE
:106450000246B0B3A3492846FBF71EFA044680BBA8
:10646000FCF700FEA048A14DA14EA24FDFF8C48268
:10647000FCF75CFE142041F0D9FEE110304604F038
:1064800007020131FDF772FF95F81D9095F91C0088
:10649000B9F1000F0ED006F0F1FC4A460146404625
:1064A000FCF7F8FD0134102C05F12405E5D10BB003
:1064B000BDE8F08F06F0E2FC01463846FCF7EAFD45
:1064C000F0E728468C4905AA49F069FF054620B93E
:1064D00001464120FCF749FEE9E78849FAF72AF925
:1064E00020B987494046FEF7D9FEE0E7854E0827E8
:1064F000002431682846FAF71DF9002808BF344601
:10650000013F06F11006F4D154B97F492846FAF745
:1065100011F928B17D492A464046FEF7BFFEC6E77D
:10652000002075498DF8130005AA49F038FF06468A
:10653000002C4DD0002849D0FBF78AFA031E42DB1D
:106540002279062A3AD1E268012101FA03F01042C9
:1065500039D0DBB247F6FE7040FA03F2D20732D5EB
:1065600099400139084049F0CBFF0546E08840F0EA
:1065700023FC6749D0E902230978002918BF1A468D
:10658000217A637A05FB0133002712F90390039700
:1065900002EB030A584905AA002049F000FF834690
:1065A00000283ED15B49012394B39AF9002020468C
:1065B000CDE900312946FAF72DFC78E75D1E13B1CD
:1065C000A37A9D42D2DB54493246A5E7534EFAE7FF
:1065D00068B10DF11301FBF715FA28B19DF81350BE
:1065E0002846F4F789FB20B94D49324694E74B4ED3
:1065F000FAE72846F4F73AFF8146284607F062FC9E
:106600000390284607F09AFCA24607462546C1E7B4
:10661000CDE900319DF813004A463946FAF73EFCB1
:1066200045E73649FAF786F8064658BBACB13D4F08
:10663000EDB2207972B22946F4F7F2FE00283FF459
:1066400036AF0288037800933146C2F303233846FD
:10665000120BFCF71FFD0136EBE7324C79793868F5
:1066600072B2F4F71FFF00283FF421AF02880378CD
:1066700000933146C2F303232046120BFCF70AFDB8
:106680000136EBE728495846FAF754F8002853D06A
:106690005846FBF7DDF9064642B29CB12079E9B2D3
:1066A000F4F7BEFE002849D129462046FAF766FADB
:1066B00026681E49CDF800B0034632464046FEF734
:1066C000EDFDF4E679793868F4F7ECFEB0BB9DF89F
:1066D00013301749CDF800B01A09403203F00F0308
:1066E000ECE700BFA2040708A7040708280200205F
:1066F000BD04070875F9060851FF0608E2FA060806
:10670000CE040708B405002007080708E2040708BC
:10671000488800206D300108F10407086509070862
:10672000010507081305070867020708340507086D
:10673000570507082C0607084FF0FF3606AF394605
:106740003046FBF72BF808A94846FBF727F84E45DB
:106750001CD076B274B18AF8006029462046FAF758
:106760000DFA266800970246134808AB3146FCF73D
:1067700091FC9CE69DF81320039B10489E70110924
:10678000009708AB02F00F024031F0E75CB12946F8
:106790002046FAF7F3F926680246094808AB314665
:1067A000FCF778FC83E69DF813200648110908AB36
:1067B00002F00F024031F3E77F050708A205070842
:1067C000CA050708E50507082DE9F04F07468DB013
:1067D00008460D4647F07EFC044630B901460120CC
:1067E0000DB0BDE8F04FFCF7CBBD0246A5492846E9
:1067F000FBF752F830B9A44938460DB0BDE8F04F68
:10680000FEF74CBDA14922462846FBF745F8002873
:1068100054D1FCF727FC9E48DFF8B4A2DFF8B4B2ED
:10682000FCF784FC172041F001FD0E271AF9018BBB
:10683000B8F1000F36D041465846FDF797FD0025C8
:106840002E46B10089B2404607F0B2FB814607F000
:106850003BFC90F9003004460136CBB10DB9FCF792
:1068600001FC99F80630657894F90000894A8A4C51
:1068700003F00203002B18BF1446B5B106F0FEFA70
:1068800000950346224685483146FCF703FC012566
:10689000042ED6D115B98248FCF748FC013F17F009
:1068A000FF07C3D10DB0BDE8F08F06F0E7FA22462E
:1068B000034631467B48FCF7EDFBE8E700247649C8
:1068C0008DF81B4007AA284649F069FD18B93846DB
:1068D000FEF7FAFCE6E70DF11B01FBF793F88146A2
:1068E0000028F4D09DF81B502846F4F705FA20B98B
:1068F0006D493846FEF7D2FCD4E7DFF8DC81234649
:106900004FF0FF3403EB430218F8022095420BD0FE
:10691000002C02DA002A08BF1C460133152BF1D1E6
:10692000002C16DA6149E4E71C465B4907AA0020FF
:1069300049F035FD0646002800F096805149F9F7E8
:10694000F9FE30BB5A4FDFF84C81DFF890910446D6
:1069500016E04FF00009E8E7306896F807A0F5F771
:1069600093F8B179737911F0020F0CBF39464146A3
:106970009B0802460091013351464846FCF78AFBCA
:1069800001342146284607F0B1FA06460028E3D133
:1069900088E7484902223046FAF77EFF4FEA151A87
:1069A0000AF1400A05F00F0B002845D10390B01CF6
:1069B000FBF74EF8039902460491284601310592EF
:1069C000039107F093FADDE90313059A38B93A49C0
:1069D00000965B4652463846FEF760FC62E7C07997
:1069E0009042E9D11F466300B9F1000F31D01A1966
:1069F00042445678013E7A1C234414BF29460021A4
:106A000008EB030208F803107B1C53700AACFF2349
:106A10009370394622462846FAF7D0FE08AA314636
:106A20002846FAF7CBFEB74216D1244808AB5A469F
:106A30005146FCF72FFB35E721493046F9F77AFE3E
:106A400020B1204900965B465246C4E74FF0FF371D
:106A5000C9E74FF0FF36CEE71B48009408AB5A4613
:106A60005146FCF717FB1DE704EB4404174B00935A
:106A7000A044024698F8011001232846FAF754FA78
:106A800010E700BFE2FA0608CE040708A2040708D0
:106A90000106070880F7060851FF060821060708C7
:106AA0004206070833060708480607085F06070876
:106AB00065090708880607088B060708DD0607082A
:106AC00067020708B7060708FB0607086D300108CC
:106AD000688306081A060708AC2200207306070818
:106AE0002DE9F04F89B0074605AA08469C4949F0B0
:106AF00056FC054630B901464120FDF7B3FB09B00D
:106B0000BDE8F08F9749F9F715FE044600283CD1FF
:106B10009548964D964EDFF89882FCF707FB1420B7
:106B200041F084FB95F9060006F0A8F92968AA88C7
:106B300001F13F4101F57E01B2FA82F2890A034672
:106B40004131C2F11F023046FDF710FCE97911B165
:106B50004046FDF70BFC0134FCF784FA602C05F18C
:106B60000805DFD17E4905AA002049F018FC8149BB
:106B7000F9F7E0FD0028C2D138467A49FFF724FE34
:106B800078493846FFF75CFCB9E7DFF8FC91002450
:106B900019F9340006F072F9804601462846F9F7E3
:106BA000C9FD40B10134212CF2D173492A4638463F
:106BB000FEF774FBA3E76A4905AA49F0F0FB064615
:106BC00090B3FAF745FF05466C4B03EBC4034FEA5D
:106BD000C40A93F8D2314BBB002D29DC09EB0A0320
:106BE000588893F8049093F805A040F0E5F8EBB2CC
:106BF000D0F808B0009303FB09AA002E00F09A8099
:106C00003378002B00F0968006A93046FAF7FAFE9A
:106C1000002800F08C809DF8185005BB0BF80A5036
:106C20005748FCF783FA6AE70546CDE7002D05DDF6
:106C3000012B1A4638BF0122954208DD012B51492C
:106C400038BF012301223846FEF7DAFB57E74449F3
:106C500005AA002049F0A3FB013D0646BEE72846F1
:106C6000F4F74AF8814600285DD02B09403302939F
:106C70000BF80A5005F00F03434F03934FF0000841
:106C8000BB79012B38BF012301930026788897F840
:106C900004B097F805A040F08FF806FB0BA38268BC
:106CA000D15CA94222D1444504D10099B1421DD002
:106CB0000021D154DDE9021234485FFA86FB5FFA05
:106CC00088FAFDF753FB59465046FEF73FF8444516
:106CD00009D12F48FDF74AFB50465946FEF736F8D2
:106CE0002C48FDF743FB2C48FCF720FA019B0136AA
:106CF000B342CBDC08F10108B8F1210F07F1080716
:106D0000BED1D9F80010B9F80420244801F13F4160
:106D100001F57E01B2FA82F2890AC2F11F02413105
:106D2000FCF7B8F9EBE63846FEF7CEFAE7E61C4981
:106D300032463CE71BF80A30013573B11A0919498C
:106D400003F00F03403206A8FAF7B0FC06AB164872
:106D50002A464146FCF79EF9D1E6144BF7E700BFFF
:106D600051FF0608A204070821070708901A00200F
:106D70005F0707086A0707086E070708D823060891
:106D8000900707088A070708A4250608A20707082E
:106D9000C6070708C9070708D90E0708D307070859
:106DA000EF070708E9F606080B080708CBF3060803
:106DB0002DF7060820B10078B0FA80F0400970473E
:106DC000012070472DE9F74F81460846FFF7F2FF93
:106DD0000E46054670B1002401A9204641F056FB3D
:106DE000013401464846FFF7EDFF122CF4D103B001
:106DF000BDE8F08F0846FAF72BFEC4B2112C71D80B
:106E0000701C3D4D3D4EF9F7C4FF05EB440867008B
:106E100098F884A28346B8B9AAF102014B424B41CB
:106E20003D4495F88422B25C002B54D095F885320D
:106E3000192040F2EE2100FB03133148214603B034
:106E4000BDE8F04FFCF726B90178304649F0DBFA8F
:106E500078B1032C94BF002201222A4902EB42029E
:106E6000831B0A4452FA83F393F8A0A6BAF1030FE6
:106E700005D1484603B0BDE8F04FFEF725BA5846A5
:106E8000F9F787FFF0B1BAF1020FF2D1FAF7E0FD9E
:106E900040F6CA0380B29842A8BF184640F2EE23DB
:106EA0009842B8BF1846A0F2EE201923B0FBF3F0C9
:106EB00088F88502AAF1020253425341EA1982F886
:106EC00084A2ADE7BAF1020FF4D1484603B0BDE8A1
:106ED000F04FFEF735BA0C48214603B0BDE8F04F3D
:106EE000FCF7D8B8094911232A46484603B0BDE843
:106EF000F04FFEF785BA00BF409900206094060865
:106F00001F080708D82306082F0807083C080708A9
:106F10002DE9F041054686B00846FFF74BFF0F46C6
:106F2000064640B100235C491A46012006B0BDE880
:106F3000F041FCF7E1BA0846FAF78AFD1328044647
:106F400000F3A18006254543781C8DF81760F9F7FA
:106F500020FF524E074660B1FAF77AFDC0B211F039
:106F6000AFFC30B17319027983F8402601238DF804
:106F700017303846F9F70DFF074668B1FAF768FD94
:106F80000D2809D8062303FB046383F841069DF806
:106F9000173001338DF81730DFF8FC80A91C0DF194
:106FA000170241443846FAF757FDF9F7F2FE074653
:106FB00068B1FAF74DFD012809D89DF8173006226F
:106FC00002FB0462013382F844068DF8173038461C
:106FD000F9F7DFFE80B1FAF73BFDC0B211F070FCAB
:106FE00050B19DF817300179062202FB046201338B
:106FF00082F845168DF817309DF81720042A4FF0B7
:1070000006032FD103FB04630022A3F844260625C0
:1070100005FB046520F0E6F995F8400611F034FC14
:1070200095F8431695F8427619234FF4617280461D
:1070300095F8450613FB012613FB072711F024FCE6
:10704000437998F80520039395F844360097CDE9E5
:107050000163134895F841362146FCF71BF806B04A
:10706000BDE8F081052A05D103FB0463002283F803
:107070004526CCE7062ACAD008EB0502002348F8CB
:1070800005309380C3E7074913233246284606B0EC
:10709000BDE8F041FEF7B4B9888E00204888002092
:1070A0003CF506088A0707082DE9F04780468CB0B2
:1070B0000846FFF77FFE054640B1002359491A46AE
:1070C00001200CB0BDE8F047FCF792BACDE9090009
:1070D0000B90079107A8544949F034F9064641F04E
:1070E000B9F8431C04460ED12B460A2208A93046A3
:1070F000FAF70EFC089B1B782BB9C4B2132C96BF71
:10710000333444B264B2204607F06EFF054628B916
:107110004046FEF7D9F80CB0BDE8F08742498DF83B
:10712000284007A849F00EF9B0B300230A221946F7
:10713000FAF7EEFB02260990DFF8EC90DFF8F0A0FA
:107140000027494607A849F0FDF8F8B1FAF780FC96
:10715000364A002352F8041B88421FD1DBB20AEBE7
:107160008302D2F88C21904210D1022F20D0032F1D
:1071700023D05A1E012FD2B215D00B2A03D88DF876
:1071800029300136F6B20137042FDAD1052E1AD88C
:107190004046FEF7D5F8BEE70126CDE70133102BB8
:1071A000D8D10023DBE7052AEDD88DF82A30E8E7AF
:1071B000092BE8D88DF82C30E3E79A1E0D2AE2D887
:1071C0008DF82B30DDE709AB03CB286018686960C8
:1071D000A860204641F044F9154A9DF82B1002EBB7
:1071E00081010346D1F88C1104919DF82C1002EB1B
:1071F0008101D1F88C1103919DF82A1002EB8101D5
:10720000D1F88C1102919DF8291002EB8102002126
:10721000D2F88C210192099A00920846054AFBF7A0
:1072200025FF78E77C8D002051FF060864250608BD
:10723000D823060855F506082DE9F04F0346A1B0FE
:107240000846FFF7B7FD054628B1184621B0BDE84E
:10725000F04FFEF775B8DFF8C4920B90FF238DF85E
:107260002830D9F83C32ADF83000CDE9050093F86C
:1072700038200D908DF838200F90ADF84000119314
:10728000099107464FF0FF38934909A849F05AF889
:10729000044618BB914F01460AAC0B0190481A579F
:1072A000002310F9016BB24240F0D28010464E1C10
:1072B00041F0D6F8314602463846FBF7EBFE022E87
:1072C0004FF00101E9D19DF938A09DF928305345CF
:1072D00040F0C5808348FBF7DDFE4DE02378002BAE
:1072E000D2D0032FD4BF00260126062F00F2A9809A
:1072F000DFE807F00447509104475000042F10D0F6
:1073000079492046FAF7ECFA58B14FF4806007F05B
:10731000E3FE002800F0B58190F9040001230693F4
:107320000AE072492046F9F705FA70B9D9F83C32FB
:1073300093F93800042F22D0119B119320AB03EB5B
:10734000061606F8580C01379EE7204640F082FFEB
:107350000028EFDA01230A2212A92046FAF7D8FA08
:1073600040B2002803DB129B1B78002BE2D0604860
:107370002246711CFBF78EFE21B0BDE8F08F002382
:10738000DBE72046FAF764FB20AB03EB061646F872
:10739000540CD8E757492046FAF7A2FA5649B0F1FB
:1073A000000A204618BF4FF0010AFAF799FA08B10F
:1073B0004AF0020A3301DFF868C1079320AB03EB00
:1073C0000616BCE80F0006F850AC12AE0FC6BCE8BB
:1073D0000F000FC6BCE80F000FC69CE8030086E84C
:1073E000030000260DF1480AB346DAF800102046E3
:1073F00049F060F810B19AF804301E430BF1010B0C
:10740000BBF1070F0AF1080AEFD1079B80336B44E9
:1074100003F84F6C97E739492046F9F78BF9A0B18B
:1074200037492046F9F786F900288CD02046FAF72C
:107430000FFB0328804686D901463248FBF72AFE17
:107440009AE731482246082194E7012305937AE719
:107450000133072B7FF425AF2C4801318AE70B9BC2
:107460001BB9AAF114025542554100235F1CE36881
:10747000002B62D194F900B0584607F0FDFDD4F816
:10748000049018B10668002E40F08B80B9F1000F0F
:10749000237A14BF4E464FF46146666023B91C48F8
:1074A000FBF7F8FD03232372627A2AB11948079289
:1074B0003946FBF7EFFD079A0292237ACDE9006384
:1074C00000231A461946584607F062FEE06048BBA2
:1074D00011483946B2E700BF51FF0608C008070847
:1074E000091C0608DD0807085F0807086A0807087E
:1074F0006E08070889080708620D07081AFF0608C2
:10750000670207088C080708A4080708CB080708C3
:10751000F6080708110907082C09070840990020F8
:10752000802A06085849594A5948B9F1000F18BF2E
:107530000A4633463946FCF719FF022F04F11004BE
:107540004FF0010392D1119E0D9F4DB15148FBF7B1
:10755000EDFD33681B6A1BB14F493A4630469847E8
:10756000059B002B50D04D49474BBAF1140F18BF63
:1075700019464B48FBF78EFDBAF1140F09D1059B54
:10758000002B43D03368DB691BB1464900223046EB
:107590009847069B002B43D100223146384640F0E5
:1075A00071FEE660B9F1000F2CD04946304601F07B
:1075B00089FE3D4AB3683D483946FBF76BFD94F8B8
:1075C0000890B9F1000F0CD03279914509D03848B4
:1075D0004B463946FBF75EFD336849469B693046AA
:1075E0009847637A23B1727932483946FBF752FDE6
:1075F000F36A002BA1D030483946FBF74BFD00233E
:10760000F3629AE7204AD5E71F49B2E7B8F1000FC5
:10761000BFDB3368DB69002BBBD028494246B6E7A5
:1076200005F0E6FB0520F3F729FADFF89490DFF880
:1076300094A000254FF0030B9AF80030AB42ABD971
:1076400019F8014FC4B1204606F078FC804698B185
:107650002046F3F751FBEBB2044610B180F806B0B8
:10766000C37120460121F3F7AFFA98F80630DB0723
:10767000204603D5F3F79EFC0135DDE7F3F794FCD4
:10768000FAE74FF0FF3049E66509070844080708A4
:1076900048090708FE090708C592010852080708AB
:1076A000270A0708AD0D01084D08070866090708F5
:1076B0008B090708AE090708E5090708410B01080F
:1076C000F3220020D01100102DE9F04380468BB04A
:1076D0000846FFF76FFB0F46044640B100235E49A2
:1076E0001A4601200BB0BDE8F043FCF707B8084686
:1076F000FAF7AEF91D28054600F3A5800A26464391
:10770000781C8DF82740F9F744FB10B101238DF860
:107710002730F9F73EFB514C074668B1FAF798F964
:107720000D2809D80A2303FB054383F8A8029DF816
:10773000273001338DF82730DFF81C91711C0DF1D3
:10774000270249443846FAF787F9F9F722FB07463A
:1077500068B1FAF77DF9232809D89DF827300A2265
:1077600002FB0542013382F8AB028DF82730384620
:10777000F9F70FFB074668B1FAF76AF90D2809D83F
:107780009DF827300A2202FB0542013382F8AC0241
:107790008DF827309DF82730062B0CD009EB060218
:1077A0000023404649F80630536013810BB0BDE812
:1077B000F043FDF7C5BD0A2606FB05460023384603
:1077C000A6F8AE32A6F8B032F9F7E3FA074618B1D8
:1077D000FAF73EF9A6F8AE023846F9F7DAFA30B110
:1077E000FAF736F90A2303FB0543A3F8B0021C4B52
:1077F0004FF0FF325A600A2303FB05424FF46170D9
:10780000B2F8B0320693B2F8AE32059392F8AC32C9
:10781000049392F8AB32039392F8AA12192313FB44
:107820000101029192F8A91213FB0103019392F84E
:10783000A832009300210B4A2B460846FBF716FCA2
:107840000BB0BDE8F08308491D23224640460BB02B
:10785000BDE8F043FDF7D4BDE89B0020409900202F
:10786000A805002072F506088A0707082DE9F14FE0
:10787000DFF894B106460D462846FFF79BFA074607
:1078800040B1002359491A46012001B0BDE8F04F2C
:10789000FBF798BF564905222846F9F7FDFF60B966
:1078A000524B00221A601A611A621A631A641A652E
:1078B0001A661A6701B0BDE8F08F042259462846BF
:1078C000F9F7EAFF04462846002C42D1F9F761FA9D
:1078D00007460028EED046F0FDFBDFF830A15FFA46
:1078E00080F85AF8049BB9F1000F07D141492A46A4
:1078F000304601B0BDE8F04FFDF7D0BC42464946E6
:107900003846F9F7C9FF013484460028E9D1374ADF
:107910000346154600210133082B42F8101BFAD10B
:10792000354B03EBC40257682FB93448344D4946F0
:10793000FBF7B0FBA0E713F834E0F445F5DA07EB0A
:107940000C130FCB05EB0C1484E80F000CF1010CA9
:10795000F3E7FAF77DF8072804463DD82846F9F7FB
:1079600018FA074658B3F8F787FF204B03EB0413C8
:1079700083ED000A01253846F9F70BFA074638B1BE
:10798000F8F77AFF194B03EB041383ED010A013575
:107990003846F9F7FEF9074638B1F8F76DFF134B93
:1079A00003EB041383ED020A01353846F9F7F1F9C8
:1079B00038B9304601B0BDE8F04FFDF7C1BC05460F
:1079C000D9E7F8F759FF094B032D03EB041383EDB7
:1079D000030A3FF456AFECE70A4907233A4630461C
:1079E00001B0BDE8F04FFDF70BBD00BF8C2C0020AF
:1079F0001AFF060825FF0608101C060836FF0608B1
:107A0000650907088A07070820FF06089429060861
:107A10002DE9F34105460846FFF7CCF90C46074629
:107A200040B1002333491A46012002B0BDE8F041BD
:107A3000FBF764BF30492046F8F77CFE70B92D4B48
:107A400004224FF47A704FF4FA61013A1880598099
:107A500003F10403F9D102B0BDE8F0812046F9F743
:107A6000F7FF0328064641D82046F9F792F9074662
:107A700098B1F9F7EDFF4FF0010804463846F9F7E1
:107A800088F920B1F9F7E4FFB8F1000F09D12846D1
:107A900002B0BDE8F041FDF753BC40F2EE24804651
:107AA000ECE7A4F2EE2240F2DC539A4203D8A0F2B3
:107AB000EE229A420AD9114940F6CA0340F2EE2258
:107AC000284602B0BDE8F041FDF79ABC0C4B0D4AC8
:107AD00003EB86030021A3F8D443A3F8D603CDE932
:107AE000004033460846FBF7C1FAB4E706490323D2
:107AF0003A46E5E7149D00201AFF06084A0A0708DF
:107B000040990020A9F506083C080708F0B507468B
:107B100089B00846FFF74EF90E46054640B10023EE
:107B20001A491A46012009B0BDE8F040FBF72ABF08
:107B30000846F9F78DFF1F2804461DD83046F9F78F
:107B400028F90146204634F0FDF978B10F4803AE1C
:107B5000314600EB840040F031FC0D4A009623468C
:107B600029462846FBF782FA09B0F0BD384609B02D
:107B7000BDE8F040FDF7A8BB06491F232A4638465A
:107B800009B0BDE8F040FDF73BBC00BF249D0020DC
:107B9000BAF506088A070708F0B5074685B0084613
:107BA000FFF708F90E46054640B100231D491A4665
:107BB000012005B0BDE8F040FBF72CBF0846F9F7FF
:107BC00047FF0F28044623DC3046F9F7E2F8014668
:107BD000204634F09DFAA8B1134B04F1200203EBC8
:107BE0008203294693F8E723029293F8E623019251
:107BF000B3F8E43300930D4A23462846FBF736FAE0
:107C000005B0F0BD384605B0BDE8F040FDF75CBBFF
:107C100007490F232A46384605B0BDE8F040FDF776
:107C2000EFBB00BFA49D002040990020C4F50608CA
:107C30008A070708F0B5054685B00846FFF7BAF889
:107C40000B46044640B100231B491A46012005B0EB
:107C5000BDE8F040FBF726BF1849184F6A461846A2
:107C600048F09DFB01AE88B1032C04D12846FDF7F6
:107C700067FB05B0F0BDF9F7EBFE6A4646F8040B6A
:107C800039460020013448F08AFBECE7032CEDD1A3
:107C9000DDE90146039F31463A46E0B234F074FA1A
:107CA00018B92846FDF710FBE3E705483B46324686
:107CB0002146FBF7EFF9DCE7249D002051FF060881
:107CC000D6F50608F0B506468BB00846FFF772F801
:107CD0000D46044628B300233E491A4601200BB046
:107CE000BDE8F040FBF77CBF2D2903D0A1F13003A4
:107CF000092B49D8052C05DD30460BB0BDE8F04016
:107D0000FDF71EBB2846F9F7A3FE0AAB621C03EB86
:107D1000440424F80C0C15F8013F303B092BFAD928
:107D2000144629780029DFD1062CE5D1BDF81C20A6
:107D3000BDF91C30072ADFD8BDF91E50A5F5FA722F
:107D400092B2B2F5FA6F18D8BDF92070A7F5FA72A1
:107D500092B2B2F5FA6F10D8BDF922C065450CDCBD
:107D600067450ADBBDF924E00EF1640292B2C82A2D
:107D700003D8BDF92640112C11DD174930460BB050
:107D8000BDE8F040FDF78ABA202902D1013522462C
:107D9000C6E730460BB0BDE8F040FDF795BA0F4A94
:107DA0000C2000FB032264B2A2F8BC51A2F8BE7101
:107DB000A2F8C0C182F8C2E182F8C3410846CDE909
:107DC00003E4CDE9017C064A0095FBF74FF90BB0BF
:107DD000F0BD00BFF89A002059FF06084099002026
:107DE000EAF506082DE9F04F074689B00846FEF788
:107DF000E1FF8B46054640B100234D491A4601205C
:107E000009B0BDE8F04FFCF70FB84A4B084693F8AD
:107E1000DCA693F8DD9693F8C687F9F719FE0928D2
:107E200004467BDC062646430BF101008DF81F500B
:107E3000F8F7AFFF3E4D834638B1F9F709FE0D283C
:107E400003D80123A8558DF81F305846F8F7A1FF35
:107E5000834660B1F9F7FCFD504508D8062303FBC3
:107E6000045358709DF81F3001338DF81F30584669
:107E7000F8F78FFF824660B1F9F7EAFD484508D868
:107E8000062303FB045398709DF81F3001338DF8CF
:107E90001F305046F8F77DFF814660B1F9F7D8FDF5
:107EA000804508D3062303FB0453D8709DF81F3088
:107EB00001338DF81F30311D0DF11F022944484652
:107EC000F9F7CAFD9DF81F30062B09D0AA19002327
:107ED0003846AB51938009B0BDE8F04FFDF730BA9A
:107EE0006343EA184FF461765079192111FB006061
:107EF0000590107911FB00610491D178039191787C
:107F0000029152780192EB5C009300210A4A2346C9
:107F10000846FBF7ABF809B0BDE8F08F0749092325
:107F20002A46384609B0BDE8F04FFDF769BA00BFF0
:107F3000AC2D00204888002034F606088A07070880
:107F40002DE9F74F05460846FEF734FF0B46044679
:107F500018B9334A92F8D4742FB9284603B0BDE853
:107F6000F04FFDF7B1B92F49DFF8C890DFF8C8A08E
:107F700001AA184648F013FA264610B904F044FF47
:107F800008E056B9012201462846FEF713F8421CC4
:107F900004461AD103B0BDE8F08FF9F759FD2F2838
:107FA000834636D80FB104F023FFBBF1060F13D080
:107FB0001D49012309785FFA8BF2E0B204F034FC2A
:107FC00059464846FBF766F80027164901AA0020E3
:107FD000013648F0E4F9D0E7DAF800301B0114D597
:107FE000FF2C0ED0E1B22846FEF70EF8E8E728464F
:107FF000FEF70AF8013798F80020F9B28A42F6D85D
:10800000DEE7DFF824800027F5E70848FBF78EF865
:10801000D6E707492F222846FDF740F9D5E700BFEC
:108020004099002051FF0608D01100107702070880
:10803000690A0708580A07082C2C00202DE9F74385
:1080400007460846FEF7B6FE0B46044628B13846FA
:1080500003B0BDE8F043FDF773B92F49DFF8B890DE
:1080600001AA184648F09BF926460546A04665B980
:108070002A4B3246D3F83C02A1B242F0E9F968BB80
:1080800027493846FDF70AF928E0B8F1000F06D075
:10809000B8F1010F25D03846FDF752F91EE0284609
:1080A00046F018F81F49064602462846F9F7F4FB41
:1080B00050B31D4932462846F9F7EEFB30B31B4951
:1080C00032462846F9F7E8FB10B3194932462846EC
:1080D000F9F7E2FBF0B13846FDF7F6F803B0BDE87A
:1080E000F083B31E5A425A4129463846FDF762FFD3
:1080F000421C0446F2D001AA4946002048F04FF93C
:1081000008F101080546B2E74646F4E70126F2E722
:108110000226F0E70426EEE751FF0608409900200A
:10812000950A0708890A07088C0A07088F0A0708B2
:10813000920A07082DE9F74380460846FEF73AFE03
:108140000B46054628B14046FDF7FAF803B0BDE8F6
:10815000F0832D49DFF8B09001AA184648F01FF9C6
:108160002F4604462E467CB9022DECD1A7F57A7332
:10817000B3F57A7F21D925494FF4FA634FF47A7227
:108180004046FDF73DF9E1E74DB1012D10D001AAC0
:108190004946002048F003F901350446E3E701228F
:1081A00021464046FDF706FF431C0646EFD1CDE7CA
:1081B0002046F9F74DFC0746E9E7154B1B68B8B2B6
:1081C0005B689847FF2EBCEEC00A124B0BD1124AD7
:1081D000F8EE407A1278A24212DC10EE101A0F4824
:1081E000FAF758FFB2E7F8EE407A03EB860310EE99
:1081F000102A0B48C3ED007A3146FAF74BFFA5E78A
:10820000E3EC017A0134E6E751FF0608A30B070807
:108210004C170010189E0020D0110010C00A07084B
:10822000B30A0708F8B507460846FEF7C3FDD0B104
:10823000204BD3F898600136304606F0C7FE34462E
:108240000546F0B90134182CA8BF0024204606F0DA
:10825000BDFE0546A8B9B442F4D138461649BDE87A
:10826000F840FDF71BB80846F9F7F2FB044606F0A4
:10827000ADFE054628B921461048BDE8F840FAF79A
:1082800009BF0C4BC3F8984007F018F80C482A4671
:108290002146FAF7FFFE172C09D80A4B0C2202FBE5
:1082A000043393F8E006BDE8F84007F043B8002037
:1082B000F9E700BFA8050020CF0A0708E30A07086E
:1082C000F90A0708D823060838B5124D04460846AF
:1082D000FEF770FD60B1104B104893F900104B1C75
:1082E0000ABF0F4BC9B21978BDE83840FAF7D2BEC1
:1082F0000846F9F7ADFB032804D8C0B2FAF7E8FA4C
:108300002946E4E720460749BDE838400322FCF748
:10831000C5BF00BF65090708A8050020120B0708A4
:10832000002C0020220B0708F0B5032985B0054674
:108330000C46164614D80B4F3970FAF793FE0A49CB
:108340002846FFF7C1FF0949224601A8F9F7AEF90F
:1083500001AB324608212846FCF71EFFFF233B7085
:1083600005B0F0BDA805002065090708120B070835
:1083700038B5124D04460846FEF71CFD60B1104B9F
:10838000104893F901104B1C0ABF0F4BC9B2597822
:10839000BDE83840FAF77EBE0846F9F759FB0328D6
:1083A00004D8C0B212F044F82946E4E72046074951
:1083B000BDE838400322FCF771BF00BF650907081C
:1083C000A80500200E0B0708002C00201D0B070835
:1083D000F0B5032985B005460C46164614D80B4F58
:1083E0007970FAF73FFE0A492846FFF7C1FF0949AD
:1083F00022466846F9F75AF96B463246102128465C
:10840000FCF7CAFEFF237B7005B0F0BDA805002075
:10841000650907080E0B07082DE9F74F444BDFF8F5
:108420002C911A785B7889F80130424B00911B78C7
:1084300089F8002005460BB904F032F83EF0F6FC4E
:1084400000263D4CB0460D233B4A0099734352F839
:1084500003A05046F9F744FA002841D0B8F1000FC4
:1084600001DDFAF7FFFD35485146FBF77FFF00229B
:1084700021462846FCF704FFFAF7F4FD237903F0C0
:108480001803082B46D0102B49D02046FBF77BFF62
:10849000294B0D2202FB0633B3F809003EF08CFC99
:1084A0008346D8B12046F8F717FBDBE902210746DF
:1084B000024401442046F8F7A7FA78B901905146E2
:1084C0001F48FBF753FFDBF80810019A28461346B4
:1084D000CA192146FCF776FDFAF7C4FD08F1010838
:1084E000013640F26A239E4204F10D04ABD1002014
:1084F000F8F7D1FAFF2389F8003089F80130B8F194
:10850000000F11D1009A0F49284603B0BDE8F04F83
:10851000FCF7C4BE0C492846FFF7D6FEB5E70A496A
:108520002846FFF725FFB0E703B0BDE8F08F00BF96
:10853000002C002048880020E432060889FE060846
:108540003D0B070825FF060865090708A805002058
:108550002DE9F74F804608460F4645F0BBFD04461F
:1085600020B1012825D13B782A2B22D1A948AA4E37
:10857000AA4FFAF7DBFD0025B1464FF00D0A04F0D3
:1085800001040AFB05F3384659F80310FBF7EEFE29
:10859000314622464046FCF773FE0135FAF762FD8C
:1085A00040F26A239D4206F10D06EAD103B0BDE810
:1085B000F08F3D21384647F026FF002800F0238148
:1085C00003469A4613F8012D202AFAD0AAEB070A8F
:1085D0000130054610F8013B202BFAD0DFF838B205
:1085E0005FFA8AFA4FF000090D2303FB09F35246A4
:1085F0005BF80310009138460BEB0304F9F74CF9D4
:10860000064670BB0099084645F064FD824528D1B6
:10861000277907F0E001402900F0898012D871B372
:1086200066797F4A02EBC606002796F8D8220092A8
:10863000BA463B46009ABA4202D9BAF1000F62D05C
:108640002BB12DE06029ECD0802900F0A4804046B9
:108650007449FCF723FE204603B0BDE8F04FFBF75A
:1086600092BE09F1010940F26A239945BCD16E49D5
:108670003A46404603B0BDE8F04FFCF70FBE07F0A6
:108680000703042B1CD10B460A222846F9F740F9B0
:10869000D4F8053083420146D9D32046F8F736FB9B
:1086A0000D2303FB09F961485BF80910FBF75EFE37
:1086B00000222146404603B0BDE8F04FFCF7E0BD84
:1086C000052B0DD101230A222846F9F721F9D4F808
:1086D000053083420146BADB5B428342B7DCDCE70C
:1086E0002846F9F7B5F917F0050F0BBFB4F80520C8
:1086F000B4F90520B4F80730B4F9073090420146C8
:10870000A5DB9842EAE7D6F8D41251F8270060B109
:1087100029460193F8F70EF8019B30B939462046F7
:108720004FF0010AF8F7F2FA5346013782E763790E
:10873000009307F00707013F009BB342B0DDAA4654
:1087400015F8013B202BFAD02046F8F7CBFA054666
:10875000042F04D8DFE807F0030E0E141D00504666
:10876000F9F776F9A8552C21504647F04CFE013612
:10877000451CE1E75046F9F76BF925F81600F2E7DA
:1087800000230A2200215046F9F7C2F845F82600D6
:10879000E9E70123F5E7284645F09CFCE37994F8E6
:1087A00005A0A779DB0706460AD52046F8F79AFA0E
:1087B0000378014623B13246284647F04AFEE0B925
:1087C000DEB1B74219D32046F8F78CFA3A460021B9
:1087D00047F002FEB2453FF663AF154932462846E0
:1087E00047F037FE00283FF45BAF2046F8F77AFAEF
:1087F0003246294647F098FD52E70E493A46404630
:10880000FCF74CFD23E73946404603B0BDE8F04F86
:1088100002E600BF4D0B0708E432060889FE060891
:10882000D82306089B0B070825FF0608900B0708AE
:1088300015100708600B070870B5044608460E4679
:1088400045F048FC3146054602462046F9F724F833
:1088500068B9635D1846F9F709F800B933B901350D
:108860002C44204601340378202BFAD070BD002020
:10887000FCE708B504460948FAF7ECFBFAF7CEFB2B
:10888000074BD3F83C0206F049FC04F095FA012CA2
:1088900001D142F071FCF4F731F800BFA90B0708D1
:1088A0004099002010B5044608460B46FEF782FAB0
:1088B00028B9094903221846F8F7EEFF28B90748F6
:1088C000FAF73AFC0120FFF7D4FF20460449BDE83F
:1088D0001040FCF7E3BC00BFB50B0708B90B070855
:1088E000750407082DE9F74F064601AA08462E49E8
:1088F000DFF8C480DFF8C490DFF8ACA047F04FFD8C
:108900004FF0000B04465D46012714BBBBF1000F7E
:1089100027D1264C002D43D025482946FAF7BAFB2B
:1089200023780BB903F0BCFD3EF080FA002384F8F5
:108930004D30FAF749FB15B12846F8F7ACF89FB16E
:108940003046FDF743FD78B1FAF7A8F90020FFF7AC
:1089500090FFBBF1000F0AD02046F9F779F885B2F5
:10896000C5B93046FCF7B0FC03B0BDE8F08F414616
:108970002046F8F7B5FF80B949462046F8F7B0FF22
:108980000028EED05F4601AA5146002047F007FDBF
:108990000446BAE74FF0000BF5E74FF0010BF2E7A2
:1089A0000448FAF7C9FBBFE751FF060848880020D2
:1089B000E40B0708070C0708DB0B0708C30C0708C4
:1089C00010B50C46FDF702FD78B1084B01229A73F1
:1089D000FAF764F90648FAF7AFFB06492046F7F7BD
:1089E000A9FE10B10020FFF744FF10BD002C0020AD
:1089F0001D0C0708F0F406082DE9F04F93B00E4661
:108A00000290A04930461746FFF716FF054600289A
:108A100040F021819C493046FFF70EFF05460028B3
:108A200040F01B8199493046FFF706FF05460028B4
:108A300040F0158196493046FFF7FEFE05460028B6
:108A400040F00F8193493046FFF7F6FE00280546B7
:108A50000ABF0124082435467F4207F010078E49DB
:108A600028463C43FFF7E8FE002800F0FC8044F075
:108A700020048A4B1B780BB903F012FD3EF0D6F9A7
:108A800014F0090F00F050838548FAF755FB0020D9
:108A9000FCF7B6F814F48073059340F0EE8081483B
:108AA000FAF74AFB8048FAF741FB04F01803182B49
:108AB00005D17E48FAF740FB7D48FAF737FB0123E2
:108AC0000493FAF7CFFA7B497B48FAF7E3FA7B493C
:108AD0007B48FAF7DFFA04F48473082B07D179494D
:108AE0000298FAF7E6FA77490298FDF75FF814F072
:108AF000800307930ED1744B93F8F824002A734A2D
:108B000003F59F6306BF012113460021704A2046EA
:108B1000FAF7ACFA6F492046FBF7A4FB6E492046F2
:108B2000FAF72EFC6D492046FAF71FFB6C4BD3F881
:108B300000A06C4B14F010061D6840F0A0806A483D
:108B4000FAF7FAFA0396694B069399466AEA05031F
:108B50004FF00008099359F804BBBBF1000F21D076
:108B6000099B039A012707FA08F73B400CBF012134
:108B7000002120460893FAF7EBFA65EA0A033B4224
:108B800014BF012100215A4A03905B462046FAF7A0
:108B90009BFC0899564A00395B4618BF01212046C4
:108BA000FAF764FA08F10108B8F11D0FD3D165EAAC
:108BB0000A03DFF8549108934FF00008069B53F81E
:108BC00004BB0693BBF1000F24D0012707FA08F776
:108BD0003D420AD06AEA05033B424A465B4614BF5F
:108BE000012100212046FAF76FFC1AEA070F11D085
:108BF000089B039A1F400CBF012100212046FAF771
:108C0000A7FA391E03905B464A4618BF0121204649
:108C1000FAF72CFA08F10108B8F11D0FCED12A4D50
:108C2000344B354A05F5AC612046FAF7E1FC079B69
:108C3000002B6BD0134B029822461821FCF7ACFA9C
:108C4000049B002B00F0D4812C48FAF775FA2C48CD
:108C5000FAF76CFACCE10124FEE60224FCE60424D7
:108C6000FAE68124F8E627492846FFF7E5FD0028C3
:108C70003FF4FFAE44F48074FBE6002320E71A4B78
:108C8000039360E7430C07084A0C0708520C0708D7
:108C9000580C07086A070708FE0B070848880020D9
:108CA000660C07086E0C0708860C0708920C07086C
:108CB000BA0C070811FC06087701070821FC060812
:108CC0009501070865090708409900201510070855
:108CD000CA0C0708D70C0708E10C0708F9F80608C2
:108CE000BC330020C4310020240C0708042A0608E5
:108CF000E70C0708FE0C07087C8D0020C20D070852
:108D0000D80D0708610C0708F30C0708DFF8C0A3AB
:108D1000DFF8C0B39AF800209BF80030BC4F9A42AD
:108D200014BF01210021BB4A20460CBF4FF00109AE
:108D30004FF00009FAF70CFA9BF80030B64A07EB3F
:108D400083038046D3F8B83549462046FAF7BCFB82
:108D50009AF80030B04A07EB83074946D7F8B83590
:108D6000AE4F2046FAF782F9D7ED007AAC4AF5EE1D
:108D7000407AF1EE10FA0CBF012100212046FAF7EB
:108D800075F9A84943463A462046FAF71BFDA64B1B
:108D900005F5DC7205F5B7612046FAF721FF26B12B
:108DA00095F94A31002B00F02981A048FAF7C4F95F
:108DB0009F48FAF7BBF900239E4A9F4F9F4D02F54B
:108DC0009A612046FAF7B4FF9D4B9E4A01930092A8
:108DD0003A6829682046FBF7EFF940F202229A4BE5
:108DE00001930092BA68A9682046FBF7E5F9002EC6
:108DF00040F006819548FAF79FF93246944F95481E
:108E0000DFF8D4C20125002117F8013B10F8018BCF
:108E100003F1480EEE440EF8208C1CF801EB0EF125
:108E20004809E94409F8108C002D00F0EB80A3EB11
:108E30000E056B426B41013108291D46E4D183F0D8
:108E40000101002720468DF83070FAF781F9824A37
:108E50008DF840700EAB29462046FAF735FB7E4A66
:108E60000AAB29462046FAF701F97C4A7C4B02F509
:108E700036712046FAF786FD7A4A7B4B02F5367149
:108E80002046FAF7C7FD754A784B02F53671204641
:108E9000FAF708FE764B774A77492046FAF72CFB1B
:108EA000764A774B02F27C512046FAF727FC754A46
:108EB000754B02F27C512046FAF720FD734B744A41
:108EC00074492046FBF710F8734B744A74492046E6
:108ED000FAF7AAFF002E40F097807248FAF72CF9B3
:108EE000B346714DDFF8F481A5F5FF6700263946DA
:108EF0000222284647F0F4FA00285A4614BF0121FE
:108F00000021204695F800A00CBF4FF001094FF05A
:108F10000009FAF71DF9BAF1020F834640F0E0802C
:108F20007B784FF0190A40F2EE221AFB03230193DB
:108F30003B785E4A18F80330009349463346204692
:108F4000FAF7C2FA6B7840F2EE221AFB0323019380
:108F50002B78564A18F8033000934946334620468A
:108F6000FAF784F80136122E05F1020507F102071F
:108F7000BDD100214E4B02982246FCF70DF9210786
:108F800040F1C6800025E9B2029822460135FFF77C
:108F9000CBF9042DF7D1474F474D3B782B70059BFC
:108FA00033B94648FAF7C8F845490298FFF78CF9F3
:108FB000FF232B700026F1B2029822460136FFF7FC
:108FC00007FA042EF7D17B786B70059B002B40F0DD
:108FD0009C803C48FAF7B0F839490298FFF7C8F985
:108FE0003948FAF7A9F83948FAF734F8FF236B70D3
:108FF000002013B0BDE8F04FF7F74DBD0B4BDBE69B
:10900000124AFBE62B4616E7DFF898B069E700BF87
:10901000D8230608320C0708050D07088C2C002001
:109020000E0D07080C32002053FF06082C0C070811
:109030001D0D0708889A00204C2D0020E0330020E9
:109040002A0D0708FFFF7F00310D0708380C0708BD
:10905000C89F002098920608FAFE0608249D00206A
:1090600033020708A49D00203D0D0708380D0708AE
:10907000430D0708888E0020ECA00020E89B00200C
:10908000470D0708149D0020500D0708580D0708CC
:10909000248F0020A0A20020610D0708AC2D002025
:1090A000C83200203C0C0708BCA300201F0807089A
:1090B000430C0708B4320020A8050020650D0708FE
:1090C00065090708880D0708AF0D0708C50C0708D4
:1090D000D4330020842C0020488D002060940608A2
:1090E0003B781B4A18F80330009349463346204624
:1090F000FAF7EAF92B78164A18F803300093494634
:1091000033462046F9F7B2FF2CE7FF236B7097E553
:10911000104D029829782246FFF706F969780298DF
:109120002246FFF755F98BE5A20706D5094B0298B1
:1091300019782246FFF7F8F85AE763077FF558AF2A
:10914000044B029859782246FFF742F950E700BFD6
:109150002F080708B4320020224BB0F5FA6F1A68C6
:109160000346A8BF4FF4FA63B3F57A7FB8BF4FF454
:109170007A73D20416D540F2DC52904215D007EE35
:10918000903A40F2DB529042F8EE677A1FD8DFED5A
:10919000166A9FED167A9FED160A77EEE67AA7EE2D
:1091A000870A7047B0F57A7F02D89FED120A7047A0
:1091B00007EE903ADFED106A9FED107A9FED100AEE
:1091C000F8EE677A77EEE67AA7EE870A7047DFED6A
:1091D0000D6A9FED0D7A9FED0D0A77EEE67AA7EE08
:1091E000870A70472C2C002000007A44D62000C04B
:1091F00000E082440000000000407A446610004015
:109200000000404200A0BB44D62000400000834440
:10921000002310B409490A4C0A4A03704FF4EB7C4E
:1092200043822E23C0F80A40A0F806C05DF8044B24
:10923000C0F80210C0F80E20038170474A01B40044
:10924000C2010E0196004400704700BF0020704725
:10925000704700BF0020704701207047704700BF73
:10926000704700BF704700BF704700BF9FED010A05
:10927000704700BF0000000000207047064B1B78BD
:10928000834206D9054B00EB400003EBC00358694D
:1092900070470020704700BFD00500100C0500107B
:1092A000034B00EB400003EBC003587C704700BF4A
:1092B0000C050010024B1878003818BF01207047C9
:1092C000D005001003681B6903B11847704700BF41
:1092D00070B5094C236873B10546002606E099680D
:1092E0001A681E7321609047236823B15A68AA1A2E
:1092F000002A1846F3DA70BD0CAA00200B4B1A792D
:10930000D20700D570479A68002AFBD04FF47A71D3
:1093100001FB02F29042F5D3054A12781AB9054AC8
:10932000916812690A6000229A6070470CAA0020B6
:10933000282D0020A02B002070470022FFF75CBBE7
:109340000122FFF759BB2DE9F84F00261E4DDFF82B
:109350008090DFF880A007460C46B0462046FDF717
:1093600029FDD5F800B048B921465846F8F7B8FAB3
:1093700020B968682146F8F7B3FA80B15846F9F782
:1093800069FE696811B15046FAF7F0FFA96811B19A
:109390004846FAF7EBFFF9F765FE4FF00108013692
:1093A000362E05F11005D9D12046FDF703FD48B949
:1093B000B8F1000F06D1224638460449BDE8F84FFF
:1093C000FBF76CBFBDE8F88F48520608260E070869
:1093D000200E07081A0E0708F8B5354C2368002B35
:1093E00053D00A2801D00D284DD1324D2B7B0BB123
:1093F000F9F738FE304E2321304647F004F808B123
:10940000801B2060236800226BB902B12360F9F74A
:10941000F5FD2B7BEBB1BDE8F8402848F9F71ABE03
:1094200001220B46F0E7591E705C2028F8D08AB95B
:109430000022234C204FF2543726013E0CD13146F6
:10944000204B9C4211D2E368206898476B7B002B2D
:10945000DDD1F8BD2360EBE721683846FFF7ECF972
:1094600001460028ECD11034E7E72B7B23B11649E5
:109470001648FBF78DFDCAE71548F9F7EBFD0E48D6
:10948000F9F754FEC3E7FF2BE3D8A0F120025E2AD0
:10949000DFD80BB92028DCD05A1C2260064AD054F1
:1094A000044B1B7B002BD4D0BDE8F840FAF702B880
:1094B000949100200CAA002094900020EBF4060860
:1094C00048520608A85506083A0E0708560E07081F
:1094D0005C0E070808B5254B1B68DB040AD5B5EE02
:1094E000400AF1EE10FA12D19FED210A46F044FA3B
:1094F00080B208BDDFED1F7AB4EEE70AF1EE10FA94
:109500001CDA9FED1D0A46F037FA80B208BDDFED88
:10951000197AB4EEE70AF1EE10FAE5D49FED177A66
:10952000B4EEC70AF1EE10FA14D870EE677A9FED28
:10953000147A9FED140AA7EE870AE4E770EE677AC3
:109540009FED117A9FED110AA7EE870A46F014FAF3
:1095500080B208BDDFED0E7A9FED0E7A70EE677A6D
:109560009FED0D0AA7EE870ACDE700BF2C2C002047
:109570000080BB440000404200007A4400E0824486
:1095800066BEFFBE0060BB4438DFFF3E00407A4449
:109590000000834466BEFF3E00A0BB442DE9F843B3
:1095A000CE4B1E6816F004072DED048B40F01D8194
:1095B0009FEDCB8ACB4C16F0200605D094F8DC60EA
:1095C00016F0020640F0AA802379DFEDC78A94F8EE
:1095D0001C2113F0010340F0B680002A40F099806E
:1095E000D4ED487A9FEDC17ADFEDC16A67EE877AE4
:1095F00094ED4A7AE8EE267A38EE477AC4ED487A56
:1096000084ED497A66B1012284F81D2194F8302155
:10961000D4F8E030C4F82C31012A18BFC4F8243142
:10962000B44B93F80080B8F10D0F0BD1D4ED387A1C
:109630009FEDB17AB14B67EE877AFDEEE77A17EED0
:10964000902A9A809FEDA67AAD4DB0EE489A0023FD
:10965000D4ED4F7AD4ED506A94ED4E8A37EE677AA6
:10966000E6EE877A37EEC87AC4ED4F7AA6EE878A9F
:1096700085ED008A84ED4E8A0BB184ED498A94ED24
:10968000517AD4ED537ADFED9F5AD4ED546A94EDBC
:10969000520A84ED518A38EE477AB0EE676A97EE47
:1096A000256AE6EE867A37EEC07AC4ED537AA6EEE6
:1096B000870A84ED520A84ED550A46F05DF902B23C
:1096C00082EAE273A3EBE2739BB2092B40F2FB80C8
:1096D000002AACBF0A380A3005B2B8F10D0FA4F861
:1096E000585100F0CE80B8F1240F00F0E180B8F1BD
:1096F000380F05D1B0EE480A46F03EF97F4B98800E
:10970000BDEC048B002E18BF374684F85A71BDE8B3
:10971000F88384F81D3184F81C3161E7D4ED3B7A7D
:10972000B4F8F030F8EEE77AC4ED387A002B7CD14B
:10973000DFED6D8A237994F81C2113F001034FF0BB
:1097400001063FF44AAF002A67D0D4ED4A9A694B2C
:1097500094F81D9193F8008038EE699A002E49D054
:10976000B9F1000F73D094ED380AD4ED4B7A644D03
:1097700030EE670AB8F10D0F85ED000A07D1DFED75
:10978000627A20EE270A46F0F7F85C4B988094F84E
:109790003031002B40F0998095ED007A002F3AD0BF
:1097A00094F831319FED596A77EE487A06EE903A97
:1097B00077EEA97AF8EEE66AF0EEE77A67EEA67A37
:1097C0003B46F4EEC67AF1EE10FAC4BF28EE866A84
:1097D000C6EE278AF7EE007A77EEE87A67EE897AA6
:1097E000E8EE877AB0EE677A32E73E4C012794EDD7
:1097F000348AE0E6B8F10D0F37D0414DDFED388AFD
:10980000B9F1000FC3D1002F64D094F83031002B90
:109810005ED1B0EE497A01231AE7D4ED489A0123CC
:10982000C4ED4A9A84F81C3191E707EE903ADFEDD7
:10983000356A9FED377AF8EEE77AC6EEA78AF4EE3E
:10984000C78AF1EE10FA88BFF0EE478A72E7002F60
:1098500060D094ED380A70EE487A012377EEA97A49
:1098600084F81D31C4ED4B7A81E7254DDFED267A72
:1098700095ED000A20EE270A46F07EF81F4B9880EF
:10988000BCE7DFED207A9FED200ADFF8708068EEFC
:10989000A77A29EE000AFDEEE77A17EE903AA8F8CB
:1098A000003046F069F8A8F80650A8F8020027E74B
:1098B000DFED157A94ED490A20EE270A46F05CF8B0
:1098C0000E4B58801CE7002507E7022B02D00FB192
:1098D000012B9ED095ED007A0123B9E6A8910020D6
:1098E000000000000CAA00209A99993ECDCC4C3F74
:1098F000CDCC4C3E772200200AD7233C7822002092
:10990000E83100200000C842CDCCCC3D00401C46D0
:109910006666663FB8F10D0F064DDBD1DFED067AC6
:1099200095ED000A20EE270A46F026F8034B9880B2
:10993000D0E700BFE8310020CDCCCC3D782200201C
:10994000484B1B681B0600D47047F0B5464C2DED04
:10995000048BD4F8683185B013B104F5AE70984724
:109960000023CDE90033CDE90233D4F86C213F4820
:1099700069469047009BD4F88421BDF90460A4F89F
:1099800070619D1A03D105B0BDEC048BF0BD94F855
:109990008C219DED020A9DED039A002A5ED0B1EE66
:1099A000408AB4F88E21002A55D094ED657AD4ED22
:1099B000687A94ED666AD4ED696AD4ED678A38EE08
:1099C000478A79EE675AA6EE087AE6EEA57A94ED14
:1099D000648A84ED657A37EE485A77EEE85AA6EE47
:1099E000058AE6EEA58AC4ED687A84ED648AC4ED42
:1099F000678A1F4A84ED5D0A127884ED5E9A1C2AFC
:109A000084ED5F8AC4ED608AC4F88431BBD1DFED98
:109A1000199A20EE290A45F0AFFF29EE290A0446DB
:109A200045F0AAFF28EE290A074645F0A5FF0023C6
:109A30001A4666F30F0364F31F4367F30F020E4CDD
:109A400060F31F4228EEA90AC4E9003245F094FFF2
:109A50006581208197E7F0EE498ACAE7B0EE408A37
:109A60009FE700BFA89100200CAA002068AB00204F
:109A70007722002000007A4478220020AC4B1B683B
